:020000040000fa
:080000000abe0400000000002c
:020000040000fa
:10020000aa0d040000000000889fbe008004780052
:10021000124780000200e000020032000200780075
:100220000c003700408e200003003700918f5400ef
:10023000240036000180e800900078000100e00012
:10024000faff3a000f003700918f54001d0036006e
:100250000180e800900078000100e000faff3a0019
:1002600012017800408e200003003700918f540067
:10027000140036000180e80090007800828f500062
:10028000faff3a0008478000890f5400010031004e
:1002900009047800080078007c0007000000e000f6
:1002a00004003a00890f5400050032000804d10010
:1002b000f5ff37000818780041000700d4ff370029
:1002c0000000eb004f04be0000000600881f78000d
:1002d000630440000800a100800f54002300360092
:1002e000e30f540001003e004800200008007800a1
:1002f000c5ff0700800078000000e0001b0032000e
:10030000100178009201780064805100880f50003d
:1003100003003100120090008008780007003700c9
:1003200008004100800878009201900013009800b6
:100330001100780012081400080978009100780074
:100340000100e00005003200110090000000e00014
:10035000020032000180e800010037000000eb00dd
:10036000104788000280e800010037000000eb0021
:100370004f047800000006000004780006003700f3
:100380008200410040478000e10078000200e80060
:10039000304788000100010032478000504780004c
:1003a000800f5100f6ff3900808820004047880008
:1003b0002002200050478800080078003a0007001b
:1003c0000000e000300032008080e90091027800f7
:1003d000e38f52002c0036000508a3002a003a00e3
:1003e000224780000200e00002003200828f5000ad
:1003f0000400310002087800214788001600370009
:1004000003017800920190000300e0000200320036
:10041000818f5100faff3900120278000400410078
:10042000808f500018003900810f500003003a00ff
:100430000509420082007800070037000300e00051
:100440000300320005804000808f51000e0039000b
:100450009300980011019800110190000200e00043
:100460000900320011804000820f500006003a005f
:10047000e228ef001100900011017800900841007f
:100480001000900090009800000006000000e000be
:10049000030034000c000700e10f400001003a00a7
:1004a0000000eb00000006000c02e20004003d002a
:1004b0000f42ab00020032000f02ab00feff320021
:1004c0000040da00feff3700889fbe0080047800fd
:1004d000ee08e20004003a000000eb001000070004
:1004e0000000e0000a003500704780000900e000cd
:1004f00002003a000004780006003700000478008b
:1005000009004000060007000000e00001003d0077
:100510000084eb00080078004f04be0000000600d5
:10052000800078000000e00004003a00a05422009f
:100530007047880001017800060037000081eb0059
:1005400020612200808f500002003e007147880029
:100550000001eb0002007800000006001400fa0021
:100560000000eb00500798000000eb0040079800e7
:100570000000eb00300798001000200020079800d2
:100580006000b800008fbe006303070040c7bf00d3
:10059000614060000004e000020032004007a90052
:1005a0000000fe004f0907000000e8002007980047
:1005b0000000eb0040079800170037009d06070079
:1005c0000000eb00500798000c0037000000eb0023
:1005d00030079800030037003e0090000000e8005c
:1005e000300798003e009000e90f5000faff3600f7
:1005f0005e0090000000e80050079800de009000c8
:1006000070de2f00808f5000f0ff36004e0090000b
:100610000000e800400798004e009000e40f5000f2
:10062000e6ff36008000eb0080002000ad030700ed
:100630000000eb00500798000c0037000000eb00b2
:1006400030079800030037003e0090000000e800eb
:10065000300798003e009000e90f5000faff360086
:100660005e0090000000e80050079800de00900057
:1006700070de2f00808f5000f0ff36001100200048
:10068000800020009703070010c0b300250007007a
:1006900000000000070207000004e000fcff320039
:1006a0008d60a900a1e2a9008000eb00800020007d
:1006b0008c0307000000eb00500798000d00370086
:1006c0005e019000de009000008f20006140780005
:1006d0008000fb002e0090000088b9008040780068
:1006e000008f2000017178005e0090000000e8009b
:1006f00050079800de009000f0c12100808f50006c
:10070000efff36009a080700008f200001c2210089
:10071000a4080700704680000000e000fdff3a00da
:10072000f9ff37000200fa00004f780010c0b30054
:100730009e4f100004003a00c151220010c0b300c7
:100740008048780003003700c15122000040eb00d0
:10075000804878000000eb00001588000000eb00e6
:10076000101588000000eb00201588000000eb0049
:1007700030158800a802a800a822a800a842a90055
:10078000a862a900a882a900a8a2a900a8c2a900dd
:10079000a8e2a900a902a900a922a900a942a900ca
:1007a000a962a900a982a900a9a2a900a9c2a900b9
:1007b000a9e2a900aa02a900aa22a900aa42a800a7
:1007c000aa62a900aa82a900aaa2a900aac2a90095
:1007d000aae2a900ab02a900ab22a900ab42a90082
:1007e000ab62a900ab82a900aba2a900abc2a90071
:1007f000abe2a900112a200091407800c0cfb300dd
:1008000000c060000004a000a1e2b700a042a80060
:10081000012a20009140780000ceb30000c0700093
:10082000a0e2b700212a20009140780030ccb3002c
:1008300000c06000c041b300a2e2b700a342a8001c
:10084000512a20009140780000ceb30000c0600023
:100850000004a000a5e2b700c051220010407800bb
:100860000004e00005003200a4c2bf00f1c3b300e1
:1008700001407000a4e2b70007003700412a2000c1
:100880009140780000ccb30000c0600091c2b3007a
:1008900001407000a4e2b7008560a9008d60a80047
:1008a000a1e2a800c0512200104078000004e0003e
:1008b00001003a00000000000080fa00000006007d
:1008c000809fbe00829fbe003400f80000c0b300cd
:1008d000a00188000a00fa00a15122000040eb00ac
:1008e00080487800b15122000040eb008048780039
:1008f0008560a900c0512200104078000004e0008b
:100900001700320000282000000f7800b228810074
:100910001e007800100078004400de00804078005f
:10092000008f2000017178001e8fe800b028810040
:100930000000e800b0288900b1288100f0c1210042
:10094000808f50004d0136000000eb00b028890078
:10095000b151220010c0b300804878004701370031
:10096000c001200050158800212a20009140780005
:1009700030ccb30000c060000034a000a2e2b70099
:10098000412a20009140780000ccb30000c06000f4
:1009900091c2b30001407000a4e2b700e051220010
:1009a00010407800ec4f50000f003a00c00f2000bc
:1009b00050158800212a20009140780030ccb300e7
:1009c00000c060004041b300a2e2b700412a20000d
:1009d0009140780000ccb30000c060004041b300fb
:1009e000a4e2b70031003700e05122001040780047
:1009f000ed4f50002d003a00212a20009140780050
:100a000030ccb30000c060000044a000a2e2b700f8
:100a1000412a20009140780000ccb30000c0600063
:100a200051c2b30001407000a4e2b700d0512200cf
:100a3000104078000080fb00400798004e009000b6
:100a4000e10f5000110032004e009000e10f500005
:100a500004003c004e0090000000e000080032005e
:100a6000120037004e009000e20f50000a003200e2
:100a70004e009000e30f50000a0032000b003700d8
:100a8000c01121005015880008003700c021220045
:100a90005015880005003700c0412400501588001b
:100aa00002003700c081280050158800002820006f
:100ab000000f7800b22881001e0078001000780036
:100ac00080407800008f2000017178001e8fe800c0
:100ad000b02881000000e800b0288900b12881001a
:100ae000f0c12100808f5000020036000000eb00b2
:100af000b0288900e051220010407800ed4f5000ee
:100b000025003a00c02881000000e800c0288900c4
:100b1000c02881000000e000020032000000eb006d
:100b2000c0288900c22881001e00780010007800cb
:100b300080017800015122000200410001004000c4
:100b4000030878001e8fe800c22881001e0078008c
:100b5000100078008001780001512200020041005d
:100b6000010040000080e800030878001e8fe800c4
:100b7000c22881001e0078001000780080017800f3
:100b800001512200020041000100400064004000c9
:100b900003087800a5003700e051220010407800db
:100ba000ee4f500049003a00d0512200104078002a
:100bb0000080fb00300798003e009000e10f5000dd
:100bc0001b0032003e009000e10f500004003c008a
:100bd0003e0090000000e000080032009300370063
:100be0003e009000e20f50001e0032003e009000d8
:100bf000e30f5000280032008c0037001e00780000
:100c0000100078008000780000522200010878006f
:100c10001e8fe8001e007800100078008000780029
:100c20000052220041009800e2e2a8007f00370055
:100c30001e0078001000780080007800005222002a
:100c4000110098001e8fe8001e0078001000780048
:100c5000800078000052220051009800e302a800b2
:100c6000720037001e0078001000780080007800c5
:100c700000522200210098001e8fe8001e0078001c
:100c80001000780080007800005222006100980077
:100c9000e802a800650037001e0078001000780008
:100ca0008000780000522200310098001e8fe8007a
:100cb0001e007800100078008000780000522200aa
:100cc00071009800e822a80058003700e051220087
:100cd000104078000004e00054003a00d051220097
:100ce000104078000080fb00200798002e00900044
:100cf000e10f50001e0032002e009000e10f500066
:100d000004003c002e0090000000e00008003200cb
:100d1000460037002e009000e20f50002400320001
:100d20002e009000e30f5000310032003f003700ea
:100d30001e00780010007800800078000053220028
:100d4000010878001e8fe8001e007800100078006f
:100d5000800078000053220041009800e2e2a900e0
:100d6000d151220010c0b300804878002f00370016
:100d70001e007800100078008000780000532200e8
:100d8000110098001e8fe8001e0078001000780007
:100d9000800078000053220051009800e302a9006f
:100da000d151220020c0b300804878001f003700d6
:100db0001e007800100078008000780000532200a8
:100dc000210098001e8fe8001e00780010007800b7
:100dd000800078000053220061009800e802a9001a
:100de000d151220030c0b300804878000f00370096
:100df0001e00780010007800800078000053220068
:100e0000310098001e8fe8001e0078001000780066
:100e1000800078000053220071009800e822a900a9
:100e2000d15122000040eb0080487800e0512200c0
:100e300010407800304798000040eb0020479800b1
:100e40003e409000ee4f50000200360010c0b3004c
:100e5000204798003e4090008040e800e05122008a
:100e6000014878002e4090000004e00003003200aa
:100e7000e15122000040eb0080487800a15122009f
:100e800010c0b300804878000080fa003400f900f8
:100e90004f01be004f00be00004006000000fa00f7
:100ea000a0512200104078000080fb000080fa0072
:100eb000000006000000fa00b05122001040780047
:100ec0000080fb000080fa00000006000000fa002d
:100ed000a1e2a8000080fa00000006000000fa006d
:100ee000a1e2a9000080fa00000006000000fa005c
:100ef0000000eb008008880001112000914078007c
:100f0000f0ccb30000c0600010e1b7000000eb00bf
:100f100030088800205c20006008880084c0a90098
:100f20008cc0a80011e1a8000080fa0000000600b3
:100f30000000fa0011e1a9000080fa00000006009c
:100f40000800fa001007980021079800302a810055
:100f5000000f78000b0037001e007800b0009000f2
:100f60001e009000808f500003003a001100200006
:100f7000310798001f0037001e007800c000900065
:100f8000010f78001e00e000f3ff3a00a0002000ef
:100f9000cefc0700000f78001e00e00002003a00bf
:100fa00010002000f4fc0700ae0090001e00780046
:100fb000010878009e0078000000eb009000980087
:100fc0009e00780010c0b300c04098001e0078005a
:100fd0009e00900031009800312a81001e007800a8
:100fe000410098001e007800302a8900110020007e
:100ff000310798003e0090000080fa0000000600d3
:101000000800fa00200798000000eb001007980085
:10101000302a8100000f78001a0037001e00780087
:10102000b00090002e009000808f500010003a0019
:101030001e0090000000e000050032001e00780055
:10104000c00090001e00900041009800030037008f
:101050001e00780040009000302a89001e007800b1
:10106000d7fc070011002000310798000900370065
:101070001e007800100798001e007800c000900045
:10108000010f78001e00e000e4ff3a00200020007d
:10109000300798003e0090000080fa000000060033
:1010a0000800fa001007980021079800302a8100f4
:1010b000000f78000e0037001e007800b00090008e
:1010c0001e009000808f500006003a00ae00900095
:1010d0001e007800010878001100200031079800f8
:1010e000070037001e007800c0009000010f780054
:1010f0001e00e000f0ff3a002000200030079800ba
:101100003e0090000080fa00000006000600fa0091
:1011100010079800302a8100000f78000e00370079
:101120001e007800b00090001e009000808f5000dc
:1011300006003a009e0078000000eb009000980046
:101140001100200021079800070037001e007800da
:10115000c0009000010f78001e00e000f0ff3a0090
:1011600020002000200798002e0090000080fa0048
:10117000000006000600fa0010079800302a8100df
:10118000000f78000e0037001e007800b0009000bd
:101190001e009000808f500006003a009e007800ec
:1011a0000040eb00c040980011002000210798008b
:1011b000070037001e007800c0009000010f780083
:1011c0001e00e000f0ff3a002000200020079800f9
:1011d0002e0090000080fa00000006000600fa00d1
:1011e00010079800302a8100000f78000e003700a9
:1011f0001e007800b00090001e009000808f50000c
:1012000006003a009e00780010c0b300c04098006d
:101210001100200021079800070037001e00780009
:10122000c0009000010f78001e00e000f0ff3a00bf
:1012300020002000200798002e0090000080fa0077
:10124000000006003600f800809fbe00829fbe00ae
:10125000849fbe00869fbe003400f80000c0b3002b
:10126000a00188000200fa00302a8100000f7800f7
:1012700084c0a9001e0037001e0078004040900086
:10128000e14f500017003a001e007800100078006f
:101290000000e000130032001e00780010009000f3
:1012a0008000e8001e007800110098001e00780001
:1012b00010009000800078001e0078001000780078
:1012c0000000e900808f5000060036001e00780004
:1012d00030009000000001009e0078000000eb004c
:1012e000900098001e007800c0009000010f780068
:1012f0001e00e000e0ff3a000080fa003400f90030
:101300004f03be004f02be004f01be004f00be00a3
:101310003600f900004006000000fa00c4c2a9002f
:10132000c4e2a900c522a900c582a900c542a9003e
:10133000c5a2a900c5c2a900c5e2a900c0c2a900f2
:10134000c0e2a900c122a900c182a900c142a9002e
:10135000c1a2a900c1c2a900c1e2a900d022a9006e
:10136000cc22a900d042a900cc42a900e2e2a90007
:10137000e302a900e802a900e822a900dee2a90030
:10138000df02a900e402a900e422a900e202a90008
:10139000de02a900d602a900d622a900d642a900e1
:1013a000d662a900d682a900d6a2a900d6c2a900f9
:1013b000d6e2a900d202a900d222a900d242a900f5
:1013c000d262a900d282a900d2a2a900d2c2a900e9
:1013d000d2e2a900d1a2a900cda2a900e842a900a9
:1013e000e862a900e442a900e462a900de22a800a4
:1013f000dec2a800e4c2a800e4e2a800e502a8005a
:10140000e522a800d302a800d322a800d342a80056
:10141000d362a800d382a800d3a2a800d3c2a80098
:10142000d3e2a8000080fa00000006000c22ef00c2
:101430000e22ef000ee2a9000ec2a9008520a9002d
:101440008d20a8000de2a80070002000a0108800e8
:101450008540a9008d40a80081e0a900c00480005b
:10146000f1002f0000806000015520000080400046
:10147000c00488000fe2a8000f42a8004028ef0037
:101480004228ef00000006001622ef001822ef00ad
:1014900018e2a90018c2a9008700a9008f00a800bf
:1014a00017e2a80070002000f01088008720a90033
:1014b0008f20a80081e0a9000005800001f02f0026
:1014c0000080600051052000008040000005880079
:1014d00019e2a8001942a8008428ef008628ef002e
:1014e000000006000600fa00000f780011079800bf
:1014f0001e007800200798002e009000e30f500097
:10150000670032002e009000e30f500007003e00fd
:101510002e009000e10f50002e0032002e009000af
:10152000e10f500041003e000d0037002e009000fa
:10153000e50f5000940032002e009000e50f50009f
:10154000740039002e009000e60f5000ab0032000e
:101550002e009000e70f5000c5003200da0037007f
:101560001e009000e10f50000f003600c4c2bf0003
:101570000080fb004600de00614060000004a20025
:1015800061406000614060004601dd00412c2000a8
:1015900091407800f0cbb30000c0600002407000c2
:1015a000c4e2b7001e0137001e00900061406000d9
:1015b000614060004601dd00412c20009140780030
:1015c000f0cbb30000c0600002407000c4e2b7007e
:1015d000130137001e009000e10f50000b00360091
:1015e000c4c2bf000080fb004700de000004a20070
:1015f00061406000c700dd00c4c2bf000074a100ec
:1016000001407000c4e2b700050137001e009000e1
:1016100061406000c700dd00c4c2bf000074a100cb
:1016200001407000c4e2b700fd0037001e009000ca
:10163000e10f50000f003600c5c2bf000080fb0064
:101640000000d100614060000004a2006140600021
:101650006140600000414000512c20009140780022
:10166000d0cfb30000c0600002407000c5e2b700f8
:10167000eb0037001e009000614060006140600098
:1016800000414000512c200091407800d0cfb300a1
:1016900000c0600002407000c5e2b700e000370003
:1016a0001e009000e10f50000f003600c5c2bf00c1
:1016b0000080fb004400de00614060000004a200e6
:1016c00061406000614060004401dd00512c200059
:1016d00091407800f0ceb30000c06000024070007e
:1016e000c5e2b700ce0037001e00900061406000e8
:1016f000614060004401dd00512c200091407800e1
:10170000f0ceb30000c0600002407000c5e2b70038
:10171000c30037001e009000e10f50000f0036009c
:10172000c5c2bf000080fb004200de0061406000d7
:101730000004a20061406000614060004201dd00e1
:10174000512c200091407800b0cfb30000c0600061
:1017500002407000c5e2b700b10037001e009000e3
:1017600061406000614060004201dd00512c2000ba
:1017700091407800b0cfb30000c06000024070001c
:10178000c5e2b700a60037001e009000e10f500030
:101790000f003600c5c2bf000080fb004500de0020
:1017a000614060000004a200614060006140600090
:1017b0004501dd00512c200091407800f0cdb300b0
:1017c00000c0600002407000c5e2b700940037001e
:1017d0001e00900061406000614060004501dd0036
:1017e000512c200091407800f0cdb30000c0600083
:1017f00002407000c5e2b700890037001e0090006b
:10180000e10f50000f003600c5c2bf000080fb0092
:101810004600de00614060000004a20061406000fc
:10182000614060004601dd00512c200091407800ad
:10183000f0cbb30000c0600002407000c5e2b7000a
:10184000770037001e00900061406000614060003a
:101850004601dd00512c200091407800f0cbb30010
:1018600000c0600002407000c5e2b7006c003700a5
:101870001e009000e10f50000b003600c5c2bf00f3
:101880000080fb004700de000004a2006140600011
:10189000c700dd00c5c2bf000074a1000140700098
:1018a000c5e2b7005e0037001e0090006140600096
:1018b000c700dd00c5c2bf000074a1000140700078
:1018c000c5e2b700560037001e009000614060007e
:1018d000c700dd00c5c2bf000074a1000140700058
:1018e000c5e2b700c5c2bf000080fb004700de00b4
:1018f000614060004601dd00512c200091407800dd
:10190000f0cbb30000c0600002407000c5e2b70039
:10191000c5c2bf000080fb004600de0061406000e1
:10192000614060004501dd00512c200091407800ad
:10193000f0cdb30000c0600002407000c5e2b70007
:10194000c5c2bf000080fb004500de0061406000b2
:10195000614060004201dd00512c20009140780080
:10196000b0cfb30000c0600002407000c5e2b70015
:10197000c5c2bf000080fb004200de006140600085
:10198000614060004401dd00512c2000914078004e
:10199000f0ceb30000c0600002407000c5e2b700a6
:1019a000c5c2bf000080fb004400de006140600053
:1019b0006140600000414000512c200091407800bf
:1019c000d0cfb30000c0600002407000c5e2b70095
:1019d000c5c2bf000080fb000000d1006140600074
:1019e000c700dd00c4c2bf000074a1000140700048
:1019f000c4e2b700c4c2bf000080fb004700de00a5
:101a0000614060004601dd00412c200091407800db
:101a1000f0cbb30000c0600002407000c4e2b70029
:101a20000080fa00000006000000fa00c4c2a9000d
:101a3000c4e2a900c522a900c582a900c542a90027
:101a4000c5a2a900c5c2a900c5e2a9000080fa008c
:101a5000000006000200fa00000f780010002000cd
:101a60009e0f10000f003600d0c2bf000080fb00a8
:101a70004200de00614060000004a200614060009e
:101a8000614060004201dd00012d2000914078009e
:101a9000b0cfb30000c0600002407000d0e2b700d9
:101aa0000a0037001e00780061406000614060005d
:101ab0004201dd00012d200091407800b0cfb3003d
:101ac00000c0600002407000d0e2b7000080fa0061
:101ad000000006000200fa00000f7800100020004d
:101ae0009e0f10000f003600d0c2bf000080fb0028
:101af0000000d100614060000004a200614060006d
:101b00006140600000414000012d200091407800bc
:101b1000d0cfb30000c0600002407000d0e2b70038
:101b20000a0037001e0078006140600061406000dc
:101b300000414000012d200091407800d0cfb3003b
:101b400000c0600002407000d0e2b7000080fa00e0
:101b5000000006000000fa00c4c2bf000080fb00c5
:101b60004600de006140600000c0ea0061406000a5
:101b7000614060004601dd00412c2000914078006a
:101b8000f0cbb30000c0600002407000c4e2b700b8
:101b9000c4c2bf000080fb004700de0000c0ea00b6
:101ba00061406000c700dd00c4c2bf000074a10036
:101bb00001407000c4e2b700c5c2bf000080fb0056
:101bc0000000d1006140600000c0ea006140600098
:101bd0006140600000414000512c2000914078009d
:101be000d0cfb30000c0600002407000c5e2b70073
:101bf000c5c2bf000080fb004400de006140600001
:101c000000c0ea0061406000614060004401dd0006
:101c1000512c200091407800f0ceb30000c060004d
:101c200002407000c5e2b700c5c2bf000080fb00e3
:101c30004200de006140600000c0ea0061406000d8
:101c4000614060004201dd00512c2000914078008d
:101c5000b0cfb30000c0600002407000c5e2b70022
:101c6000c5c2bf000080fb004500de00614060008f
:101c700000c0ea0061406000614060004501dd0095
:101c8000512c200091407800f0cdb30000c06000de
:101c900002407000c5e2b700c5c2bf000080fb0073
:101ca0004600de006140600000c0ea006140600064
:101cb000614060004601dd00512c20009140780019
:101cc000f0cbb30000c0600002407000c5e2b70076
:101cd000c5c2bf000080fb004700de0000c0ea0074
:101ce00061406000c700dd00c5c2bf000074a100f4
:101cf00001407000c5e2b7000080fa000000060055
:101d00000000fa00c4c2bf000080fb004600de00f5
:101d10006140600000c0ea00614060006140600016
:101d20004601dd00412c200091407800f0cbb3004b
:101d300000c0600002407000c4e2b7000080fa00fa
:101d4000000006000000fa00c4c2bf000080fb00d3
:101d50004700de0000c0ea0061406000c700dd000f
:101d6000c4c2bf000074a10001407000c4e2b7000b
:101d70000080fa00000006000000fa00c5c2bf00a3
:101d80000080fb000000d1006140600000c0ea005c
:101d9000614060006140600000414000512c200023
:101da00091407800d0cfb30000c0600002407000c6
:101db000c5e2b7000080fa00000006000000fa004b
:101dc000c5c2bf000080fb004400de00614060002f
:101dd00000c0ea0061406000614060004401dd0035
:101de000512c200091407800f0ceb30000c060007c
:101df00002407000c5e2b7000080fa000000060053
:101e00000000fa00c5c2bf000080fb004200de00f7
:101e10006140600000c0ea00614060006140600015
:101e20004201dd00512c200091407800b0cfb3007a
:101e300000c0600002407000c5e2b7000080fa00f8
:101e4000000006000000fa00c5c2bf000080fb00d1
:101e50004500de006140600000c0ea0061406000b3
:101e6000614060004501dd00512c20009140780068
:101e7000f0cdb30000c0600002407000c5e2b700c2
:101e80000080fa00000006000000fa00c5c2bf0092
:101e90000080fb004600de006140600000c0ea00f8
:101ea00061406000614060004601dd00512c20006f
:101eb00091407800f0cbb30000c060000240700099
:101ec000c5e2b7000080fa00000006000000fa003a
:101ed000c5c2bf000080fb004700de0000c0ea0072
:101ee00061406000c700dd00c5c2bf000074a100f2
:101ef00001407000c5e2b7000080fa000000060053
:101f00000200fa00000f78009e007800a0da20009e
:101f10000bfc07000080fa00000006000000fa0039
:101f2000a0da200036fc07000080fa00000006005e
:101f30000200fa00000f78001e00e00003003500e8
:101f40009e007800a0da200055fc07000080fa000f
:101f5000000006000000fa00005422001040780043
:101f60000004e0000e003a008000eb00700020004a
:101f70005cfd070000542200104078000080fb0048
:101f80001100200057fd0700005422001040780087
:101f90008040e80000542200014878002300370008
:101fa0000054220010407800e74f50000f003a0024
:101fb00000542200104078000080fb000000e9007f
:101fc0008000eb0047fd070000542200104078001d
:101fd0000080fb001100200042fd07000154220098
:101fe0000040eb00804878001000370000542200c9
:101ff000104078000080fb000000e9008000eb004a
:1020000038fd070000542200104078000080fb00db
:102010001100200033fd070000542200104078001a
:102020008040e80000542200014878000080fa0057
:10203000000006000200fa00105422001040780050
:102040000080fb00000f78001e007800e20f5000b7
:102050001c0032001e007800e20f500007003c0018
:102060001e0078000000e0000b0032001e00780027
:10207000e10f50000c003200230037001e007800f2
:10208000e30f5000160032001e007800e40f5000ed
:102090001a0032001c003700210020000000eb0075
:1020a00010fd07001800370021002000100020005c
:1020b0000cfd0700210020007000200009fd070032
:1020c00011003700210020002000200005fd07003e
:1020d000210020006000200002fd07000a003700f8
:1020e0002100200030002000fefc0700210020001d
:1020f00050002000fbfc07000300370021002000f7
:1021000040002000f7fc0700105422001040780027
:10211000e34f500006003e001054220010407800ab
:102120008040e80010542200014878000300370086
:10213000115422000040eb00804878000080fa0033
:10214000000006000000fa00205422001040780031
:102150000004e00013003a00805422001040780090
:102160000004e0000f0032002154220010c0b30030
:10217000804878008000eb000000eb00d9fc0700ed
:1021800020542200104078000080fb001100200045
:10219000d4fc0700815422000040eb008048780006
:1021a0003600370020542200104078000004e00080
:1021b00013003a0080542200104078000004e00030
:1021c0000f003a002154220070c0b300804878000c
:1021d0008000eb000000eb00c2fc0700205422004e
:1021e000104078000080fb0011002000bdfc0700bb
:1021f0008154220010c0b300804878001f003700cf
:102200002054220010407800e74f50000c003a00a4
:10221000215422000040eb00804878008000eb0051
:1022200070002000affc070020542200104078000e
:102230000080fb0011002000aafc07000f003700ff
:102240002054220010407800e14f50000b003a006b
:10225000215422000040eb00804878008000eb0011
:10226000100020009ffc070020542200104078003e
:102270000080fb00110020009afc07000080fa009b
:10228000000006000200fa003054220010407800de
:102290000080fb00000f78001e007800e10f500066
:1022a000150032001e007800e10f500004003c00d1
:1022b0001e0078000000e000080032001a0037001d
:1022c0001e007800e20f5000120032001e0078005d
:1022d000e30f5000130032001300370021002000ec
:1022e0000000eb007ffc07002100200040002000e0
:1022f0007cfc07000c0037002100200010002000ab
:1023000078fc0700210020003000200075fc070049
:1023100005003700210020002000200071fc07008c
:1023200001003700c0fd0700305422001040780043
:10233000e24f500006003e0030542200104078006a
:102340008040e80030542200014878000300370044
:10235000315422000040eb00804878000080fa00f1
:10236000000006000200fa004054220010407800ed
:102370000080fb00000f78001e007800e10f500085
:10238000150032001e007800e10f500004003c00f0
:102390001e0078000000e000080032001a0037003c
:1023a0001e007800e20f5000120032001e0078007c
:1023b000e30f50001300320013003700210020000b
:1023c0000000eb0047fc0700210020004000200037
:1023d00044fc07000c0037002100200070002000a2
:1023e00040fc070021002000500020003dfc0700b9
:1023f00005003700210020006000200039fc0700a4
:102400000100370088fd070040542200104078008a
:10241000e24f500006003e00405422001040780079
:102420008040e80040542200014878000300370053
:10243000415422000040eb00804878000080fa0000
:1024400000000600809fbe008520a9000042800099
:10245000f003b20001802000810040000000eb008a
:1024600012c2bf00804878004028ec004f00be0038
:102470000040060000428000114280000100500030
:102480000000060001428000124280000208e100c4
:1024900008003200f203b2000180200002814000f7
:1024a00092407800014878004228ec00100020009b
:1024b000000006000000eb00000006008540a900b7
:1024c000809fbe00821f7800d808e200150032000d
:1024d000d408e20016003200d608e20014003200f0
:1024e000a1468000420020000f22af00feff37000f
:1024f000b04680000000e000070032000000e90064
:10250000d6a8b7003140780010e2b7000201e90018
:10251000f5ff3a0002003700d428ef000100370031
:10252000a14688004f0178004f00be000040060021
:1025300000002000c04688004f0178004f00be0018
:1025400000400600d808e200feff3a008d40a900d6
:102550008100e900b1468800b04078008110880011
:10256000a046880011002000c14688008d40a800c8
:1025700000000600c046800000000600809fbe00ec
:102580008700a90020448000f003b20041842000ad
:10259000810040000000eb001cc2bf0080487800b2
:1025a0008428ec004f00be0000400600204480005c
:1025b00031448000010050000000060021448000ea
:1025c000324480000208e10008003200f203b20049
:1025d0004184200002814000924078000148780048
:1025e0008628ec0010002000000006000000eb0030
:1025f000000006008720a900809fbe00821f78008f
:10260000de08e20015003200da08e20016003200af
:10261000dc08e20014003200d146800042002000b5
:102620001922af00feff3700e04680000000e00006
:10263000070032000000e900dca8b7003140780054
:102640001ae2b7000201e900f5ff3a000200370084
:10265000da28ef0001003700d14688004f017800ea
:102660004f00be000040060000002000f046880039
:102670004f0178004f00be0000400600de08e20077
:10268000feff3a008f20a9008100e900e1468800a2
:10269000b0407800d1108800d0468800110020009a
:1026a000f14688008f20a80000000600f046800058
:1026b00000000600811f7800801f7800f0ff2700cf
:1026c000c0128800003020000000b300d012880043
:1026d000de02a90000000000e002a900900109004c
:1026e00000000000e002a80041e2a8004602ae009f
:1026f000feff3700f0ff2700c012880000402000d6
:102700003001b300d01288004602ae00feff370051
:10271000f0ff2700c0128800001020000030a00049
:102720000040a000d01288004602ae00feff370035
:10273000f0ff2700c012880000202000d01288007f
:102740004602ae00feff3700f0ff2700c0128800ef
:10275000006020000010a000d01288004602ae00e9
:10276000feff3700f0ff2700c01288000070200035
:10277000f005b300d01288004602ae00feff37001d
:1027800001f0200030128000010060000000e00035
:10279000fcff3a0030128000010060000000e00001
:1027a000fcff320030128000010060000000e000f9
:1027b000fcff3a0030128000010060000000e000e1
:1027c000fcff32004662ae0002003700801280003b
:1027d0009012800041e2a900f01e20001012880033
:1027e0004362a8004342a8008920a900a8c0a8000d
:1027f000a8a0a900a880a9009120a80041e2a800f3
:102800004f007800cf00780000000600801f78009d
:102810004022ef004222ef004422ef004822ef0066
:102820004c22ef00c6e2a800e5a2a900e582a800bc
:10283000e5e2a900e5c2a9004002a9004022a900e2
:1028400040a2a9004122a90040c2a8004102a9005b
:102850004142a900f00e2000101288004362a90036
:102860004342a80070002000201288004c02a800fb
:102870004802a8008920a9009120a90041e2a900ee
:102880004f007800000006008920a900809fbe004c
:10289000829fbe008012800090128000a0128000f3
:1028a000b0128000cc08e2002c003a00d008e20010
:1028b0002a0032006147800011007800f00fb2005a
:1028c0004800dd000000a100c01288000000eb00fd
:1028d000110078000000a1000010a1000020a1005c
:1028e0000030a1000040a1000050a1000060a10044
:1028f0000070a100d01288008180e8000000eb0089
:1029000011007800f00fb2004800dd000000a100c7
:10291000e01288000000eb00110078000000a10028
:102920000010a1000020a1000030a1000040a10083
:102930000050a1000060a1000070a100f01288000a
:102940008180e800d0a8ed00d0a8ed0061478800a4
:102950004f01be004f00be0000400600ce28ef0031
:10296000cca8ef004f01be004f00be0000400600a3
:102970000200fa00e202a8000000eb00000f78005d
:10298000010037001e0fe800f07022009e0f1000bb
:10299000fcff34009dff070046ff07000080fa009f
:1029a000000006000400fa00000f780011079800ec
:1029b000cea8ef00cc28ef009e0090001e0078000b
:1029c000060007000080fa00000006000000fa0080
:1029d000e202a9000080fa0000000600811f7800d2
:1029e000821f7800030037004f017800cf00780085
:1029f00000000600814688000001eb00800078009e
:102a000011007800f00fb2004800dd000000a100c6
:102a1000c01288000000eb00110078000000a10047
:102a20000010a1000020a1000030a1000040a10082
:102a30000050a1000060a1000070a100d012880029
:102a40008180e8000000eb0011007800f00fb20078
:102a50004800dd000000a100e01288000000eb004b
:102a6000110078000000a1000010a1000020a100ca
:102a70000030a1000040a1000050a1000060a100b2
:102a80000070a100f01288008180e800d0a8ed005d
:102a9000d0a8ed00614788008920a900d2ff370047
:102aa0000800fa0020079800310798006000b8007d
:102ab000008fbe000400370010002000010020003d
:102ac0001e0f40005e9748002e009000be00900050
:102ad000be0f1000ae8f1800f7ff35000080fa001f
:102ae000000006000000fa00e6c2bf000080fb0004
:102af0004600de00614060000081fb00e7c2bf00cd
:102b00000080fb000000d100614060000080fb00fd
:102b10000000400080007800e7c2bf006140600014
:102b20000080fb0000804000000040008000780032
:102b3000e6c2bf000080fb004700de000080fb0013
:102b40000080400000004000000041000080fa00ca
:042b5000000006007b
:020000040000fa
:0200000401f009
:04000000e6ff000017
:020000040000fa
:0200000401f009
:04000400ff7f00007a
:020000040000fa
:0200000401f009
:040008007fff000076
:020000040000fa
:0200000401f009
:04001400ffff0000ea
:020000040000fa
:100008008abe00008abe00008abe00008abe0000c8
:100018008abe00008abe00008abe00008abe0000b8
:100028008abe00008abe00008abe00008abe0000a8
:100038008abe00008abe0000220900008abe0000b5
:100048008abe0000221200005e1200006004000058
:100058008abe00008abe00008abe00008abe000078
:100068008abe00008abe00008abe00008abe000068
:100078008abe00008abe00008abe00008abe000058
:10008800be120000fa1200008abe00008abe0000fc
:100098008abe00008abe00008abe00008abe000038
:1000a8008abe00008abe00008abe00008abe000028
:1000b8008abe00008abe00008abe00008abe000018
:1000c8008abe0000441400008abe00008abe0000f8
:1000d8008abe00008abe00008abe00008abe0000f8
:1000e8008abe00008abe00008abe00008abe0000e8
:0800f8008abe00008abe000070
:020000040000fa
:100108008abe00008abe00008abe00008abe0000c7
:100118008abe00008abe00008abe00008abe0000b7
:100128008abe00008abe00008abe00008abe0000a7
:100138008abe00008abe0000220900008abe0000b4
:100148008abe0000221200005e1200006004000057
:100158008abe00008abe00008abe00008abe000077
:100168008abe00008abe00008abe00008abe000067
:100178008abe00008abe00008abe00008abe000057
:10018800be120000fa1200008abe00008abe0000fb
:100198008abe00008abe00008abe00008abe000037
:1001a8008abe00008abe00008abe00008abe000027
:1001b8008abe00008abe00008abe00008abe000017
:1001c8008abe0000441400008abe00008abe0000f7
:1001d8008abe00008abe00008abe00008abe0000f7
:1001e8008abe00008abe00008abe00008abe0000e7
:0801f8008abe00008abe00006f
:020000040000fa
:102b540006000000260000001f0000001200000014
:102b640027000000180000001c0000002d000000d9
:102b740041000000fd000000e500000032010000fb
:102b84008b0200001e0200004400000024ff00002d
:102b9400b8fe0000bdfe00003dff000027ff00005e
:102ba4003dfe000026fe00009efc0000dcf9000053
:102bb4003bfe0000c908000044100000d60e0000cf
:102bc4009405000033fb00005ff600008ff700005f
:102bd4008afa00008afb0000a3fa0000a1fb0000af
:102be40021010000e7080000a60d00001a0c0000f7
:102bf400bb03000046fb0000a9f80000d3f9000065
:102c040037fd00004aff00005afe0000c3fd00002b
:102c1400d6ff0000f90300002c060000d8010000d4
:102c2400d0f8000029f80000cf030000ff0f0000d7
:102c34007f110000d406000014f9000088f200009f
:102c4400ddf5000006fd00007a0000009ffd000095
:102c540059fa000033fd000016060000d30d0000f1
:102c6400b20d0000ec04000025f9000007f5000097
:102c74009bf8000020ff0000150300000001000085
:102c8400adfd0000e6fd0000a702000027070000dc
:102c94008703000013f7000027f100003dfd00004a
:102ca400bd100000b41900009e100000f7fd0000e4
:102cb400c3f00000d8f000003ff900003bff000023
:102cc400b2fc000016f7000030f80000c601000056
:102cd400a20d0000211300003a0d0000a501000020
:102ce400acf8000082f5000006f9000051fd000078
:102cf40048fd000002fb0000f7fa0000c9ff0000d5
:102d0400d70600002e0700001afd00004bf6000055
:102d14002dff0000980f0000d21600009b0d00004c
:102d2400a4fb000013ef0000a5ef00005ff8000013
:102d340010ff00009efd000076f900007dfa0000ff
:102d440021010000390b0000b112000050100000f6
:102d54001006000049fa0000bbf20000edf3000089
:102d640083f9000095fc000066fc0000c6fb00002f
:102d740015ff00003005000078040000befc0000d0
:102d840022fb00003006000051130000be130000b7
:102d9400bf050000a0f40000beec0000cbf0000072
:102da4003bf9000017fd00004ffa000009f900008c
:102db4007cfc00008e030000790d0000db12000093
:102dc400470e0000c7010000c8f40000b1ef000086
:102dd400e5f300002cfa000026fc00001dfb0000b7
:102de400d7fa00005e00000017060000d4010000be
:102df40011fa0000f6fc0000120c00003617000067
:102e04009511000010ff000067ee0000e5ea0000e5
:102e14005ef200002afb000032fc0000abf8000068
:102e240087f900007bfe00002708000098130000cb
:102e340000160000000d0000c8fd00004cf000006a
:102e440057ed0000c0f30000e1f90000cffb0000e3
:102e540077fa000065fc00001d04000098060000dd
:102e6400ea00000094fd000044070000b4140000d0
:102e74008d1400003204000080f0000075e80000aa
:102e840049ee00001df90000defd00009afa000082
:102e9400f2f9000009fe0000ec0400007a0f0000c3
:102ea4007c1500000d1200004c050000ebf400003e
:102eb400d3eb00000fef000015f70000e4fb000067
:102ec400d8fb0000d8fa00008d0100005c07000068
:102ed40079050000ef010000450600006b110000b9
:102ee400d1130000d40600006df3000041e9000096
:102ef40040ed00005df8000088ff000070fd000058
:102f04004bfc00005eff0000fe020000f10900001f
:102f1400dc110000fa1500000a0f0000d5fd0000c6
:102f240021ee00002aeb0000e7f2000006fb00009f
:102f3400a4fd0000dffa000071fe00009805000007
:102f4400cc0800008a0a0000b80b0000f50e00004f
:102f5400d40d0000020300002af400008cec0000f1
:102f64009fef000020f8000077ff0000feff000044
:102f740050010000ca030000ee010000100200002e
:102f8400e7090000ab160000bd180000ff080000b0
:102f9400daf20000b5e7000046ed00000df900008c
:102fa400a0ff00002cfc000085fa00008601000050
:102fb40060080000780f0000d9120000e81000003b
:102fc400ae0a0000bffe0000daf2000031ee00009d
:102fd40047f2000040f8000091fd0000f3fe0000fd
:102fe400c8020000890800009405000028000000c1
:102ff400bf0100003a0f0000181a0000db110000a6
:103004000cfb00008ee800002ae800005ff40000da
:10301400deff00009bff0000bcfa000037fe00004a
:10302400fe030000eb0a0000d31000003c13000074
:10303400ea1000000c05000059f5000042ec000005
:103044000fef000001f60000c1fb000026fc0000a9
:10305400d9fd000011060000b908000011080000a5
:1030640034070000850a000086100000630c00008d
:10307400c9fc00000aed0000cee90000bef100002a
:10308400fdfc0000530100005cff00000102000091
:10309400af02000067020000190700002d0f0000b6
:1030a400e31500001c0f000057fc0000eceb0000cf
:1030b400c0e9000065f2000030fb00001dfd0000c7
:1030c40016fa0000c4ff00004f0700003809000092
:1030d400070b0000a90b0000e90d0000950b000090
:1030e40065ff0000ebf00000ffea000058ef00006d
:1030f400c1f7000087fe0000b8fe00005d0200007a
:10310400b70600000a040000f70200005906000098
:10311400ca0f0000251400003c0800002ff4000032
:1031240050e80000d7eb0000a7f60000a7fe00005f
:1031340024fd000006fc0000230300002306000019
:10314400430700009d090000110e0000b6110000a5
:103154004c09000040f800004deb000001eb0000ba
:10316400c6f2000032fb000078fd000085fd00007f
:10317400d4040000ff07000041070000cf0800004e
:103184000e0b0000f60e00007a0a0000b5fb0000ea
:10319400d3ed0000e9ea0000fff1000027fb000086
:1031a40001000000b6fe00002d0300000807000027
:1031b40058030000dc020000870700005f110000d4
:1031c4001014000081060000f5f20000ade80000d4
:1031d400eeec00008bf70000f8fe000096fd000006
:1031e400f4fd0000c7050000d1070000e20700005d
:1031f40046090000900c000027100000c1080000e0
:1032040011f900009eec0000d1eb0000c4f30000b3
:1032140047fd0000d1000000d4ff0000300500008d
:103224001807000097040000a605000089080000a4
:10323400ab0e0000810e00005902000019f30000db
:1032440026ec00008ff00000f5f900008200000079
:10325400fefe0000deff00003c0500001a04000032
:103264002c030000bf060000330e00008913000089
:10327400fb0b0000cffa0000e0ec000072eb000052
:10328400c3f3000016fd00008dff00005ffd000089
:10329400af020000d60700002f060000e60500007c
:1032a40039080000e00c0000640d0000da0300009f
:1032b400daf50000dfed0000b3f0000038f900009b
:1032c4001d000000fffe00002afd00004102000076
:1032d4009d0300000a030000eb060000b70b00008a
:1032e4001f0f0000fb0b000066ff0000baf2000095
:1032f40083ef00006cf40000c2fa0000a5fc00009b
:103304007bf900003bfc00008a05000096060000e3
:10331400c403000037060000310c00006d100000eb
:10332400c00a0000b8fb000080ef000016ee0000a9
:10333400e0f4000092fb00004cfc0000f1f80000f7
:10334400b2fd0000c50700004c0700000a0300009e
:1033540077040000540b00007d100000cc0900002d
:10336400cbfa0000f9ef000099ef00001df6000011
:1033740040fb000068fa00005af700008afd0000d4
:103384002e0800005808000017040000b1040000d3
:10339400440a0000750e0000220900002dfc000004
:1033a40072f10000e1ef00005bf50000ccfa0000d0
:1033b400a4fb00007df90000e6fe0000d907000030
:1033c400e50600005602000080030000c909000061
:1033d400f30d0000dc09000001ff000081f500008e
:1033e4000df2000028f40000a3f80000ccfa00005d
:1033f400b5f90000aefd000075060000e606000009
:1034040065010000c50100003d0a00003d110000f7
:10341400bd0e0000e901000093f4000077ef000006
:1034240062f200005ef8000069fa0000f9f800009a
:10343400ccfb00002d070000240d000088060000ce
:103444001b010000a7030000ba0800001d0c0000c7
:10345400650700009bfb00005ef20000def0000048
:1034640054f7000074fe000031ff000046fb00002a
:103474006afe0000c0040000ec02000087ff0000a8
:1034840082040000090e0000aa120000530e00007e
:10349400a5000000e8f3000011ef0000e6f10000d1
:1034a400a7f7000032fa000003fa0000a0fe0000b3
:1034b400450a0000f90c0000de02000024fd0000b3
:1034c40040040000490e0000da1000006e080000fd
:1034d400f7f90000d3f00000a0f00000f5f60000ba
:1034e400dafc000072fd0000c0fb00005401000083
:1034f400c50a0000180800004afe000030fd000064
:1035040026070000de1000009d11000029070000be
:10351400a1f800007bf0000003f20000d2f80000e4
:10352400c1fb0000faf90000f6f900007f04000076
:10353400cb0e0000f6080000b9fd000063fe000099
:10354400ec080000f40e0000510c000074020000ae
:10355400cef70000d6f200000bf5000088fa000058
:10356400c6fb0000bbf9000037fa00002905000083
:103574001a0e000084050000f1f9000087fd000028
:10358400c30c00001e150000580f00000d000000c1
:10359400d0f2000083ef000057f40000c2fa0000ec
:1035a40009fb000091f80000e6fa0000e5070000be
:1035b40037110000e205000067f60000eef8000095
:1035c400740b00009a170000b6110000ecff000015
:1035d40001f10000d2ee00004af500006efb00008d
:1035e400fff9000037f6000076f900006c080000cf
:1035f40045140000eb08000002f50000aaf30000e7
:1036040002070000d91600003a130000f801000078
:10361400baf20000dcf00000c8f70000edfc000086
:10362400f1f90000e2f3000013f50000520300007a
:10363400e1120000550c00006af700001ff20000c0
:10364400180500005819000054180000b0040000c8
:1036540047f0000036eb0000f0f30000bdfd000071
:103664003bfe00006ff600008bf300005afe0000e2
:10367400171200006d140000b0fd000037ec0000cc
:1036840004f7000036110000ac1b00007d0f0000a1
:1036940005fa0000dced0000a2f200000afd0000c3
:1036a400b3ff000072f600000dee0000fcf3000012
:1036b4002f090000601a0000750d0000e5f10000fc
:1036c400c6eb0000d1030000491c0000ba19000039
:1036d4003403000013ef00003fee000020fb000065
:1036e4002d03000042fc000031ee00006eec0000ef
:1036f4006cfd000099160000e01a00009cfe00001a
:1037040031e5000013ee0000bd100000e2240000cb
:103714009b160000d5f9000006ea000096f10000af
:10372400290100005e030000dbf4000075e70000df
:10373400b6ee0000be070000881e0000ce16000092
:1037440016f300004ddf000070f40000e01a0000e2
:1037540031260000b50d000023f00000d2ea00007d
:10376400cffc0000ed0a0000ac0100009cea000060
:1037740069e00000dcf10000bf0f000069200000d8
:103784002f100000afea0000cfdc0000fdf90000bc
:1037940019230000402b00007d0c0000afea00005c
:1037a400f3e8000021020000201100009100000055
:1037b400bae20000edd9000022f400004018000035
:1037c40038250000220e0000e2e5000034d9000094
:1037d4003bf900000a2500008c2d00008a0d000032
:1037e4008aeb000082eb0000da050000f81200000a
:1037f400e7fe000075df00004fd800008cf40000e5
:103804007d180000ae220000420d00004ce90000cb
:1038140097db00001ff7000094200000f22c00004a
:103824003112000044f0000072eb00003a03000083
:103834005b130000e902000015e30000c8d8000093
:10384400b9f1000099150000611f0000e00a0000b2
:1038540086ef00008ce2000050ee00007f0a0000ba
:1038640093200000261f00008d0c000032fe000093
:1038740097000000bc070000afff0000f0e8000064
:103884001cda0000b2e5000039030000e61700006e
:103894001a140000f803000004f5000015ef0000fe
:1038a40087f90000760d00008b1800004d11000010
:1038b400bc0100006dfc0000110600004c0c00006f
:1038c400acff000061e900000fe000008ced000097
:1038d40045050000c71100005b0c000090ff0000cc
:1038e40042f300005cef000073fc0000a91000002c
:1038f400f9190000c01300008c080000d604000071
:10390400f40500001b00000070f000003de2000020
:1039140057e4000095f60000260a00002d10000070
:10392400550900000501000046f80000acf2000053
:1039340099f900007b0b00005119000010160000db
:103944003008000031000000b70200000903000045
:10395400cbf7000005e90000e9e4000043f10000b2
:1039640051040000d60d0000fd090000b3fd000065
:1039740030f10000d0f2000021060000961800008b
:10398400d7170000c8070000b6fb0000cc000000f9
:10399400de0b000089080000def4000081e4000072
:1039a400a5e9000032fd0000140a0000f60500003d
:1039b4002efb000080f80000b7fa00008afa00002d
:1039c400f8fc000077080000d2130000dd110000ad
:1039d400d9060000750100002f070000070b000046
:1039e4004b0100004af0000098e800007cf1000060
:1039f400e2fe000049020000cafc000017fb0000c0
:103a04007b0100000e03000058f800009cf1000048
:103a1400c5000000ed170000e31a0000240a0000ae
:103a24005cfb0000c3fc000052080000440b0000d3
:103a3400d8fd0000d5ec000022ea000063f7000086
:103a440019060000f50600008bfc000048f5000094
:103a5400fef50000faf900007aff00007509000085
:103a6400de1200008211000097060000f3ff000040
:103a740041020000d902000036fb000055f20000ac
:103a8400c9f200000afe0000ed080000d60700009d
:103a9400dbfd000056f3000057f0000071fa00004f
:103aa400c40900004f0e00000e0600007aff00005b
:103ab4009a030000970b0000d609000011fb0000d8
:103ac400e8ec00000bee0000f4fb00002d09000000
:103ad400c80b0000fa0500006aff000026f8000089
:103ae40065f20000dcf70000b90600004612000091
:103af400f91100005d090000b9030000de020000b6
:103b0400befe000081f30000c2e70000a7e700004a
:103b140080f6000001090000f60f0000230a0000ef
:103b2400a101000075f80000e9f20000edf90000c1
:103b3400c60b00006a190000e4150000f707000036
:103b44002b000000c6020000f20200008ff7000004
:103b5400d8e80000fde400008ef1000091040000ac
:103b6400de0d0000da09000078fd000012f100000b
:103b740000f3000080060000be180000ab17000030
:103b840082070000a2fb0000ff000000f40b00000d
:103b94005808000086f400005fe40000e7e9000034
:103ba4007dfd0000250a0000d10500000cfb00008b
:103bb40089f80000bafa000085fa000017fd000039
:103bc400b0080000e8130000b8110000ae060000c1
:103bd4007a0100004e070000000b000008010000fd
:103be4000cf00000a2e80000adf100002dff000081
:103bf400ea020000eafc0000dcf90000b9ff000062
:103c04004f0200007df90000d8f300002d020000ef
:103c1400f016000018180000a50800005dfd000063
:103c24004b000000730900003e09000069fc00001d
:103c340083ef000051ef00002ef90000bf000000e8
:103c44000cfe00001ef70000dff700008afe0000f3
:103c540023ff0000cff900009bfd00007e0c000054
:103c6400851400008e0b000051ff0000a1fe00002f
:103c7400650500002b0900005c05000036fd00000e
:103c84001df9000022fb000029fc0000d2f700000f
:103c9400b1f10000caf1000066fb0000dd04000081
:103ca400c8000000ddf60000b8fc0000af0e000004
:103cb4000a1400007805000041f3000054f40000e9
:103cc400320a0000a6190000e310000047fd0000be
:103cd4005ff60000bfff0000880600001ffb000025
:103ce400a3e7000009e300008cf50000980b000036
:103cf4006c0d00000bfe000086f2000024f80000aa
:103d0400520900006d100000ce00000089f200008e
:103d140028fa0000010e0000441900008910000078
:103d24006601000079fe00004d0500008d050000cd
:103d34000ef90000a9e9000072e60000c6f30000d5
:103d44007103000056070000b000000032f90000c3
:103d540095fa000090010000130800008c05000093
:103d640090fa000029f7000027000000680f000007
:103d74004c150000100e00004e04000094000000da
:103d8400e1040000f0070000670000000af10000f1
:103d9400c7e8000091ef0000d1fc0000f002000031
:103da400a5fe000037f900004bfa000055ff0000a3
:103db400fe0100005c03000061020000ccff000073
:103dc400090000005c0300000d08000086090000e3
:103dd400e0080000bb0500006a02000007040000c0
:103de400de060000740400005afe0000bcf9000066
:103df40025f800008af70000dbf5000059f4000004
:103e04001cfa0000420500001e06000005f900002f
:103e140044f0000025fd0000e30c00005a0a0000f5
:103e2400c7f80000d5f400007008000091110000ec
:103e340038060000f6fc0000d90000005708000016
:103e44000c0a0000c905000021030000030400005f
:103e54004102000030fd000041f90000d2f50000ed
:103e640028f4000095f8000073fb000087fa0000b6
:103e740019fa00003ffb00000fff00005f03000081
:103e8400d006000036020000c1f700004dfa000021
:103e94007f0800000f0c0000ab020000ee000000e1
:103ea400510a0000c90d0000b3080000c101000060
:103eb400eefe00004e00000054ff0000fcfb00007a
:103ec40055fc00005f0000004aff000035fa0000c6
:103ed400f7f60000f8f7000060fc0000e5fc0000c5
:103ee400c9fd00003400000038f9000030f700007c
:103ef400ca00000098030000ea050000b5090000ac
:103f0400910000005dfb00004e060000cd0d000096
:103f14004e060000f7fa000082f900007b02000060
:103f24007209000004040000b7fc0000f4ff000064
:103f3400790500002d010000e4f8000004f90000f8
:103f44000fff000067ff000097fa00009df90000d2
:103f540021fc0000aefd0000a9ff0000c801000024
:103f640041ff0000fafb000000fd0000f8ff000024
:103f7400f40300007b040000c3ff000013020000f0
:103f84002a0800000f0800003e070000800100001e
:103f940077fb000057000000f00400005bfd000008
:103fa4000cf80000aafe00000d02000031fe000023
:103fb400dbf90000d0f90000c0fd0000b9fe0000ec
:103fc400bcfe000084fe000005f900004bfa00006e
:103fd400ac020000d2020000700400004d08000092
:103fe400ed000000b9fc000075050000ac0b0000fa
:103ff400f6040000e0f9000004f80000f0010000fd
:1040040036090000f5010000e1f9000093ff00000b
:104014007d070000f50100003bf800002afc0000c9
:104024009d050000e00100004ff9000078f9000050
:10403400fafd000029ff00000100000095ff0000c8
:10404400eaf70000b5f80000930300003e03000007
:1040540094fd000039fd0000dbfd0000200300009a
:10406400950300002f0100001007000093000000da
:10407400daf50000b2020000fd0e000020fd000091
:1040840022ef000023fd0000ee090000ab07000052
:104094004900000026fd0000600000005e030000ef
:1040a40031ff0000defb000065000000ff0000009f
:1040b4005bfe000097fe00001bff00000a010000e9
:1040c400470000006cfb0000c0fb0000d9000000aa
:1040d400eb010000cffe0000d2fd0000e102000071
:1040e40093030000affd00006cfa000050ff0000d5
:1040f4008306000074020000eefd0000ccff000007
:104104008e0000004101000033ff0000c8fb0000e6
:1041140069010000ab0600009efe00003dfc0000ab
:1041240048060000190a000026fe00004af40000b8
:10413400e1fd0000230b0000a6030000b0f5000021
:104144001ffd0000100700006e03000058ff000070
:1041540020ff000017fe0000170000002c050000df
:104164003504000088ff000016fd000063fe000017
:10417400ac0100003c0000001efe00005dff0000da
:104184006d000000c10100001b010000ac00000034
:104194006d0200002601000089fe0000fdfe000003
:1041a40019ff0000bcff0000fc0200002600000014
:1041b40088fc000048010000ae0400006700000015
:1041c400fafd0000d3000000980100001700000071
:1041d400fcfb0000a0fe0000be070000410300003d
:1041e40077f7000041fb000063070000ff040000b4
:1041f40002fc000067ff00002b03000050000000d9
:10420400fafd00000afe000073010000f700000040
:1042140016fe0000aefe00005ffd0000f2fc000090
:10422400550300000005000085fe00004afd000063
:10423400b70100000802000067ff00003c00000016
:104244005700000046fd000090fd000053010000ef
:10425400b402000037fe0000dffc0000a0010000f3
:104264004e0200008afe00007ffd00001c020000d8
:1042740090030000d5fc00003efb0000ce010000ce
:104284005005000097000000e6fa00003efd000023
:1042940027010000610300009203000073ff000087
:1042a40026fb000065fd0000dd0300007f04000024
:1042b4002dfe000010fc000009000000bdff0000fe
:1042c40088ff00009fff0000f6ff000019010000b6
:1042d40002000000a9fd00002cfe00002a020000dc
:1042e4009a0100006efe00002bfe000052ff000049
:1042f400abff00007fff000082ff000044000000cd
:104304004101000002010000a6fc000094fd000031
:10431400e30300000902000091fb0000fef9000025
:1043240045fd0000fd010000db0200000900000063
:1043340058ff000036000000a40100005f010000e7
:10434400d8ff0000bffc00002dfc00004cfd000065
:1043540069fd000015020000ab000000d9fc00005c
:1043640077010000c304000054020000a8fe00000e
:104374004cfc0000e2fc00009d0000001a0000005c
:1043840053fe0000aa000000f300000095010000a5
:10439400ae0100004bfc00004bfc000000030000d9
:1043a400ae010000e5fe0000e5fe000030fc000068
:1043b400e9fe0000c50300003b010000dbfb000038
:1043c40098fc00005202000042040000a9ff000013
:1043d400c7fd00001c0200001402000075fd00006f
:1043e40024ff000069030000d700000075fc0000f2
:1043f40057fd000078ff0000ea00000034020000ce
:10440400dc000000020000004e000000d1000000ab
:1044140036010000c4fe000062fd000024fe00001e
:10442400be00000017030000380200001d00000059
:104434001dfd0000b3fe00005202000077010000e1
:1044440081fe0000b3fe000054020000b902000027
:104454004bff0000c8fd00004d0100006e0300008a
:104464002dff00007ffc0000f5fe00006401000049
:104474007300000066ff0000a30100007d0200003d
:1044840006ff00003bfd000048020000b8030000e6
:10449400c7fd00000cfc00006ffe0000aefe000033
:1044a4001afe000005ff00003b000000430200006c
:1044b4003d030000520200005e020000d70100002c
:1044c4001f00000092fe0000a8fe000064fe000031
:1044d4002afd0000f9fe0000ef00000078ff000054
:1044e400fbfe000048010000f3010000540000003e
:1044f4009c00000072000000bafd000099ff00005b
:104504009f020000b3000000fcfd000058ff000003
:104514006601000097fe000011fd0000ddff0000b1
:104524005302000036000000fcfc000045000000bf
:104534009a0400006f020000ecfd000030fd000052
:10454400790100008a02000041fd000071fd0000b5
:10455400b4020000110200002dfe000073fe0000f2
:10456400f90100006c0200001aff0000e7ff0000e0
:104574001c02000054ff000099fd000038010000f7
:104584005c02000009fe0000ccfc00007301000086
:10459400c40300009eff00006dfd0000e701000061
:1045a400dd030000dcfc00009cf90000d3000000e7
:1045b4005c0400002fff0000b1fd00003403000084
:1045c400d2040000a1ff000095fc0000edff0000f4
:1045d4000a02000033fe000000fc00003c00000062
:1045e400a5020000e7ff0000befe000039ff000046
:1045f4003aff000000010000890100005bff000099
:104604001aff000072000000e5000000c8ff00006f
:1046140086fe000023ff00005d000000f6ff00009e
:10462400a0fe0000c9ff0000f50000000e0100001c
:10463400ed00000012ff0000e5fe00004f00000046
:10464400410000007e0000007500000033fe000001
:1046540091fe00005d0000004cff0000abfe000076
:1046640066000000210100007cff000054000000ef
:1046740004020000b200000097fe00000cfe0000df
:10468400ccff000097ff000026fe000045ff00005d
:10469400ba00000076ff0000effd0000f801000002
:1046a40077040000f4ff0000ddfd0000b800000006
:1046b4004b02000098ff0000d9fc000093fe0000ac
:1046c400540000009dff00001bfe00001aff0000c4
:1046d4006c0200006d0200002b00000051ff00007e
:1046e40082000000a600000010fe000034fe00005e
:1046f4008c00000042ff0000e1fd0000faff000012
:104704007d01000083000000a8fe000005ff0000fa
:10471400340100001a0100007aff000037ff000096
:1047240075000000f200000004ff0000b7fd000067
:104734006eff00009f00000040000000c4ff000066
:10474400e5fe000047000000280200000a00000007
:10475400ecfd0000a6ff00008901000061000000dc
:1047640037ff000096ff00002d000000430000000a
:10477400daff00000e000000fbff00007cff0000d9
:104784002800000033010000f4000000a8ff00002e
:104794003fff00005f0000008700000080ff000072
:1047a4007aff0000de0000001901000091ff000004
:1047b400defe0000a4ff0000840000001f000000d3
:1047c40017ff0000d7ff0000f4010000b301000050
:1047d40054ff00001d000000670200006f0100008c
:1047e4004fff0000fafe0000180100003202000032
:1047f4008dff00000cfe0000af000000ea01000085
:104804006dff000021fe0000780000005702000048
:104814007a000000a3fe0000720000009c02000069
:104824000b0100001dff00009b0000004702000078
:1048340089000000c4fe000059000000b901000016
:10484400ac00000004ff000001000000350200007d
:104854000b010000e5fe000054000000b20100005e
:1048640022000000f5fe000098ff00001601000081
:104874000f0000007cfe000065000000eb0100005a
:104884000f000000c9fe00006400000001020000e7
:104894000301000097fe000046ff00009d01000098
:1048a400d2000000f5fe000052ff00000e010000df
:1048b40056010000f2fe00004afe0000e300000082
:1048c400080100008cfe000087fe00004e0000007e
:1048d4007b0000003cff0000dafe00007e000000c8
:1048e4003201000052ff000006ff0000c700000074
:1048f400f9000000a5ff00001eff00000f000000eb
:10490400b0000000120000002dff0000ceff0000e8
:10491400060100007d00000069ff0000f0ff0000b8
:10492400b3000000490000005fff000021ff000009
:10493400550000006200000035ff0000caff0000bf
:10494400ed0000004800000075ff000015000000a5
:1049540015010000ce00000043ff000075ff0000b9
:10496400fe0000009200000079ff0000acff000090
:10497400af000000e800000058ff0000ccfe00007b
:1049840099000000b6000000d0fe0000ecfe00001c
:1049940030000000f6ff000019ff000019ff0000be
:1049a4005f0000009e000000e7fe000026ff0000fc
:1049b400c60000005d00000052ff000058ff000028
:1049c400e3ff00001b000000bbff00004bff0000e2
:1049d400a5ff0000340000001b000000ceff000013
:1049e40096ff0000e2ff000078000000bcff00001a
:1049f400a5fe000092ff0000cb000000fdff0000b8
:104a0400fefe0000b6ff0000a80000005d000000ec
:104a140090ff0000a1ff0000960000007900000054
:104a2400c1ff0000d8ff00003f000000ac00000000
:104a340054000000baff000022000000cb00000078
:104a44000f0000007eff00006100000082000000f3
:104a5400fbff0000d5ff0000eaff00003b00000060
:104a6400f3ff000081ff00003c000000af000000e5
:104a74002b0000000c000000530000007d0000002b
:104a840018000000b7ff00001500000054000000eb
:104a9400d0ff0000a0ff00004400000075000000eb
:104aa40016000000dbff00003d000000be00000017
:104ab4005d000000ceff0000ceff00005a000000a1
:104ac40091000000f0ff000075ff0000dfff000010
:104ad4005b000000070000009bff0000daff0000fd
:104ae4005a00000037000000d3ff0000f3ff00006d
:104af4001d0000002c0000000c000000d9ff000085
:104b04000500000045000000510000000300000003
:104b1400100000006a000000610000001f00000097
:104b2400deff00001b00000051000000efff00004a
:104b3400d1ff00003e0000005c000000fdff00000b
:104b4400d5ff0000380000006d00000020000000c8
:104b5400dbff00000900000007000000cfff000099
:104b6400e9ff0000feff000012000000ffff00004c
:104b7400deff0000080000001a000000ecff000047
:104b8400fbff00005400000047000000e6ff0000a7
:104b9400e1ff00004a00000059000000e6ff0000a9
:104ba400caff00004e00000080000000f9ff000072
:104bb400e1ff000043000000560000000200000076
:104bc400bfff00000f0000003e000000f9ff0000de
:104bd400caff0000f3ff00002c00000004000000e6
:104be400d5ff0000e8ff00001500000020000000d1
:104bf400e5ff0000d2ff00000500000011000000e6
:104c0400dfff0000c7ff0000efff00000c00000002
:104c1400e1ff0000c3ff0000eeff000004000000fd
:104c2400d8ff0000c9ff0000e5ff0000feff000000
:104c3400e5ff0000c5ff0000dcff0000eeff000000
:104c4400deff0000d0ff0000d8ff0000e8ff0000f6
:104c540002000000edff0000daff0000d8ff0000b2
:104c6400a4ff000095ff0000b4ff0000b3ff0000a4
:104c7400c1ff000093ff0000cfff000063ff0000ae
:104c840065ff000032000000b50100005e01000075
:104c940034fc000051fb000024040000e302000087
:104ca40002f9000019030000d0f6000010fa000019
:104cb40083120000e9fb0000b8fa00006d05000053
:104cc40000f50000d201000046170000470a00006a
:104cd40008dd0000d4f50000151f000086ef000079
:104ce40092f80000b00d00002cf60000f90300005b
:104cf4007804000040090000b1f80000b3e90000a6
:104d040094140000c207000081eb00006901000058
:104d140066130000a8fc0000e8f700004b07000041
:104d240016f400000dfa0000c30c00002afa00007b
:104d3400fdfd00005c0200004d0300005a0100006c
:104d440059f90000ca000000c4ff00002a00000056
:104d5400990100007e050000e6fe00001f16000019
:104d6400da0a0000fed10000e80900006d18000016
:104d74006fe100009ffe0000990e0000fafd0000a4
:104d8400890500008df3000038ef0000111e0000bb
:104d9400990800009df40000860c0000240a00001d
:104da400170d000064fa00003dee000012f200004e
:104db40036030000600b00002bf60000d703000050
:104dc400b90a00000f010000cffe000051fc0000f2
:104dd400bcfe00000bfa0000f5010000a007000073
:104de400c4f30000990500005a0c0000cdf7000040
:104df40081120000800000000ae00000de000000d4
:104e04004909000054f90000c3ff00004cff0000f2
:104e1400690a0000a20c00002df2000089fb0000ca
:104e2400600a0000420100006efb000072020000f4
:104e3400ba2000001e1b0000c2cc0000c5e2000026
:104e440023200000a4ef0000bbf40000ba0d000012
:104e5400a6010000bbf9000057f40000630700003e
:104e6400af0e0000e70700007cfb0000fd0500001a
:104e7400c213000027090000d3fe00003eeb00002f
:104e840036f00000b80400000500000044fa0000f9
:104e9400210100007f010000a4fc000005f20000d5
:104ea40084010000671d000074020000c8f10000c6
:104eb400bf010000aafd0000c7fb00000a010000ba
:104ec40027060000b10a0000f4f7000076f20000a3
:104ed4004bff000028f90000dffa000019fd000074
:104ee400fbfe0000ca04000024fa00007004000065
:104ef40089060000f201000008110000e0f500003e
:104f0400b5ff00000e1b0000f0fc000023f90000b8
:104f1400cdf700006dec00008dfc00005003000094
:104f2400dbf90000e5fd0000fa04000036f900009a
:104f340080010000850a0000fdfc0000fb08000061
:104f44000a07000066f5000061ff0000b1010000df
:104f54006efb00005d0a000033020000d8f200007e
:104f64008e000000f0f8000083f40000dd0400006f
:104f7400cc000000a2f7000060040000540400000c
:104f8400f2f70000b6030000b60900009ffd000020
:104f9400f1fd0000b70d00004c0e0000b40c000041
:104fa4004ef400001adf00009afc0000e7fd000048
:104fb40031f80000f20a00009b02000038eb000008
:104fc400a90000008b0f0000c4fd0000310e00009a
:104fd400cd1d0000e0fe0000af0300006a0d0000dc
:104fe40079e50000e9ee00005104000040f3000000
:104ff40052f900007309000047fc00002cf900007e
:1050040035f80000110d00003113000022fd0000ee
:1050140024080000c3fb000056fa000054050000f9
:105024007a010000120000006ffb0000d2fc0000b7
:105034005df70000cdf800002cff0000f5fe000035
:105044008bfb000042fc0000c9fb00007f0b00004a
:105054009e12000031fa00006dff0000df0a00001c
:10506400ad000000470400008e0f0000bff20000f6
:1050740024ef00004efd000057ed0000680400001e
:1050840084070000a8fa00009e1000005f050000dd
:1050940031f20000ae0300002e050000b0fb00005a
:1050a400a6fd0000a7010000820d0000120b000005
:1050b40018f70000d6f9000027fd0000d7f700001c
:1050c40075f900003502000074fe000075f400005c
:1050d400bd0d00006f01000010fc0000f90b000082
:1050e4009c03000088170000edfc00004e11000036
:1050f400d60400003ed300000206000091ec00003c
:10510400fbf500007b0c0000e1f60000f503000055
:1051140058f100002e0c0000a327000005fc00003d
:10512400c5f10000ba1600003107000086f4000043
:10513400610b000084df0000ffec00009b0c00000a
:105144000afc00003c040000d9020000a8ff000093
:105154008cf50000ed100000e20c0000bdee000034
:1051640017f400008afe000069060000da09000056
:1051740044080000180a00002ff5000001e10000b7
:10518400d9060000b8fe0000cdf60000e9fe0000dc
:10519400fdf9000071090000f8f30000fd1400009f
:1051a400991b00005eee0000080c0000930800004c
:1051b4000ff60000c70100008bf9000020f7000083
:1051c40022fd00006bfb000057f600000306000000
:1051d400540d0000b6fa0000a8f80000bffe00005d
:1051e40078fd000084080000f102000013f90000bb
:1051f40099090000c70800007cfd0000dbfe0000e8
:1052040065fb000035f000004bfc00003508000091
:10521400bcf5000012f900007203000004fa00005b
:105224007d130000c80700008f0700004319000029
:105234005ff700009d06000034ef00007af00000e4
:10524400880b000039e4000043f90000af100000af
:1052540067f7000025f300000e0800008d1d000014
:10526400fe060000aff90000f00b0000a0fb0000f8
:10527400470300008401000033ea000001fc000041
:1052840018fd000045fd00009a0c0000c9ff000055
:10529400c0fd000058f900006ffd0000ec0e000096
:1052a4001200000099fe00002ffb0000a0ff000088
:1052b4006411000028fd00003cf60000bcfd000065
:1052c4003ff800005ffb000046040000e1fb000023
:1052d400b4f90000fc0100003ef60000900e00004e
:1052e400dc17000074fe0000d1060000830b0000f0
:1052f40056f8000094f8000006fd0000cafb000008
:1053040077ff0000ebef0000a7ff00005208000049
:105314005dfe00006d07000061fd0000fbff000062
:105324006105000006fd0000c0050000e70900005b
:105334001f00000011fb00001eff0000f20200002d
:1053440040fb00003af300001efd0000b30400001f
:10535400bef900001306000047010000eaef000058
:105364005b110000c8090000a8fa0000b91300008e
:105374006b0e0000b6f1000080f20000b9030000db
:1053840062f600001df60000bb020000bffd000035
:1053940002ff000088f900005df30000ca1b000052
:1053a4004d1800006ffd0000d70300009f000000af
:1053b400ff00000092ed0000cd070000fbfe00009e
:1053c400cbdd0000b1120000c00b00007ef5000030
:1053d400880a000087f30000110100004710000054
:1053e400fdf700008a09000035fe000083f7000085
:1053f400cc0b0000b0ff000029000000f7ff000004
:1054040071f10000c8f40000c6080000fdff0000b0
:105414002cfa00004b070000aaf20000250c000043
:10542400221b00003cf900007ffe0000e0f40000b5
:105434002000000008140000bbfe0000bcf70000c0
:10544400d4ef000074f80000b00500003903000038
:10545400400600004f0100003afd000024fd00005a
:1054640037fe00005eff000046020000a9010000b4
:105474009e0100008f0c000044fd000023f5000095
:105484004403000014f70000f5f500004e05000089
:1054940048010000e2f90000f6060000f1fd0000fa
:1054a4000bf900005b14000053fc000031ff000006
:1054b40011160000d3010000ef01000070ee00009f
:1054c40089f50000bfff00005bf600009b050000ab
:1054d4005b00000000fc0000cb000000bcef0000fb
:1054e40099fd00001e1b0000810700005d0e0000f6
:1054f4005b0400006cf500003cfa000010f50000ad
:10550400da090000a6f6000098ee00005a08000030
:105514005f040000160200005e010000f0f00000cd
:1055240021020000100f000050ff0000b2fe000036
:1055340054f90000defb0000ba0600005608000023
:105544009cf90000bdfc0000bd020000c7f1000092
:10555400acfe0000270200004df8000023fd00000f
:10556400e0010000ce000000bbff00007a10000044
:105574009707000096fb000074030000d4fc0000b1
:105584004d05000022ff00008df400009902000088
:105594006df90000f0f70000f0ff000085ff000047
:1055a40090ff00006402000019fc000033f80000c2
:1055b4000b1100003c0800009bf80000c40f000021
:1055c400a404000047f5000014fe00005bfa00008c
:1055d40088ff0000cffd000050f80000b2fb00007f
:1055e400ea01000049010000fdfe000082fc000009
:1055f400d1f00000920b00005a110000e1fb000002
:10560400a508000093070000b4f9000071fd000034
:1056140077fe000061fb00000cff00007ffb000030
:105624001dfa00000fff0000370200007aff00009f
:105634009ffe0000b80100005efd0000450500006b
:10564400a30800000df9000080ff0000ec06000034
:10565400930000006c0400007dfb0000d9f70000fb
:10566400f3ff000090f80000e40000005f04000075
:10567400bc020000ae060000b6fc000086fd00007f
:10568400bdf8000020020000740b0000c3f7000006
:105694000e020000ad0e00006bfe000098fd00003d
:1056a400edfa000081f60000ef0400005f02000044
:1056b40016fc00008301000082fd0000b1fd000023
:1056c40084070000a3fa000023f80000ea0e00009b
:1056d40084fe0000f1fa0000020a000011fb000041
:1056e400adf9000088fe0000a7ff0000a6fd000041
:1056f400730300003b0b000022ff0000d5000000f4
:10570400a500000051fe00007e050000a3f6000085
:105714001afe0000d10500007df6000031fc0000f7
:10572400e8ff00001dff000020010000b40100009c
:1057340064f80000a40000005711000064fd00009c
:1057440051000000a50f0000bcfa000054f900004d
:105754006efd000017fb0000f500000071fa000068
:1057640026f9000008fe0000310300000aff0000d3
:1057740012000000edf5000060f700005415000071
:10578400680600003cfe0000670c0000ad0000004d
:105794009df9000069ff000063fc0000cefc0000de
:1057a40092fe0000aff90000b3fb00003d010000d1
:1057b40014010000ccfd00000a01000036fe0000c8
:1057c400c3fd00008d0a00008d0400002ff90000c5
:1057d4000c0600006f0600006f0100000a030000c1
:1057e400f8f5000023fb00004d0000007bfa0000e8
:1057f4002cfe0000fafe00008f0300006800000089
:10580400a2fe000085fd000088fb00005d0b000087
:10581400d4070000f0fc00002a0f00002e0a00004c
:10582400fdf7000062fb0000c9f900003bfb00002b
:1058340089ff0000ebfa0000defd0000760700009f
:10584400c6fc0000e3ff00000d01000059eb00005e
:105854000b0d0000c91700009bfb00002310000083
:10586400520800005ff5000073fd00006dfb0000ae
:10587400c0fa000065fd0000b0fe000071fd0000ec
:10588400a101000058030000dcfc0000d601000068
:105894006afb00001af90000c7140000390900006f
:1058a400a8f60000c5ff0000e3fc0000d5010000dd
:1058b400d10300006bff00005900000003fa000050
:1058c400e8fe000081000000eef6000044ff000046
:1058d4001e030000c60000001afe00007cff00004a
:1058e4005d010000f9fa00007b0a0000d307000004
:1058f40032fc00002d020000ff010000c50700007b
:10590400cafc0000cefc000081fd000050f5000040
:10591400b0030000d5fc0000cdf80000d504000061
:1059240080020000fafb0000b50000007cfe0000cd
:105934007bf00000f1080000301000006e0200004f
:10594400760c00006f00000014fb0000f3fb000065
:10595400e2fa000008fc00001ffd0000b90300008b
:10596400e1fd000087fc0000ddff000002ff0000f5
:10597400acfb000058ff00006c04000083fa000038
:105984003d040000e70b000065f600004bfe00003c
:1059940070020000c5f80000dc030000b60000003f
:1059a4006e010000290300007cfa0000bafa00002e
:1059b40056fd0000cfff0000fefc000081ff000048
:1059c4004e01000001000000dc000000b8fe0000f1
:1059d40014fb0000bcff00006e080000b4030000cc
:1059e400f604000002ff000023fa0000ed010000ad
:1059f400d4000000e5000000780000005c03000013
:105a0400ccff00009bfb000069fd000031fa0000a0
:105a140093fc00009dff0000440300004afe0000c8
:105a2400fd000000b2fb0000daf80000da0d00000f
:105a34008006000055010000a60600007c0300005b
:105a44005bfe0000b40300001b0200007ff30000b3
:105a54000100000034ff0000c7f80000030200004a
:105a640096fc0000f1010000ed030000cdfa0000f7
:105a740030020000a9ff000047f90000860400007e
:105a84003f060000a5fd00001a08000011060000f2
:105a94002bf90000bdff000003fd000087fe00009d
:105aa4006c030000b8fc0000d400000031000000ca
:105ab4004dfc000030000000bdff000063fe00004c
:105ac400e5ff000093030000a3fc00002ffc00008e
:105ad400ce0500003800000049050000070700005b
:105ae400b5000000740200002e000000b6000000a3
:105af40075fb0000baff00005b050000e003000036
:105b040060fe0000eefb0000c00000003afa000056
:105b14004ffe0000a101000066ff00001d0400000c
:105b24000aff0000fa0000004b000000e6f7000046
:105b3400000400005d090000e9fc00008900000089
:105b4400f407000062000000c3030000e404000046
:105b54007ef6000042f80000b30100000cfe0000d5
:105b6400fcfd0000e9010000a9fd0000d0030000d5
:105b740094020000e9f8000021fe000095fe0000f8
:105b840030fe000069fe00008a01000043090000a5
:105b9400bc0200006c000000480600006100000028
:105ba400fafd0000f6ff0000c9fb0000e8fa00005f
:105bb400e8000000fe00000009fd0000ccff00002a
:105bc400ef00000057ff000086000000cdfe00003b
:105bd400b0fc00008dff0000d0fa0000f8fe0000c9
:105be400ae0a0000600300007fff000040020000d6
:105bf400dffd00007cfd00002c0000006bfc0000b9
:105c0400bcfe000066030000940000009bfe000040
:105c14006dfe00002cff000080fe0000effe00007f
:105c2400cfff0000ffff000085ff0000e502000039
:105c3400b6ff0000fefa0000b500000029fa0000db
:105c440074ff0000830b0000bbfe00004300000053
:105c54004e050000b5fb0000eeff0000a1ff0000b0
:105c640084fc00000d010000c0fe000021fe0000c5
:105c7400bd0100008802000002ff00009afe00003f
:105c8400540000006afd000024ff000087010000aa
:105c9400b80000003a010000c5fd000001ff00004b
:105ca40029fc0000f4f90000130c00008e0a000027
:105cb4004bfb0000b501000036fd000010f90000a8
:105cc400b3ff00000bfc0000c2ff0000b60500009b
:105cd40026010000a2ff000024030000f4ff0000de
:105ce40076ff0000e7020000e2fd0000aefb0000ca
:105cf4007800000075020000140000002efe000071
:105d04009cfe0000de00000095ff000007fd00007f
:105d140080ff000025020000d20300000d010000f6
:105d2400f0ff0000f0ff0000c1ff0000750000005c
:105d340099fe000072010000c401000094000000fc
:105d4400ed0000006aff0000c60000006c010000c6
:105d54008afe00006ffd000095ff00007000000047
:105d640068ff0000da000000d701000032ff0000e5
:105d74008dff000001000000d8fe000020ff00009d
:105d840090fd00003eff00008302000014020000aa
:105d9400f9ff0000c1fe00008b010000a500000017
:105da400bfff0000e20100000102000050040000f7
:105db4009e00000060fb000043fd00000dff00009a
:105dc40022fe000072fe0000080100002d00000009
:105dd4009bff000026000000fafd0000cffe00003b
:105de400670000008cfe000079fe0000e2ff000066
:105df40041010000dd0300002f01000074010000d8
:105e040073050000d5fd0000a1ff0000130200008f
:105e1400f9fa00008d0000001cff000023fc0000c4
:105e24007600000071ff000050ff0000e9ff000051
:105e340037ff00002cff000049000000c5fe0000f1
:105e44006efe000043000000d7ff0000b1ff000019
:105e54002f0100005f00000048ff0000b2ff0000b7
:105e6400b2ff0000b0000000a7ff000072010000b4
:105e74001a020000f5fe00007b0100003000000063
:105e840085fd00004e0100001c000000dffe000044
:105e9400d3ff0000f4ff000086020000d7fe0000dc
:105ea400cefd0000080200006800000092ff000020
:105eb4006bff0000a1000000370100006afe000033
:105ec400bd0000004300000056fe0000f901000080
:105ed4007c000000fefe0000b6000000d1000000bf
:105ee400f0ff00003bfe0000f4fd0000c2ff0000d4
:105ef4004e0200004c02000027010000cf00000009
:105f040043010000c3ff0000aafe0000c6fe00001b
:105f14002fff0000520100009200000070ff0000fb
:105f240050ff000073ff00000eff0000f2fe0000af
:105f34008c010000a200000050ff000036020000a7
:105f440070000000f1fd000057ff00000d0000008c
:105f540099000000fcff0000bdff0000a700000046
:105f6400ebff0000f6fe00007fff0000a1ff000031
:105f740003ff0000fbff0000280000002eff0000cc
:105f8400f3000000cb00000039000000f201000023
:105f94009f0000007bff000020010000c9010000f9
:105fa400acff000096ff0000e00000001d000000b0
:105fb400f0ff0000030100002101000093ff000036
:105fc40093ff0000c8000000ed000000d0ff0000b7
:105fd40066ff0000fcff00000a010000ce01000083
:105fe40059ff00004aff0000620100003c0000006d
:105ff40047000000baff0000d8fe0000c600000001
:1060040097000000adfe000050ff0000b7ff000045
:10601400aaff00000d01000082ff000067000000dd
:106024006702000019ff000069ff0000ec00000097
:106034008bff000097ff000026000000970000007f
:10604400acff00005bff000038000000c0fe000051
:10605400beff00002b0100008fff000085ff000041
:1060640063000000b6000000deff0000c0fe000078
:10607400cefe000043010000940100001000000067
:10608400b9000000c2000000430000009eff0000b1
:10609400e8fe000090fe0000bd000000f8000000d3
:1060a40099ff000097ff000030ff00001f00000070
:1060b4004dff00005fff00001b010000bbff00005c
:1060c4003900000076010000d7fe000055fe0000f4
:1060d400baff00002000000045000000aeff0000f1
:1060e4001c0000009200000087ff00000dff00006c
:1060f4009eff00006bff00004eff000055000000f3
:1061040096ff0000afff0000480100002d000000d2
:10611400f1000000c4010000ccff0000f1ff00000a
:10612400c7010000100100002cff0000490000001e
:10613400ba000000d6ff00004e000000520100002b
:106144008b00000044ff0000140000000801000060
:106154008f00000072ff00009dff00004c00000053
:10616400a20100001b010000a2fe00006e0000005e
:106174002b010000ffff000059000000bdfe0000dd
:1061840082ff00003901000083ff0000d4fe0000fc
:1061940095ff00003aff0000a4000000f500000095
:1061a40009ff0000a4010000be010000dcfe0000a5
:1061b400100000004600000045ff0000f9ff000049
:1061c40076000000e8ff00007cff0000c3ff000031
:1061d40029ff0000eafe000059000000440000000e
:1061e40087ff00007fff00006e000000bc0000007d
:1061f4001600000010ff0000fbff0000e701000094
:1062040022ff0000f6fe00000a010000c7ff0000a4
:10621400c9ff00004800000035fe0000b7ff000081
:10622400d20100002aff0000baff00005aff00005c
:10623400b5ff0000b801000033ff00007dfe000040
:10624400fbff0000200000007aff000015ff0000a3
:1062540065fe0000d1fe0000d0ff00004bff0000ef
:1062640072ff0000e6ff00001a0000009c0000001e
:10627400e6ff0000b6fe000068ff000053000000c7
:106284001b000000b5ff0000caff0000e0ff000093
:106294002b0000004b00000092ff000036ff0000be
:1062a400a4ff000099000000f1ff00005eff000061
:1062b400780000007b000000c4fe00009dff000089
:1062c400ac000000ddff000098ff000093ff000019
:1062d400ff000000f3ff000045ff0000ba000000cb
:1062e4005aff000050ff0000c9000000e6ff000054
:1062f400a2ff0000ae0000004c0000009dff000063
:1063040045000000f2ff00002200000039000000f8
:10631400c9ff0000be000000feff0000ffff0000f8
:10632400910000006bff0000e4ff00002501000065
:1063340092ff0000abfe00000701000039000000de
:1063440014ff0000fe000000f3ff0000e9fe00005f
:1063540090010000a00000006afe0000810000001f
:10636400820100002500000021ff0000a2000000bf
:106374009a000000250000009b000000d1ff0000ef
:10638400de0000006200000041000000a8000000e0
:1063940051ff00008f000000b9000000120000004f
:1063a400880000005f0000008f00000050ff000024
:1063b4004e0000006b0000009dfe00006b0000001a
:1063c400170100003b0000001a0000007d000000df
:1063d4000200000038ff00003100000068000000e7
:1063e400d8ff000065000000ba0000002e00000085
:1063f400b8ff0000e9ff000011000000ddff00000d
:1064040078000000530000004a000000650000000e
:106414009dff000068000000520000007cff0000a7
:106424002a000000760000007dff000071ff0000dc
:10643400c10000009f000000a4ff0000d6ff000080
:10644400abff00007dff00004a00000006000000d2
:106454005bff00001800000056000000ebff000086
:106464001b000000ebff00002eff0000a7ff000050
:106474005c000000e5ff00002600000099ff00001a
:1064840077ff0000520000002200000066ff0000b9
:1064940005ff0000f8ff0000570000001e00000088
:1064a4007800000091ff00001cff0000a80000001d
:1064b4006800000008ff0000bfff00001e0000008d
:1064c40042ff000020000000bcff0000c0fe0000ee
:1064d400c7ff000025000000cfff000090ff000070
:1064e400baff0000b6ff0000bfff0000c1ff0000bc
:1064f40087ff0000b1ff000050ff0000b4ff000060
:10650400480000005aff00008dff0000ffff00005c
:10651400d6ff000080ff0000cfff0000b9ff00009d
:1065240037ff00003f0000002300000065ff00006b
:10653400adff0000a4ff00009cff0000afff0000bf
:10654400b2ff0000ddff000013ff0000eeff0000bb
:1065540060000000d9fe0000b3ff0000f5ff00005a
:106564003bff0000dfff0000f6ff0000c1ff00005a
:10657400c4ff0000cbff00004a000000f7ff00004a
:1065840034ff00000500000039000000d2ff0000c5
:106594000d0000003b0000001e000000fcff000096
:1065a4004900000030000000f7ff00004300000035
:1065b4005e0000006b000000610000002c00000081
:1065c4005b0000004100000023000000790000008f
:1065d4005f000000f3ff0000600000007a0000008c
:1065e4000a0000003c0000005000000062000000af
:1065f4005d000000430000008e0000002300000046
:10660400f7ff0000960000002e000000eeff0000df
:10661400630000006d0000005c00000051000000f9
:1066240063000000530000007300000050000000ed
:10663400ffff00004e0000004e0000001f0000009d
:1066440063000000600000004900000043000000f7
:10665400470000003e000000120000002800000077
:106664003a00000052000000600000005e000000dc
:10667400430000001b000000200000004700000051
:1066840017000000020000002a00000020000000a3
:1066940031000000feff000012000000170000009f
:1066a400d6ff00001e00000022000000e0ff0000f2
:1066b4001a00000024000000090000000d00000082
:1066c400060000001b000000d8ff0000e4ff0000eb
:1066d40037000000edff0000f3ff0000170000008a
:1066e400e9ff0000f3ff00000a000000d5ff0000ee
:1066f400cdff00000c000000ecff0000d2ff000002
:10670400e8ff0000daff0000f5ff000001000000d0
:10671400bfff0000cdff0000e5ff0000ccff00003c
:10672400f7ff0000eeff00009fff0000d5ff000010
:10673400f7ff0000afff0000baff0000faff0000ff
:10674400ceff0000cfff000007000000caff0000da
:10675400c2ff0000f5ff0000dbff0000c0ff0000e7
:10676400e8ff0000d2ff0000c2ff0000f6ff0000b7
:10677400b6ff0000acff0000e5ff0000a9ff000029
:10678400c7ff0000f0ff0000aeff0000b1ff0000f3
:10679400d7ff0000bbff0000b2ff0000c9ff0000ec
:1067a400bfff0000c4ff0000d7ff0000bfff0000d0
:1067b400c5ff0000d7ff0000ccff0000d6ff00009b
:1067c400c9ff0000c4ff0000deff0000e2ff00007c
:1067d400d0ff0000deff0000dbff0000e9ff000047
:1067e40005000000fdff000000000000f6ff0000af
:1067f400f0ff0000deff0000f2ff0000fdff0000dc
:10680400e1ff0000d8ff0000ffff0000e7ff0000e9
:10681400f1ff000005000000ffff0000250000005c
:10682400d6ff00003e000000a0ff000075fe00003f
:1068340015ff0000f00400003000000060f90000c3
:106844003e070000f502000044f600004902000083
:106854001107000099fb000051fc000055050000e1
:1068640087fe000033fe00005300000018fe000005
:10687400410200004efe00000bfd00007fff0000ff
:1068840024020000ed0000000e1600001bf70000bb
:10689400dde0000030220000fa0200004fdf0000bb
:1068a4001f06000099100000fb040000b0e900007e
:1068b40028f20000b4320000def400004ad20000e6
:1068c400882500004a0a000095e80000bc0000008a
:1068d400f30300000e0b0000f90d00003cdb000088
:1068e40067010000b21e00003fe90000a4ef0000b1
:1068f4004c130000250e00001ae8000059020000a5
:106904007a0b00000ff6000018fc0000e9010000fb
:1069140057000000abff00009e150000bae800001d
:1069240067ef0000ea26000026f20000c0eb00003a
:106934002a0c00008502000051fd0000f0fc00005c
:1069440013fe0000230800009405000026f6000052
:10695400f4ff000025070000cff80000ddff000071
:1069640068020000a2120000e902000011de00002b
:10697400e71400005f0e000018df0000f9000000bb
:10698400a10e0000e6fd000071f800005df90000b2
:106994002308000014130000b3fc0000eef4000010
:1069a400610800003a060000f0f7000059fa000000
:1069b4006c0d0000b50700009bfb00002eee0000ec
:1069c400620c000064060000ebdd0000db10000038
:1069d400ba0800006ef900000aff000058ff00002a
:1069e4004c0b00008ef200009a030000af0100007f
:1069f40039fa0000850600008600000076060000d3
:106a04003bf30000e3ff0000160b000020f0000041
:106a1400b8fc000074040000dbfb000004fe00006e
:106a240078010000bafe00002f01000052000000af
:106a3400b6fb00004cfc00003efe00008e09000086
:106a4400600000001c04000018050000e7f00000ce
:106a540016030000350100000bf1000032fc0000b9
:106a640075070000d7fb000014f40000ad0c000013
:106a7400edf90000c8060000fd0a000023f500003f
:106a8400720b00001f000000a0020000e5060000d9
:106a9400cdfa000035f80000b60b000001f7000045
:106aa400f7e90000e60a0000040300009df5000079
:106ab4002cff000093060000e7fe00008f0000009a
:106ac40073fe0000ff0900001c070000a0fc00008a
:106ad4007d020000e600000082fd000075ff00005a
:106ae40092ff000059f40000170200002b0300007d
:106af4008cfb000095fc0000920800003aff0000a7
:106b04000cfe00002cff0000e7fa00003c0c000023
:106b1400e6f40000ea030000120b00008cef000012
:106b2400c10d00007101000048f10000670b000076
:106b340085fa0000c5fb0000ba0300003e02000015
:106b44008700000002fd0000caff0000dc01000015
:106b5400470000000dfa000012050000a308000021
:106b6400d5080000d40200005df80000e1fd00003b
:106b7400d70a0000e8f700006def0000c70c000022
:106b8400f6040000fbf4000005fc00000c0d0000fe
:106b9400ccfa0000ae0500007913000072f5000085
:106ba40084050000f90b00002800000081fb0000b0
:106bb400c5ff0000070a0000fbf7000021ef0000fa
:106bc400900900008b020000bbf10000e801000006
:106bd4003b050000c8ff00009e090000970200006a
:106be400eafc0000dc0a0000eafe0000cbf400002e
:106bf4009f050000330600004af7000010fe000065
:106c040034000000550800003cf400002bf40000a0
:106c14005710000080f40000f5fe0000bc060000e0
:106c2400d6f900000c0200005d03000038f60000f5
:106c34001604000010060000aff200002705000053
:106c4400b6040000d2f90000d1fb000045030000a7
:106c540027010000fbfc0000ce010000d4fa000074
:106c6400fe01000050ff000010fc000004050000bd
:106c740009ff0000de07000089030000ccf70000d4
:106c84001cf80000090f000081fa000058ef000012
:106c940034090000eb030000fdfb000075f4000064
:106ca4005c09000045ff0000330200006f0900008a
:106cb400c10a0000400d0000eae900005c03000086
:106cc40018130000d9f10000e5ed0000780400007d
:106cd40004130000b1f5000031e500006411000068
:106ce400ec160000ebed0000dcf20000af14000035
:106cf4007907000095ee00001f050000df0b00007f
:106d040003fa0000acfe000010fe000052f4000084
:106d1400c2060000e80300005df4000076020000f3
:106d240058070000510200002bfb0000080000007f
:106d3400dc0900006e0100003efa0000f4fe0000d1
:106d4400f8010000030200007dfb000025fc0000a8
:106d54005e03000018020000dffa0000fffa0000e2
:106d64005e0300002200000059010000f9fd00004c
:106d74002f0c00009bf800003ef7000041110000ba
:106d840072f6000008fc000049040000050200003f
:106d94001dfe000018f90000760600002e01000018
:106da400f4f600001702000008030000b0fd000024
:106db4007bfb00001b030000fd0b0000bd02000074
:106dc4000bee0000e6fb0000e31b0000a5f300004f
:106dd400e5e500006515000037080000c2ef00007b
:106de400d9f40000010e0000cd06000097f4000065
:106df4001a0b000022070000ae050000f0f80000a6
:106e040021fd0000d20a000076fc0000f9f6000023
:106e140093f50000030a000016060000caed000006
:106e24009efd00005b0d00007b0b0000f3fa0000e8
:106e340071f70000df1000008f030000e1f2000092
:106e4400590100003d0600002d000000f5f7000088
:106e540011f80000610b0000f5030000f7f00000da
:106e6400da03000072080000d2f9000099f700006c
:106e740015110000450c00003ce9000041ff000032
:106e840071100000a6f80000a6ef0000b60600008e
:106e940020080000a6fd000070f40000fa020000c3
:106ea400f31d00009ae30000bef5000082200000fc
:106eb4006def000047f20000300900007305000088
:106ec4005307000048f1000050fe0000960f000038
:106ed400c7f400004ff10000b00700002b100000c1
:106ee40090ed00009a0200003610000043f4000008
:106ef40062fc000084ff00009d0e000046090000b3
:106f0400cee400006b0400007d1c00002feb0000a9
:106f140077f00000571200002f030000e7f2000092
:106f24006ef90000cb0c000099020000e4f30000ad
:106f340052020000de09000001fe00008ef800008d
:106f44001f160000bf02000058e100006412000098
:106f5400df1200002ad800009b000000941e0000ed
:106f640057f00000f4f70000f20200004c1000009b
:106f7400ad0100009afe0000b910000092f000007c
:106f8400cb0400006c0f00003fe500002204000069
:106f9400b5170000a8e60000e80300006f0e00002b
:106fa4005ff700006af3000025010000360c0000c2
:106fb40025fc00002c13000097ec00006ffc00007f
:106fc40053200000eede0000e1f40000cc150000c8
:106fd4006dfc00008df60000250200009dff0000fe
:106fe4000a130000ab0100000ede0000091e0000c1
:106ff400740d000071d7000042060000f51d00006a
:10700400c5f400000de3000008130000ea0a0000c4
:10701400a0e7000077f50000951100005409000076
:10702400dce20000cf05000011100000fafa0000b5
:107034005bfe0000a4000000950c000025f8000091
:10704400a7fb00002e080000bffc00001bff00008f
:10705400eeff000052fc0000acfa0000b500000096
:10706400f5ff000072fb00003d040000d5fb0000aa
:107074005ffe00003204000068f700005d130000aa
:10708400f8f90000bde80000d11900004e0000002e
:10709400bae80000100600006b0c00003ff7000087
:1070a40090f40000fe08000066070000c2f3000030
:1070b40060fe0000be060000d4000000baf8000024
:1070c4009b04000063100000cae8000026fa0000d8
:1070d400d21a0000a3ef0000b8e60000be1a0000b8
:1070e400070400007ae7000038090000f9080000ee
:1070f400f9fb00006f050000561800008eef000039
:107104005df000001e1f0000a4f9000042e400002e
:1071140083100000b4090000a1ed000040fe00004f
:10712400fc0e00002b02000022ed000039090000d3
:107134008a050000dcf60000b4fc0000df07000054
:10714400761c0000b8e30000c2ec0000022b000033
:1071540033f300009fd80000ff1d0000051000005d
:1071640041e20000c005000025070000280a0000d5
:10717400b80a0000aef30000d0ff0000dc100000ed
:10718400c3f9000011ec0000670f0000b209000011
:1071940029f20000b1f800006a06000051fc00006a
:1071a400e7f70000eaff000013030000a806000050
:1071b40055fa000084fe000038100000ba070000f1
:1071c400d3ed0000c9010000661300002af100009d
:1071d4004bf40000f8100000680100001df20000ec
:1071e4001d010000fd060000d6fd00003df9000071
:1071f40042010000b803000086fe0000aefb000060
:1072040010060000260700008df5000062fc000057
:107214004e080000a1fc000010f60000010500006b
:10722400760400007cfa000062ff000039030000cd
:1072340073000000b4020000e2010000a2fe00009e
:107244006c0a00007eff000089f0000007040000c3
:107254009a0a0000c0f70000f3f20000eb090000f6
:10726400e006000081ee0000f9ff0000610b000061
:1072740068f60000b5f90000511500007808000018
:10728400c1e9000004000000cf11000076fb0000fb
:10729400a0ee0000b8030000b00f000032f50000bb
:1072a4007cf30000d40c00006e05000052f20000d4
:1072b400d5010000050d00009c03000096000000ad
:1072c40013f7000085fc0000ae070000f5ff000086
:1072d400d3f00000aefa00007a1800002ff5000089
:1072e40036eb0000d51400001f02000052e4000039
:1072f400cc1500008d2e0000a6d8000010e9000077
:10730400942c0000b802000095dc000070f7000027
:10731400701e0000d5fc00003ddf00000f0a0000d5
:10732400fc1d0000e3f2000015ee0000041800004c
:107334004c000000aaef0000b30d00000407000099
:10734400a9f20000e6ff0000c705000062ed00009e
:10735400defe0000760c000041f60000b0f80000ec
:10736400e6080000b90e000086fc000044fc0000a2
:10737400590800007f0100006af8000086fd000043
:10738400d5030000a3ff00007afe00008df8000082
:10739400ec010000a906000038f4000077f90000b1
:1073a4005c0b0000a5010000dcfa0000f8000000fe
:1073b400fdfc000048060000aa01000003f20000e2
:1073c4000f0500004e0b0000b9f50000fef80000a8
:1073d4003f0800002e01000059f90000e8fc0000fd
:1073e4006c030000e302000079f80000dafe0000fc
:1073f4003009000015040000effd00002efa000023
:10740400cdff0000c6030000d5ff000074f80000a3
:107414003e000000fb0a000056f80000d7f7000009
:10742400090700001f02000049f800005a0000008c
:10743400241100001606000021f6000039fe0000a9
:107444004a070000b9fc0000e6fa0000bcfd000099
:1074540042ff00001f0800000cf800002cf8000098
:10746400a50a00004bff0000aeec0000c20d0000b6
:10747400b1270000dbed0000f4e50000ab130000d1
:10748400500e000090ed000044f00000540d000088
:10749400d7090000eeef000013f400008718000085
:1074a4008a060000beeb000073030000400b0000de
:1074b4006dfa0000b6fc0000730f000095ff000099
:1074c400b7f000001b050000e204000054ed0000ca
:1074d400f6fa0000c40f0000bdf90000e5f3000057
:1074e4007e090000ea0a00001c080000b70800003a
:1074f4002afd0000caf60000eeff0000320300007f
:107504005bfc00002af80000c4ff0000e70b000049
:1075140061fc000098ec000023000000490c00000e
:107524004bfb0000fefa00002e0d0000d203000009
:10753400cff5000021ff00009b060000adff000016
:1075440062f800008d00000039090000f901000014
:10755400f9f8000071fc0000b3050000fd00000014
:10756400fcf70000e9ff0000ba0d00003806000037
:10757400a5ef000084f900006d0e000097010000e3
:10758400dff20000e4fb00007c0c0000b605000004
:107594004ff3000040fc0000040900005900000003
:1075a40032fb000087030000cb0c00003d06000006
:1075b4002df6000002fc0000bc0500009d01000047
:1075c400bbfa00000ff60000190400001d0b0000b8
:1075d40055f7000088f50000900b00003e090000fc
:1075e4003cfa0000ae010000f60d00001507000093
:1075f4004ef300004afa0000bc0a0000b201000089
:10760400e9f1000022f60000c10a00000b060000a8
:1076140018f2000053f90000da0e0000a908000077
:1076240000fc0000030200002f06000059010000c6
:10763400a6f800006efc0000a5050000f7fe00009f
:10764400e6ef000040fb00007e0c000096fe000008
:107654002bf50000320200009a0c000048060000de
:107664000efc0000ddfc0000af0400001901000066
:10767400f0f7000087fc0000ac0400003ffd0000b0
:10768400cdf20000df000000360a00007ffa00009f
:10769400aff50000c4070000770d0000e4f9000016
:1076a400c9f50000bd060000060c0000cafc00007d
:1076b400b2f40000db010000b7090000e2fc0000a6
:1076c40063f0000002fe0000ad0b00004eff00005e
:1076d400d2f4000081010000e90e00003f05000023
:1076e4002ef700000ffd00008207000015030000c4
:1076f4002cf90000ecf900009804000025050000b6
:1077040056f80000f8f80000cc070000c50500009a
:107714003efb0000480100003d0900004cff000052
:1077240066f5000064040000bb0e0000fafc0000d3
:1077340052ed000012fb0000d80e0000e40400002b
:1077440015f00000c3f70000a90e0000d4080000e3
:10775400a1f90000eafe000047070000150200003e
:107764009bf8000018fd0000690500008efe000073
:107774000bf500008b010000560800008bf9000097
:10778400b4f70000ae040000ac090000460200009b
:10779400e3fb0000a5ff0000c204000030fe00006f
:1077a400a3f800004e0000008306000039fb00002f
:1077b400c8f200001a030000610800005ef800002f
:1077c400e4f70000f40a0000e20a000088f6000072
:1077d400eaf80000db090000270a0000dbf90000da
:1077e40038f60000b1040000f8070000ccf80000ef
:1077f4005df00000730100000a0c000021fc000091
:1078040031f30000f8030000940f0000ed020000c3
:1078140041f70000b9fe0000100900000902000051
:1078240072f80000d6fc0000ea030000e801000042
:107834006cf9000063fa00004a050000240400000b
:107844007afb00008f00000034040000a5f900005a
:107854009efa0000b80d0000851000001ff600001d
:10786400a3ea0000b3010000661200000204000055
:107874004aec0000cef30000ca0f0000640a0000c6
:10788400f7f2000085fa0000060b00005e04000019
:1078940063f80000e9fb0000270500004a0400002b
:1078a400f70400008d06000092fa000017f40000af
:1078b400f2fe00004303000070fc0000f1f9000038
:1078c4008b000000da07000087ff000040f800008a
:1078d40056020000e812000001150000e8fc000058
:1078e400aae9000079f30000420500007c080000ca
:1078f4009e0000007ef7000092f90000960300004d
:10790400360900004604000046f80000e7f40000d1
:10791400a9fb000058030000fb0600009f0c0000b8
:10792400ce0a0000d6f9000005ee0000dcf50000e8
:1079340002060000fe07000012fc00009ff9000090
:107944000805000010070000defd0000fdfe000039
:10795400080b00002d0b000090fb000031f200002a
:1079640054fc0000f10900004406000094fb0000f0
:10797400fffa000079000000cafd0000e5f60000ef
:1079840053fb00001105000060060000dafe000051
:107994006afa0000ea0200003d110000081300002a
:1079a4005501000097ee0000e3ef00002200000004
:1079b400010a0000510400006df900002ef90000d6
:1079c400b40200002e05000054ff000016fd000064
:1079d400c3fe00007efb0000cff80000b4080000e6
:1079e40053170000980800007cef000003eb000030
:1079f400c7fc0000c8090000650300009ff90000ef
:107a040008fc0000e00300000f020000aafe0000d2
:107a1400570700005d0c000083020000d5f400004d
:107a240044f200009cfe0000cd0a0000d1090000d1
:107a340089fe0000b2f6000054fa0000dafe0000ed
:107a44003cfd00005afc000010000000da040000b5
:107a54001402000013fb0000960000002c0f00002d
:107a640094110000a601000066ef000061ee000022
:107a7400d6fd0000300a0000f908000099fe00005d
:107a84007ff500009cf7000034000000ee040000c5
:107a9400c40100001bfc0000e5f80000da0000004f
:107aa4002c130000c713000058fe00001aec00005d
:107ab400aced000040ff0000560a0000c3030000c4
:107ac400a7f900006bf900009401000053050000c1
:107ad400b2020000de020000f0040000070400000f
:107ae4005dfd0000f7f4000029f7000037040000f2
:107af400a20c00005b080000bffd0000a7f6000018
:107b04009cf4000040f6000015fd00006c06000027
:107b14005a0a000092030000bbf900000afd0000ad
:107b24006c0c0000e313000086090000faf5000065
:107b340093ea000092f0000011010000920c000092
:107b440002090000b6fd0000b4f7000018fa0000b6
:107b5400ad0000007e0300009100000017fc00004f
:107b640066fc00006d070000da110000db0d000068
:107b7400aefd0000f7ec00000eea0000e7f600009e
:107b8400c1050000490b0000a707000064010000c4
:107b940066fc000007f9000075fc000046070000c1
:107ba400e70e0000500c0000630200004bf80000d8
:107bb40093f300001ef5000092fb00006c0400002b
:107bc40023080000690300009afc0000fdf900008e
:107bd400e3fb000059fe0000b70000003e05000072
:107be400760a00009a0c000042090000b900000067
:107bf400e3f50000a4ee00007ef20000d5ff0000d3
:107c040080090000250900009a030000affd000070
:107c1400f0f80000fbf700007cfe0000cc07000039
:107c2400d00b00005d0800006501000014fd000099
:107c340097fb00000ffb000049fc000040ff000020
:107c440077000000ddfd00006efb0000cafc0000b0
:107c5400feff0000c2010000b60100008302000024
:107c640061060000330b0000cb0c0000de060000b0
:107c740035fa000019ef00002aed0000aef500000f
:107c840048020000380a0000c00a00000505000090
:107c94003dfc000089f60000ccf80000f400000070
:107ca400f5070000a90900006c060000a30100000c
:107cb400f1fd000000fc0000b0fb0000d1fb00005f
:107cc4002dfb000030fa000093fb0000ceff000003
:107cd4002d040000ce0500001d0300009efe0000e0
:107ce4009ffd0000c1020000900a0000a60e0000e3
:107cf400eb090000bdfc0000cbee000048e90000e9
:107d040050ef00005bfc000044090000670f000016
:107d1400570c0000c903000033fb000021f70000ea
:107d24000ef90000d3fe00008e04000034070000aa
:107d3400ce0600008b0400006401000064fd000016
:107d4400acf80000c7f4000042f400008ff8000013
:107d540047000000d3070000940b00009b080000bc
:107d64006601000079fe0000b0010000d5060000a5
:107d7400bc0800008f0300001ffa0000f4f10000ab
:107d840033ef0000bff3000075fd00009b07000007
:107d9400ad0c0000740a00001704000036fd00005a
:107da40086f900007afa00007ffd000099000000c7
:107db400980300003b060000f6060000740400006f
:107dc400a3ff000053fa00004ff500006bf200001f
:107dd400bcf40000b9fc000063060000e20b0000e4
:107de400420a0000db050000ba040000b9050000e7
:107df400eb050000e40300003cfe000045f6000033
:107e04005df0000060f0000083f60000daff00007f
:107e14005b080000c80c0000f00b000035060000f1
:107e2400a3fd000046f70000e1f600000efb000091
:107e34008f0000007c05000088080000a2080000f4
:107e4400050600008401000005fc000057f6000050
:107e540012f200003bf20000fbf70000da00000021
:107e6400db0800009a0b0000f6090000b8080000c7
:107e74002c080000720700003b0500001aff0000f8
:107e8400b2f600005af00000cdee000062f20000ed
:107e940034fa000040040000cf0c0000a00f0000e2
:107ea4004a0c0000f9040000bafb0000eff40000e3
:107eb400f7f30000e8f800006b010000250900005a
:107ec400d20c0000050c000066070000edff000066
:107ed400b5f7000050f100005cef0000fff2000075
:107ee400b0fa0000c6030000370a0000270b0000a8
:107ef4000e0a0000240a0000f90900005e080000d0
:107f040059040000c7fd0000eef5000028ef000052
:107f140017ed00001cf10000cbf900003004000054
:107f2400ae0c0000f0100000760f00008107000086
:107f3400abfc00008af5000081f4000072f8000038
:107f4400140000002a080000ce0c0000290c0000d8
:107f54003b060000bcfd00000ef6000023f100000b
:107f640099f00000faf40000e0fc0000e6040000d0
:107f740046090000a2090000140900004909000094
:107f8400a509000030090000ee05000056ff0000be
:107f94000af7000073ef0000d1eb000017ee0000b9
:107fa40025f60000bc0100002c0c00006f1100003d
:107fb400b6100000470a00008e000000bdf8000063
:107fc400c9f5000077f80000a7ff0000e2060000f2
:107fd4005f0a0000f00800003f030000adfb000052
:107fe400cff400003df10000e0f20000e4f80000ee
:107ff400720000002106000073080000c1080000a0
:108004005d080000e4070000a7070000ba060000ae
:10801400e6030000ccfe000011f80000e4f10000cb
:10802400daee000043f0000005f60000e8fe000070
:10803400c90700002a0d0000040e0000650a0000b4
:10804400b10400009d0000004eff0000a5000000e8
:10805400dc020000fd020000e1ff0000a0fa0000c5
:1080640075f5000090f20000aaf30000edf800009e
:10807400860000005d070000d80a0000630a0000c3
:10808400df06000039020000cefe00001ffe0000e3
:10809400e4ff0000570200007f03000049020000d3
:1080a40003ff0000b4fa0000cff600001bf5000047
:1080b40091f60000e0fa000073000000540500008f
:1080c4001008000010080000b0060000530600006d
:1080d4002f07000095070000fe050000a70100001f
:1080e40026fb0000ecf30000c1ee000071ee00007e
:1080f40074f300007dfc0000500600007f0d0000ba
:10810400211000000f0d00002b050000c9fc000029
:1081140037f800006cf800007cfc0000a0020000ae
:10812400a4070000ef080000f1050000a0ff000014
:10813400caf80000f2f3000072f2000006f5000035
:10814400fffa0000270200008d0700004909000023
:10815400b00800005c080000b1080000f508000049
:10816400d3070000790300003ffc000014f4000072
:10817400b1ed00001bec000084f0000028fa0000c0
:10818400e1050000c10e0000db110000030f000038
:10819400e606000048fd00000ff7000016f6000098
:1081a400b7fa000085020000ab0800006c0a00006a
:1081b4004c0700009600000000f9000000f30000e6
:1081c40037f10000acf400009dfb0000db0200006e
:1081d4004f070000b2080000a90800002c080000a6
:1081e400cb07000078070000fe05000053020000e2
:1081f40074fc0000a4f5000058f00000d1ee00006b
:10820400e0f10000fcf80000540200003b0a00000a
:10821400010e00002e0d00005b080000ec020000bf
:10822400cfff00006bff00005a0100002103000093
:10823400430200007dfe00002df900008af40000d6
:10824400a5f20000cff40000b6fa00000c02000012
:10825400f20700009e0a0000d0090000cc060000ce
:108264005703000011010000bb000000670100007b
:108274008d01000030000000fcfc0000dff800006d
:108284004ef5000003f4000070f600002efc000020
:10829400f80200001c080000cd090000fd070000e2
:1082a400170500009d03000003040000660500009c
:1082b400e4050000e00300003fff0000d7f80000e1
:1082c4008ff200000cef0000e9ef0000a1f50000c0
:1082d400b2fe0000970700006d0d0000830e000041
:1082e4001b0b0000a3050000a500000001fe000018
:1082f40050fe00005a000000eb0100001e010000c7
:10830400b9fd000015f90000f0f4000037f3000097
:1083140070f500007efb000021030000000900004e
:10832400b50a0000e20800006d060000e604000043
:108334003e04000046040000170400005702000039
:1083440030fe00002ff800003ff2000009ef0000ab
:108354004ef000001cf60000dcfe00009407000054
:10836400c70d0000530f00001a0c0000170700008f
:10837400a1020000deff000015ff00001aff00004c
:10838400ddfe00008cfd00009efa0000def6000019
:1083940014f4000020f4000009f800009cfe000022
:1083a40052050000fe090000620b0000f109000004
:1083b4001e0700006f040000de02000051020000ee
:1083c400a8010000ddff00009afc00006ff8000027
:1083d40077f400002df2000025f30000d3f700002d
:1083e400edfe0000fb050000010b0000a30c0000e3
:1083f4004d0b0000bd0800001c0600003304000003
:10840400db0200005e0100001dff000083fb000092
:1084140023f7000038f300001ef1000093f200007f
:10842400e6f70000cbff00009f070000b80c000037
:10843400c50d00007a0b0000f2070000a204000042
:1084440090020000bc010000fb00000060ff00007f
:1084540059fc000058f8000056f40000c5f1000073
:1084640047f2000061f6000081fd00007b0500007a
:108474008c0b0000c40d0000580c00003b090000e8
:1084840009060000c3030000540200004a01000072
:108494008aff000020fc000099f70000fdf20000b4
:1084a40034f00000eff0000067f50000d2fc00009b
:1084b40030050000fd0b0000f00e0000a40d0000cc
:1084c400150a0000390600003d03000067010000a2
:1084d40025000000e2fe0000d4fc000081f9000049
:1084e4006ef50000e8f100003bf1000063f40000c9
:1084f400a0fa00007b0200007e090000760d000057
:108504005e0d0000a40a00007b0700009f04000029
:108514009c02000079010000620000003ffe0000a0
:10852400bffa000085f6000063f200005cf0000072
:10853400f0f1000030f700001fff00001b070000ef
:10854400b90c0000a70e0000240d0000130a00005f
:10855400e3060000630400008e020000d400000063
:10856400aefe000049fb00000ff70000e9f2000036
:1085740020f00000b6f00000fcf4000032fc000023
:10858400820400003f0b0000a00e0000220e000039
:10859400560b00002108000090050000e3030000d2
:1085a400770200009c00000072fd000008f9000042
:1085b40055f400006cf0000039ef0000b3f1000046
:1085c40083f7000095ff000095070000310d0000bf
:1085d400d70e00003e0d00004a0a000031070000db
:1085e400fa0400006b030000dd010000caff000074
:1085f40035fc00006cf70000c5f200009aef0000a3
:108604006fef0000d3f2000061f900008501000063
:10861400f6080000a20d00007c0e0000990c00007a
:10862400ab090000d5060000e90400008a0300003d
:108634000b020000d8ff000013fc00003bf7000011
:1086440063f2000017ef00001fef00009cf200002f
:1086540026f900004d010000c8080000a90d000023
:10866400ce0e00002d0d0000820a0000be0700009f
:108674009e050000ee030000f401000047ff000027
:108684005ffb0000adf6000060f2000086ef000022
:10869400a4ef00003cf3000091f900004d0100003c
:1086a4008c080000320d00003d0e0000be0c0000de
:1086b400490a0000fd0700002f060000b70400006f
:1086c400150300006b0000002cfc0000f5f6000010
:1086d40044f2000047ef0000f8ee000012f2000040
:1086e40046f8000036000000e5070000560d0000c3
:1086f400fb0e00005a0d0000b60a00003708000007
:108704005a06000023050000b703000072010000b0
:10871400b7fd000090f8000056f300007eef000063
:1087240044ee0000b0f0000062f6000042fe0000db
:1087340065060000510c0000d70e0000c10d0000ba
:108744000c0b000094080000ae0600008305000036
:1087540086040000dc020000aaff0000c7fa000043
:1087640015f5000050f0000012ee000042ef00008a
:10877400e5f3000026fb000060030000370a000058
:10878400ec0d0000c60d00006c0b00004109000058
:108794008d070000a106000034060000fa04000062
:1087a4003302000056fd00004af700009ff100006c
:1087b400f4ed0000aeed0000ebf000001bf700004c
:1087c4001eff00009a060000d40b0000090e0000f2
:1087d4000c0d0000b00a0000de0800008107000054
:1087e4004c0600004205000069030000d5ff0000ac
:1087f400d0fa000050f50000aaf0000052ee00008c
:108804000cef0000d3f2000020f900007300000018
:1088140017070000bd0b0000320d0000370c0000ec
:10882400a40a0000f8080000940700008b0600006a
:1088340036050000f1020000e4fe000084f90000a7
:1088440010f40000a3ef0000bded00001fef0000d6
:1088540075f3000045fa0000a301000008080000b9
:10886400300c0000f30c0000c40b00000a0a0000e6
:108874006c0800005c070000780600005105000049
:108884001803000015ff0000aff900001af40000ff
:10889400a1ef00008bed0000f5ee000074f3000082
:1088a40038fa0000a6010000f8070000240c0000bc
:1088b400e50c0000e20b0000710a0000da08000079
:1088c400fc070000fe060000a80500005c03000091
:1088d4001bff0000b5f9000007f4000094ef00004e
:1088e400d6ed000059ef0000c6f300001efa0000a8
:1088f400160100002d070000410b0000620c00006f
:10890400570b0000f3090000c7080000130800001b
:10891400780700006a0600004b0400005e000000b7
:108924001bfb000060f5000078f0000007ee00007b
:10893400e0ee000066f20000f2f70000acfe00007a
:1089440005050000dd090000d50b0000270b000021
:10895400e7090000d8080000a6070000d8060000b8
:108964003d060000f90400006a02000023fe000036
:10897400b7f8000052f300007bef00004aee00005d
:108984001af0000060f400005bfa00003d010000f2
:10899400f9060000ce0a0000ed0b0000710a000089
:1089a4001609000000080000ee060000a8060000fa
:1089b40033060000b4040000810100007dfc0000c7
:1089c400cff60000a6f10000a8ee0000d6ee0000ed
:1089d400b9f10000aaf60000fffc000050030000fb
:1089e4001b080000eb0a0000b80a0000140900008c
:1089f40064080000b00700003e0700005b070000a9
:108a0400b2060000a2040000cb0000007efb0000c0
:108a140000f60000a6f100007def0000f6ef000074
:108a2400c8f200006bf7000004fd0000960200008d
:108a34007b0700005e0a0000b40a0000e60900009b
:108a44000909000054080000d70700007907000056
:108a5400ad060000c20400003701000054fc000011
:108a6400f7f6000064f20000aaef0000a0ef000097
:108a740051f2000005f7000024fd00004d03000042
:108a840076080000420b0000450b0000520a00006b
:108a9400340900002c08000079070000e0060000fb
:108aa400e50500008103000077ff000043fa0000a1
:108ab400caf40000b3f0000033ef0000b5f000008a
:108ac400acf4000068fa0000ad00000022060000cb
:108ad400d6090000030b0000620a00002709000009
:108ae40042080000c40700001d070000290600001a
:108af400ff0300002e00000033fb0000c9f5000056
:108b040067f1000077ef000071f00000e8f3000067
:108b140064f90000b9ff0000810500008909000024
:108b2400c10a0000330a000065090000560800006d
:108b340043070000a0060000d20500001f04000047
:108b4400c6000000cefb000035f6000050f1000026
:108b540097ee0000bbee0000c6f10000def6000058
:108b640072fd00000c040000f1080000b80b0000c6
:108b74006d0b0000b7090000a60800007207000092
:108b8400b90600008e060000ae0500008203000056
:108b94006dff0000f3f9000059f40000f0ef00004d
:108ba4005aee0000d9ef0000b9f3000063f90000a9
:108bb400f4ff0000ac050000ad090000360b000016
:108bc400f0090000ad080000220800005f07000063
:108bd400490700003a070000f80500001e030000e2
:108be40076fe0000c5f800008ff300001ef00000c0
:108bf40051ef000042f1000046f50000aefa00001b
:108c04005c0000008805000065090000900a00006f
:108c1400dc090000f808000058080000f207000012
:108c2400bd070000660700002e0600005d0300007b
:108c3400fdfe0000c6f90000caf4000049f100007e
:108c44000df0000076f10000e2f40000c8f9000025
:108c54006fff0000ce040000f6080000900a000038
:108c64000e0a00003e09000077080000a207000079
:108c74004f070000350700005c06000028040000d0
:108c8400650000004efb0000f8f50000e9f100006b
:108c94001df00000dbf00000c2f300006af80000e1
:108ca400dffd00002e0300008e070000ba0900005b
:108cb400560900003f080000cb0700006a070000c7
:108cc4004c0700008c07000022070000620500002a
:108cd400f301000032fd0000f3f7000061f300002f
:108ce400b3f000009df00000f5f20000bdf60000b6
:108cf4008cfb00007a000000f90400003308000037
:108d0400140900005f0800004b070000f006000093
:108d140005070000fa060000fc0600005e060000dd
:108d240054040000d00000004dfc00008af700004d
:108d3400c1f30000f3f1000037f2000067f4000013
:108d4400fbf7000056fc0000df00000020050000d7
:108d5400c10700001b080000af0700000207000065
:108d6400800600009e060000ce060000d606000025
:108d74003406000032040000e7000000b9fc0000e3
:108d84005bf80000d6f400000ef300003ff300008f
:108d940017f5000014f80000f4fb0000e4ff0000e5
:108da400890300008e060000a407000034070000b9
:108db4007d0600001b0600000c06000027060000cc
:108dc400620600002a060000d90400004c020000dc
:108dd400bafe000082fa0000a5f600002df400009f
:108de4006ef3000063f40000b2f600000efa000017
:108df400effd00009f01000024050000160700009d
:108e040076060000b3050000940500004405000048
:108e1400a905000064060000990600002f06000062
:108e24006a0400003201000032fd0000f7f800007f
:108e34008cf50000ebf30000ebf3000063f5000099
:108e440038f80000c4fb000058ff00009002000046
:108e54000e050000c1050000f2040000a304000098
:108e640025050000910500005e0600004007000093
:108e74003f0700004b060000ef0300005a0000000b
:108e840052fc00007ef80000b0f5000088f40000f9
:108e9400f6f4000097f6000033f900005afc0000d5
:108ea4006cff0000170200002d04000023050000e1
:108eb400100500001105000081050000fa050000fe
:108ec40080060000f1060000d5060000dd05000064
:108ed400d5030000e400000069fd0000fdf9000076
:108ee4004af70000c1f5000079f5000070f60000b3
:108ef40068f8000013fb000011fe0000ff000000f2
:108f0400d2030000a7050000a70500001405000017
:108f1400150500003605000089050000460600001e
:108f2400ca0600008a06000045050000c6020000cb
:108f340046ff00006dfb0000eff700009bf500000a
:108f4400daf400007bf5000051f70000fef90000a0
:108f540003fd0000f8ff0000ac0200009e040000c6
:108f640012050000890400009c0400002b05000089
:108f74009f0500007406000000070000ca060000f8
:108f8400b20500004f030000f0ff000032fc0000b7
:108f9400bcf8000038f6000032f5000089f5000046
:108fa40001f700006af9000051fc000034ff0000e2
:108fb400c7010000f9030000f8040000e604000003
:108fc400e70400004d050000dc0500005806000021
:108fd400c4060000b3060000ad0500009d030000b8
:108fe400a200000029fd0000d4f900003ff70000b2
:108ff400d7f50000bff50000e0f60000f3f800002c
:10900400b2fb0000a3fe0000830100003404000052
:109014008d05000042050000e40400000605000080
:1090240037050000c205000088060000de060000c7
:109034004b06000093040000b10100000afe00008a
:109044004ffa000044f7000094f500005bf50000bf
:109054006ff6000080f800001cfb0000d9fd000042
:1090640080000000db02000066040000ac04000085
:1090740054040000ae04000034050000b9050000eb
:1090840078060000b50600005d060000210500001a
:10909400d1020000b3ff000055fc000044f90000b9
:1090a400f7f60000f3f5000007f600002cf70000c7
:1090b4002af90000aefb00004cfe0000df000000b7
:1090c40079030000b004000093040000530400007e
:1090d400bc0400005e050000aa0500005f06000055
:1090e400b70600001f0600009a04000004020000f6
:1090f400ddfe00009bfb0000b7f80000f1f6000065
:109104005ef60000b4f60000e6f70000c6f90000c1
:1091140008fc000057fe0000d300000044030000d8
:10912400c5040000eb0400008e040000cd04000020
:109134003c0500009c050000110600003a060000f2
:10914400c30500004c040000f001000004ff00000f
:10915400e4fb000028f900006cf70000c0f60000f2
:10916400fcf6000019f80000daf90000f4fb000036
:1091740049fe0000a300000027030000a304000030
:109184009e0400005c04000049040000bd040000cb
:10919400400500009c050000f5050000ae05000038
:1091a4007a0400005402000082ff000084fc0000e6
:1091b400dcf9000015f8000062f7000081f70000f8
:1091c40045f80000aaf9000099fb000096fd000094
:1091d400a1ff0000c8010000b503000075040000f1
:1091e400ed030000f30300002b0400007b040000e7
:1091f40042050000a5050000b80500003a0500007e
:10920400bb03000062010000a6fe0000e3fb0000b7
:10921400a6f900005bf80000f0f7000030f8000049
:1092240014f9000085fa000052fc000021fe000041
:109234001d0000006e020000d9030000e7030000d7
:109244008d030000b003000065040000e304000087
:10925400830500002c0600001006000050050000e5
:10926400900300000b01000058fe0000c2fb000048
:10927400d8f90000c8f8000072f80000b4f8000043
:109284006ff900009dfa000015fc0000befd00000f
:10929400beff0000c701000048030000ba0300003d
:1092a40098030000ce03000048040000d504000029
:1092b4009c0500004b06000071060000be0500007e
:1092c40025040000da01000027ff000082fc0000f2
:1092d4004bfa0000d0f800002df8000036f800002a
:1092e400d4f80000f8f900007dfb00004cfd0000fc
:1092f40061ff0000a5010000830300001b040000bf
:10930400c9030000b8030000f9030000650400006d
:109314000b050000cc05000043060000f205000028
:10932400d3040000d60200004a000000adfd000096
:1093340053fb000098f900009ff8000088f8000033
:1093440019f9000005fa000038fb0000b0fc000029
:1093540060fe00004c0000003902000066030000bb
:10936400850300001d0300000a03000057030000ea
:10937400c40300009f04000080050000d90500001c
:10938400a10500009a040000ae02000044000000a1
:10939400bafd000070fb0000c5f90000e1f8000010
:1093a400d2f8000046f9000027fa00005efb000036
:1093b400b8fc000057fe0000330000000d0200005e
:1093c4000e030000ea0200008b020000a502000068
:1093d400ff020000a3030000a1040000a205000096
:1093e40051060000340600002e0500004b03000067
:1093f400e30000005afe0000f9fb000027fa000019
:109404000ef90000c2f8000029f90000edf900008f
:10941400edfa00003afc0000b5fd000074ff000006
:1094240066010000ce0200003f030000d9020000e4
:1094340099020000aa020000dc020000b40300004c
:10944400be0400008c050000da050000550500008c
:10945400fa030000e001000063ff0000f3fc0000d9
:10946400eefa00009cf9000010f9000034f9000045
:10947400d0f90000c0fa0000e3fb00003cfd00004e
:10948400d7fe0000b00000004d020000e70200001b
:109494009b020000520200006402000099020000d6
:1094a400570300007504000078050000060600005c
:1094b400bd05000089040000840200001d000000b6
:1094c400a7fd00007bfb0000f4f900002bf900006d
:1094d4002af90000aff900007bfa000093fb0000ba
:1094e400edfc000072fe00005400000003020000c6
:1094f400f0020000d90200006a02000065020000c8
:1095040056020000ea0200000904000003050000fe
:10951400c7050000be050000e10400003e03000092
:10952400f400000081fe00003efc000093fa0000fd
:1095340097f900004ef90000abf9000053fa00005f
:1095440029fb000039fc000072fd0000fbfe000056
:10955400ce0000004a020000b30200002c0200000a
:10956400bd010000530100003a0100002202000086
:10957400530300009304000095050000e405000077
:1095840039050000a00300008c01000038ff000032
:109594000bfd00004afb000038fa0000c2f900008d
:1095a400d3f900005dfa000017fb0000fafb00008d
:1095b40008fd000062fe000015000000c501000067
:1095c4005202000008020000ca0100006d01000000
:1095d400300100005f0100005f020000ae030000e4
:1095e400b7040000840500007c0500009b04000013
:1095f400210300004e0100004cff00005bfd000051
:10960400c3fb00009ffa000018fa000000fa0000f3
:1096140068fa00002afb000029fc000065fd000038
:10962400d7fe0000b3000000fe0100002a02000083
:10963400dd0100003f010000a80000006b000000f5
:109644009b0000005c010000a9020000050400006a
:109654000705000064050000f7040000f2030000a1
:1096640060020000880000009dfe0000defc000097
:109674008ffb0000b3fa00005ffa00007bfa0000e1
:1096840009fb0000d7fb0000defc00000dfe00001b
:109694007fff0000d9000000760100006101000096
:1096a40013010000b60000003f0000002400000089
:1096b400720000002e010000580200007a0300002e
:1096c4004c040000d3040000d90400002904000065
:1096d4000303000087010000ccff000016fe000019
:1096e40092fc000054fb000093fa000066fa0000ac
:1096f400aafa00006afb00006dfc000086fd000071
:10970400e0fe00003e000000320100006a0100009b
:109714002b010000cb000000680000001d000000c9
:10972400ffff0000490000001f01000020020000ac
:109734003203000041040000f40400002b05000083
:10974400c1040000d30300005e020000a700000073
:10975400f6fe000061fd00001dfc000037fb000068
:10976400ddfa0000f3fa00005ffb000039fc0000a2
:109774004dfd000081fe0000ecff0000e50000004c
:109784002b01000021010000ea0000009700000006
:109794003e00000020000000260000004b000000f6
:1097a400e7000000a10100004c02000007030000d4
:1097b4008f030000e2030000d40300003d03000017
:1097c400480200000a010000a2ff000038fe000069
:1097d400f3fc0000f9fb000063fb00003dfb00000c
:1097e40072fb0000edfb0000c3fc0000d1fd000093
:1097f40005ff00002d000000be000000db0000009b
:10980400d2000000910000004700000006000000a4
:10981400daff00001d0000004d0000006d00000094
:10982400f00000007d010000df0100006e02000076
:10983400f10200002c0300004e030000f8020000b7
:10984400520200005a01000017000000ddfe000073
:10985400b3fd0000bdfc00001dfc0000dafb0000ad
:10986400f3fb000071fc000034fd000043fe000027
:1098740083ff00007b000000f4000000ff000000f4
:10988400f3000000b00000004100000025000000cb
:109894001a000000100000003b00000061000000fe
:1098a4007f000000b5000000ee0000004c01000045
:1098b400b40100001202000085020000da02000078
:1098c400ca02000075020000e8010000ff00000069
:1098d400f7ff0000ebfe0000f7fd000030fd000084
:1098e400b0fc000083fc0000a0fc000017fd000099
:1098f400d5fd0000cdfe0000c1ff00005d000000aa
:10990400aa000000a9000000770000005100000038
:109914001b000000070000001f0000003b000000c7
:10992400600000007a00000083000000a000000036
:10993400be000000ed0000003c01000095010000a5
:109944000a0200006f02000086020000720200009a
:109954002802000076010000a4000000b6ff000009
:10996400cbfe0000fffd000069fd000016fd0000b5
:109974000dfd000053fd0000defd0000a9fe000007
:109984007aff00000700000052000000620000009f
:10999400390000001900000001000000f7ff00007a
:1099a4001a0000004e0000007b0000009000000040
:1099b4009200000099000000a2000000a70000002f
:1099c400ce0000001901000082010000ed0100003a
:1099d40028020000610200006c0200000e02000078
:1099e4007f010000c5000000e9ff000019ff00002e
:1099f40062fe0000d4fd000085fd00007afd000039
:109a0400a6fd00000bfe0000a5fe000046ff0000be
:109a1400bfff0000f8ff0000150000000d0000006b
:109a2400f0ff0000f7ff0000140000003c000000fd
:109a34007a000000aa000000b5000000bd0000008c
:109a4400bd000000a8000000a30000009c0000006e
:109a540091000000a2000000ca000000f000000015
:109a64002f0100005a0100004d0100003c010000dc
:109a7400ef000000820000000a00000072ff0000f6
:109a8400f6fe00008bfe000033fe0000fdfd00002a
:109a9400fefd000037fe00008dfe0000e7fe000022
:109aa40054ff0000a7ff0000ccff0000e2ff00000d
:109ab400e1ff0000e2ff0000d7ff0000d6ff000036
:109ac400e0ff0000f2ff0000180000002b0000007f
:109ad40028000000270000003a00000049000000b0
:109ae400490000004800000051000000540000003c
:109af4004c00000050000000590000006900000004
:109b0400800000009a000000d1000000ed00000079
:109b1400ed000000cc0000009d0000007500000076
:109b240018000000d4ff0000a7ff00005fff000042
:109b340046ff000042ff000045ff00005eff0000fa
:109b44007fff000096ff0000acff0000cdff000087
:109b5400d6ff0000d2ff0000ebff00000b00000066
:109b64000d000000300000004c0000004300000025
:109b740060000000660000005f0000004400000078
:109b840036000000410000001c0000001800000026
:109b94001a00000016000000270000002200000048
:109ba4001500000013000000210000002500000043
:109bb4001e0000002a00000012000000e9ff00005f
:109bc400d9ff0000c9ff0000c4ff0000c1ff00006e
:109bd400b9ff0000bdff0000bfff0000bcff000094
:109be400c3ff0000c4ff0000c6ff0000c8ff000060
:109bf400c6ff0000c5ff0000c3ff0000baff00005d
:109c0400c8ff0000e1ff0000e6ff0000edff0000d8
:109c1400fcff0000f8ff0000ecff0000e3ff000081
:109c2400f4ff0000f0ff0000edff00000200000060
:109c340003000000fcff0000f4ff0000f6ff00003a
:109c4400f4ff0000feff00001000000014000000fc
:109c5400260000003100000028000000260000005b
:109c640026000000220000001b000000120000007b
:109c740023000000410000004f0000005a000000d3
:109c84005e0000004f0000003b00000033000000b5
:109c94003a000000480000004100000043000000ba
:109ca4005d00000066000000730000006500000015
:109cb40070000000870000005500000073000000e1
:109cc40048000000200000005d0000001f000000ac
:109cd4004600000061000000300000005e0000004b
:109ce4004400000033000000300000000d000000bc
:109cf40030000000260000002600000030000000b4
:109d04000c0000001c00000002000000f6ff000030
:109d1400150000000f0000002a0000001b000000d6
:109d24000d0000000c000000e0ff0000daff00005e
:109d3400cfff0000d6ff0000f4ff0000efff00009b
:109d4400f7ff0000f7ff0000d8ff0000e0ff00006d
:109d5400daff0000daff0000e7ff0000e9ff00007f
:109d6400f4ff0000f6ff0000f5ff0000f8ff00001c
:109d7400010000000a0000000a0000000e000000bc
:109d8400080000000a00000013000000100000009a
:109d940012000000140000001d0000001a00000062
:109da40017000000120000001c0000002700000043
:109db40024000000340000004000000042000000c5
:109dc40050000000480000004a0000005d00000050
:109dd400550000005c000000550000005b0000001e
:109de400550000004f000000570000003c00000038
:109df40031000000360000003f0000002600000093
:109e0400520000005400000050000000e8ff000071
:109e14001400000086000000f9ff00002400000088
:109e24001b00000028000000faff0000d6ff00001d
:109e3400200000009dff0000a3ff0000b2ff00000f
:109e440085ff000066ff000063ff00005fff000065
:109e540051ff000063ff00005cff0000cdff000025
:109e64001700000052000000fd000000c0000000c8
:109e74001b0000004900000058000000140000000e
:109e8400b9ff0000a8ff00006fff000081ff000081
:109e940065ff00002cff00005fff000030ff0000a2
:109ea40033ff000040ff000057ff00002eff0000ba
:109eb40048ff000037ff000042ff0000b9ff000028
:109ec4001b00000087000000d70000005e010000b6
:109ed4001e010000510000006d000000ad000000f4
:109ee4003e000000daff0000c7ff0000b2ff0000e0
:109ef4009bff000075ff000064ff00005fff00008f
:109f040047ff00004bff00003dff00002cff000056
:109f14002cff000024ff000035ff000095ff000027
:109f24000400000079000000e10000006c01000062
:109f340094010000e0000000a4000000bb00000049
:109f44008100000020000000f7ff0000d3ff0000a4
:109f5400c3ff0000a4ff00009dff0000a2ff00005b
:109f64007eff00008bff00006cff00005eff00001e
:109f740067ff00006fff000078ff0000d6ff0000bd
:109f84008b0000001e010000b40100002702000045
:109f94005902000097010000e100000037010000b1
:109fa400f6000000580000001b0000000a0000003a
:109fb400f3ff0000f4ff0000faff0000eeff0000d2
:109fc400f6ff0000cfff000099ff000088ff0000ab
:109fd40074ff000079ff000082ff0000eeff000024
:109fe400930000001b010000f60100005202000073
:109ff400d401000092010000a50100004b01000003
:10a004009b0000003900000001000000c7ff0000b1
:10a01400adff000093ff00008fff000090ff0000e1
:10a024007eff00007eff000037ff000023ff0000da
:10a034002fff00002aff00007dff0000adff00009d
:10a0440025000000b90000004d01000011020000cd
:10a05400190200009c0100009a010000a801000000
:10a0640027010000830000002c000000e6ff000030
:10a07400b2ff000088ff00006fff000093ff0000a4
:10a0840030ff000030ff0000fefe0000b5fe0000bf
:10a0940009ff0000ecfe000010ff000082ff00003a
:10a0a400f7ff00005c000000e1000000a0010000d8
:10a0b40009020000d0010000cd0100008801000069
:10a0c400c90000001b00000082ff00006dff0000bb
:10a0d40012ff00009afe0000d4fe0000affe000054
:10a0e40045fe000092fe0000dffe00005bfe000063
:10a0f4009efe000069ff00003dff000063ff0000ba
:10a104009dff000002000000440000006e000000fb
:10a11400940000007100000052000000fefe0000e8
:10a1240067fe000050fe0000f2fd0000fafe000091
:10a1340068ff0000b8ff00009c0000001c00000045
:10a1440084000000db00000095ff0000a7ff000072
:10a1540024ff000001ff0000d2fe0000c4fe000046
:10a1640040ff000010fe000078fe000000fe00002a
:10a17400e0fd000086fe000066fe00004aff0000cd
:10a1840084ff0000b400000051010000a60100009b
:10a19400120200009d010000250100008300000060
:10a1a400c5ff0000f9fe0000b9fd000089fd0000b4
:10a1b400d9fc0000e0fc00004cfd0000f4fd0000b0
:10a1c4004dfe000010ff0000e6ff00006c000000e0
:10a1d40069010000d1000000c60000004f0000002b
:10a1e400c8ff00006aff0000d2fe0000d4fd00009a
:10a1f40057fd00004afd000008fd000079fd000045
:10a204006bfe000075ff000036000000aa0200008b
:10a214005b030000e40200003e0300008d01000027
:10a2240096000000c8fe000075fd0000f6fb00006b
:10a23400d7fa00005cfb000085fb0000affd0000c6
:10a2440080ff00002001000062030000a302000060
:10a2540050050000db02000017020000d5000000da
:10a2640082fe00007ffd000016fc000077fb00006a
:10a2740081fa000040fc000078fc0000500000005f
:10a28400c8020000800500002d070000f40700004c
:10a29400130600007d0400005301000013fd0000bc
:10a2a400f0fb00002cf900006ff9000090f90000a9
:10a2b4000afb000012fd0000afff00006203000073
:10a2c400c0040000c209000003090000c60a00001f
:10a2d400180800002404000076000000b4fa00000e
:10a2e4008ef8000084f40000aef6000001f70000d0
:10a2f40048fd0000b7020000dd080000260e000043
:10a30400c40d0000e80d00006d040000ee01000023
:10a31400f1f90000ccf2000042f8000078f10000ee
:10a3240019ff00009dfd0000c00500008d0600001f
:10a334008f0700002b080000d4030000a4060000cf
:10a34400a9ff00009dff000071060000e2fa000072
:10a354006c040000fafd000016fd000077ff000009
:10a36400aefa0000b000000001f90000460200004f
:10a374002efd0000110300004b0400004c0b0000f4
:10a38400c8070000590a0000eb050000aff90000ff
:10a394009d0500009cf20000d9fb000045fe000072
:10a3a40055f700003808000092f700002d06000061
:10a3b40058ff00001c05000036090000600500007d
:10a3c4001d090000d90000002fff00005f040000f9
:10a3d40060f2000036ff000070fa0000cff80000c1
:10a3e4009308000087fd0000d107000031fc000045
:10a3f400d0ff0000bcf900006af90000d506000097
:10a40400ce0d0000c90c0000731500007901000096
:10a41400e1f7000006020000b8e000001f0200009f
:10a424001ff80000f0fe00003512000072f6000074
:10a43400a510000060f80000cf030000fb0300003b
:10a444004efa0000a909000095f800005308000026
:10a454003d08000012f20000880800001ff100000f
:10a46400aef500000f080000bef40000280900004b
:10a474000efd000008ff000087fc000092fa0000b7
:10a48400d012000073050000920f0000fd070000c9
:10a494006ce90000a2fa00003bfa00000eee000096
:10a4a4001414000059fd000037fc00002a060000c7
:10a4b40013e60000730a00002500000010070000e6
:10a4c400a20c000026f4000091000000b4eb000090
:10a4d400e40b000089020000b4f40000f41700004b
:10a4e4008bdd0000470500002000000051eb000058
:10a4f40015150000d3f400003cfc0000130200001a
:10a50400d40c00002e1400006e060000edfe0000c6
:10a5140090e1000018f00000b0130000c2f6000043
:10a524004f1900005200000007d900002104000068
:10a5340083f20000f4120000381c00004a020000fc
:10a5440082f300002ee300009df30000ad0800003c
:10a55400901b0000c30f00002bf4000058e700001c
:10a56400fdeb000049020000671b0000900a000098
:10a5740034f000001ef1000043e90000c8030000ad
:10a5840029230000bf180000de080000b2ef00001d
:10a59400aadf000046fa00005e1800002709000048
:10a5a400630200005cf2000032e10000f4fd0000f0
:10a5b400210c00000b1b0000f20f000034f100001e
:10a5c40097f3000002f40000cfff000053100000d6
:10a5d4009b02000010fc0000a9fc0000ceee00006d
:10a5e400bb090000870e0000b0f700003e04000025
:10a5f40074ee000094ee0000b30f0000f4090000b4
:10a6040018030000ea050000abf60000e5fb0000bb
:10a61400ff25000002080000c4e100001afb00004e
:10a62400f8ee0000db0200009213000020f50000a9
:10a6340047f90000100100005d0700008b040000d2
:10a6440040030000920100005e0b00006112000054
:10a654007af50000b4f20000e2fb0000b0ff000055
:10a66400cd0b0000160300000ff000003cfa0000c0
:10a674006809000091000000e4050000faf80000f9
:10a68400d4fe0000db0d00006bf000000c020000a3
:10a69400b10800001ff80000960700003f03000007
:10a6a40063ec0000dff900007d150000940b00004e
:10a6b40016fc0000b6fe0000e0f10000b901000045
:10a6c400a20c000044fb00004b1a00006fe50000e0
:10a6d4000ee400000e25000011ff00004ef1000002
:10a6e4002d0d0000d50d0000a0e4000072fd000057
:10a6f400b4160000b5ed0000b8fd00007a120000a9
:10a704002df800009bf600007806000088ff00008a
:10a7140078f90000880200001204000044fa0000e6
:10a724005bff0000d0030000c2fa000064ff0000d9
:10a734006efa0000d3020000db0000007712000074
:10a74400780b000045cb0000420300003a1f0000d4
:10a7540030f800008ef6000065fe000012020000d2
:10a7640068f400001d0e0000e310000022e8000061
:10a7740040ff00008a15000066fe00001101000081
:10a784005df200008df10000e5080000e909000019
:10a7940021fe00006ef0000001050000d209000057
:10a7a400aaf80000d6fa0000f4fa0000d500000070
:10a7b40085040000f0110000b0f600006add00001e
:10a7c400880e000007110000bdf90000fef500002e
:10a7d400aff90000f80000006f000000830d0000d6
:10a7e4007b05000009eb000057050000561000002f
:10a7f4001d0600004602000066de000015f700009a
:10a80400d61600007709000038f20000d6ed0000eb
:10a81400560f0000d60a00009bf5000040f9000026
:10a8240060fa000059010000e3090000cd020000b5
:10a834004cf60000fff300005e060000340b00003d
:10a8440003fb000090f6000050fa0000970400009b
:10a85400d503000065fc000059ff000098fc0000cf
:10a8640083ff0000fc03000020110000e0fc000056
:10a87400f4dc00006e060000ef1b00004201000043
:10a8840051e8000074f20000f60c000024050000fa
:10a894009f050000050100007bfb00004f03000042
:10a8a400c3130000de0b0000e7dc000084e90000b5
:10a8b400231400003614000084f700004af100005d
:10a8c400f10100002c02000047060000a50700006b
:10a8d4009df70000adf000002e000000fa0e00000d
:10a8e400e70400001cf40000e2f7000099070000f0
:10a8f400f50700001dfd0000c1f90000c3fc0000c5
:10a90400e4ff0000f30100003c0300005aff0000d4
:10a91400f2fb000070ff0000f90a0000440400008c
:10a9240035f00000a0fa00009a0d0000b00a000003
:10a93400b1f800002ded0000c0fe0000bf0a0000c9
:10a944006d020000ae01000066fe0000a4130000ca
:10a9540024110000e0ee0000a5ec0000d4f9000092
:10a96400b8100000b00700003ced0000ccf200007d
:10a97400fe0a0000a9190000130700004bf20000b2
:10a9840041f8000010010000720700007304000089
:10a9940095f80000c5fa000013ff00004904000008
:10a9a400490700009ffd000031f90000c9fd0000c7
:10a9b4007a0500004c05000042fb000032fd000057
:10a9c400a902000067fd000063fd000047020000cb
:10a9d400bf05000061010000e8f80000c6fb0000ac
:10a9e400d0020000ba020000c4fe00004dfc0000ca
:10a9f400d201000030010000d8020000580c000011
:10aa040076fa000088ef0000e4fb0000f50c00007b
:10aa1400fc0f0000eaf6000081eb000033fb0000ad
:10aa2400d90f00009e1000001efd0000e0f700009a
:10aa3400f0080000bf0a000065f70000ddec00002c
:10aa4400a1fb0000fc1000002a0800001af300001b
:10aa540033f80000930d000022140000cff700002b
:10aa64007ee400000afe000076160000990f000044
:10aa740030f200007feb00008e040000361400006a
:10aa84000909000064ef000007ed0000ad040000b8
:10aa9400301300006b0800003ef6000097f700003a
:10aaa400540400000405000064fc0000f0f90000f8
:10aab4004b0100003a080000470300002afa000096
:10aac40001f8000061ff0000780600009e0200000b
:10aad40000fe0000a2fb0000c5080000300d0000cd
:10aae4001cfa0000f3ef000043f60000990900008f
:10aaf4006e0f00009e01000064f300003df50000ad
:10ab0400ad0600005c0e00004a070000b1fa000028
:10ab140071f600008c020000ca070000acfe0000c1
:10ab2400eff6000021fa000071060000280700007b
:10ab34005afb000060f6000078fe00002f0b0000b6
:10ab44007c0a000042030000c6fd00004cfa00002d
:10ab540022fd00004efd000069fd000046020000d9
:10ab640072060000440600009dfe000023f700006a
:10ab74002df9000045000000a8040000ae04000008
:10ab84000102000008fe000023fb0000ccfc0000d2
:10ab9400f0020000210600009802000053fc0000af
:10aba400dcfb0000550000008e020000f6010000ee
:10abb40055fe0000d4000000b10500000c020000a6
:10abc4005bfb0000b8f70000bbfe0000dd070000df
:10abd4006e060000b1fd00005ff700008dfc000070
:10abe400ce050000130a0000c6050000fafc0000b0
:10abf40075fb0000a9ff0000c60200001cff000056
:10ac04003ffa000013fc0000bb0200000c06000029
:10ac14006902000075fe0000ecfd0000290200003e
:10ac2400d80400002c0300007a0200001e0100007a
:10ac340008fe00006af80000ccf900002c050000b2
:10ac4400d80a0000ab03000041f6000055f50000ef
:10ac5400670100000e0b0000c5070000ccfa0000dd
:10ac640059f6000044fe00008f060000b005000005
:10ac740046ff00007ffd0000c4ff0000dbff000072
:10ac84000bff00002501000075040000980300007c
:10ac9400bdfc0000a4f80000a6fb0000b8030000ff
:10aca4002d0700005601000029fc00005efa000098
:10acb400cb040000f6080000f2fd000039f70000a4
:10acc40017fa000066060000ea0900000e01000001
:10acd400e6f70000c1f9000080050000ed0800005f
:10ace400ed0200008dfa0000c1f900005d040000cf
:10acf4005c060000fefc0000cbf600006ffb0000c9
:10ad040026070000a406000065fb000024f70000ed
:10ad140079ff00003b0b0000ad090000d6020000e3
:10ad240049fd00005efa000065fd00002ffd0000f3
:10ad3400b3fd0000b8020000a3060000e405000013
:10ad4400c5fd0000e9f60000b5f90000d4000000dc
:10ad5400d204000087040000ac010000b5fd00002f
:10ad640011fb000038fd0000710300001206000012
:10ad74000c020000f2fb00002ffc0000a500000004
:10ad8400a2020000b601000029fe000066010000d6
:10ad9400b80500007d010000d0fa0000dbf70000d8
:10ada400b4ff000035080000dc050000ddfc0000f5
:10adb40057f7000060fd00006f0600000e0a000057
:10adc400e1040000bffc00005dfc00001d00000069
:10add400a90100003dfd000019fa0000d5fc0000a7
:10ade4003b0200009d050000430400004f010000e9
:10adf400bdfd000037ff0000f90400007e070000dd
:10ae04005204000044fc00003cf7000037fa000044
:10ae1400ea010000ff06000069050000b5fe00001d
:10ae2400e7f80000baf9000047ff00007a060000c6
:10ae34000208000007020000e3fa0000b1f8000075
:10ae440035fe00006e050000da060000dc0000009c
:10ae5400e5fa000011fc0000d60200005a080000c8
:10ae64007b06000062fd0000c3f50000e6f7000069
:10ae7400f3000000d0080000a707000063ff0000f3
:10ae840070f90000a0f70000b7fb0000da0300002f
:10ae9400c10800005f060000f9fe000059fb000035
:10aea4001dfe0000dc030000cb060000710300005f
:10aeb4009ffc000003f6000095f60000b7fe0000ba
:10aec40072060000840700003300000018f8000038
:10aed400cdf700002eff0000bd060000520900005f
:10aee400cf0400001bfe000036fc0000010000003f
:10aef40028050000f7040000d6fe000007f7000054
:10af0400c0f400001cfb000082040000880800005c
:10af14004304000036fc0000d7f9000084fd000063
:10af240087020000c6040000dbff0000b7fa00003f
:10af3400e7f90000d2fd0000ad0300001905000090
:10af44000d03000007ff000009fc000053fd000092
:10af540035010000aa050000c6050000b800000085
:10af6400e5f9000062f60000ddf80000d2fe000002
:10af74001805000017050000430000008bfc0000ca
:10af84004efa000047fc00006c0100004a06000075
:10af94003209000031070000ec020000b2fe00009c
:10afa4008cfa00004bf80000a4f8000023fb00001a
:10afb400d7fe0000730300003c06000042040000ba
:10afc40046ff00007df90000abf9000087ff000098
:10afd4006b0400003d0600004103000008fd000072
:10afe40054f7000071f600002ffc00004c04000030
:10aff4009a090000af0900000104000037fd0000b9
:10b00400edf8000091f900004aff0000320400004e
:10b014007f060000f50300006ffc00005bf60000f3
:10b024003ff50000f1f90000c9000000ec06000043
:10b0340032080000a803000001000000b7fd000072
:10b0440059ff00006f04000034070000570500009a
:10b0540064fe00000ef70000f4f2000080f400002b
:10b064001efc00003e050000a70b00001a0c0000a7
:10b07400060600004dfc000053f500001ef600001b
:10b0840087fc0000f8030000d40700008f050000cf
:10b0940058ff000034f9000062f6000037f80000a1
:10b0a40012fe0000df060000840c0000de0b00002e
:10b0b4006106000095fe0000e6f9000025f9000095
:10b0c40017fb00008dfd000029ff000022ff000097
:10b0d4000bfe00005afe00001fff0000a20000004b
:10b0e400d90100009f0200007e0200005a01000006
:10b0f40052010000cc0000009eff0000edfd0000a6
:10b1040000fc000043fb0000a0fc00007cfe0000eb
:10b11400610000000a030000b1040000a70400005d
:10b1240048030000f7010000ac0000002aff000003
:10b134002efe000099fd0000edfd00008cfe0000d5
:10b14400effe0000caff00001a000000c5ff000067
:10b15400fafe000088fe000054ff000042010000d7
:10b16400fe0300007b050000bc040000b3010000e6
:10b174007dfd000026fa000090f80000faf90000b6
:10b1840031fe0000bf0200009e050000ce05000055
:10b194008f030000f6ff00000cfd00008bfb000095
:10b1a40049fc0000f6fe0000740200006a0600007c
:10b1b4001a0900006109000081060000e400000093
:10b1c4000afa000049f40000faf10000e1f300007b
:10b1d40019fa000041030000760c0000d8110000a9
:10b1e400a910000076090000f5fe000078f50000c3
:10b1f40005f000004bf1000051f800004a01000086
:10b2040010080000a90a00006e080000e201000016
:10b214006dfc00003bf8000032f70000e0fb00008a
:10b22400a6030000810c000049120000f411000084
:10b23400b30a000039fe00006ff100009ce8000032
:10b2440018e700008ded000083f900006707000097
:10b25400d81200001a180000c1140000a80a000047
:10b26400ccfd0000c5f200004fed00008fee0000a1
:10b27400a0f5000066fe00006e05000070080000e6
:10b284002f0700003203000045ff00002ffd0000df
:10b2940035fc000020fe00001002000093060000b0
:10b2a400f5090000930900005f0600009700000004
:10b2b4005af90000b6f2000091ee000087ef00009a
:10b2c4006cf500006efe0000ec070000860e000026
:10b2d400d6100000570e000059070000dafd0000e8
:10b2e400b9f50000adf20000b5f4000061f900000a
:10b2f4007afe0000ab010000330200000f010000e1
:10b30400fcff0000fbff000046000000610200009b
:10b31400460600007b090000f60a0000210900002f
:10b32400900400001bfe0000c7f60000c8f00000f7
:10b33400e7ed00004df00000e2f60000d3ff00004e
:10b3440047090000f60f000086120000cf0f00002e
:10b354006c080000f0fe0000d0f60000eef20000e1
:10b364008df30000a1f700003efd0000df010000a6
:10b37400fc0300006903000079010000570000008d
:10b38400d9ff0000e5000000010400006e07000082
:10b39400560a00009d0a0000460700003001000024
:10b3a4001afa0000f8f30000ebef000074ef00005d
:10b3b400f5f200002cfa000077030000610b000096
:10b3c4000d100000871000000d0d00006406000041
:10b3d400bdfd0000d7f60000d5f30000a5f4000081
:10b3e40005f8000028fc0000a0ff00001501000083
:10b3f400680100007c010000a90100003202000085
:10b40400bf030000a30600005a0900006b0a0000f5
:10b414008f080000ea03000058fd00006af60000ef
:10b4240034f10000fbee000071f0000090f5000024
:10b43400c7fd0000960600008a0d00006811000098
:10b44400f8100000520c000087040000effb00001d
:10b45400b6f500004df3000096f400004bf8000030
:10b46400cefc00007b0000001e020000370200003a
:10b474002a0200007c020000cd0200001c0400002f
:10b484009a060000c50800007e090000e7070000d6
:10b49400f5030000d9fd00003cf7000043f2000072
:10b4a40001f000001bf100007af50000cffc000061
:10b4b400410500009c0c000012110000fb1000006c
:10b4c400e50c0000d7050000b0fd000037f70000d0
:10b4d400f6f3000036f400002cf7000080fb0000b7
:10b4e400bafe0000230000009b000000870100005a
:10b4f400c20200001303000076040000d00600001e
:10b504001f090000390a00001f0800008f03000013
:10b514003afd000061f600000af100007cee000034
:10b5240090ef000011f40000cafb0000b904000011
:10b53400e80b00002910000071100000070d000046
:10b54400820600009cfe000034f80000aaf400000b
:10b5540040f400001ff6000073f90000b7fc00007f
:10b5640097fe000096ff00005f000000e00100006d
:10b574004c03000092040000cf060000b80800004d
:10b584007a090000110800002704000095fe00005d
:10b5940021f80000cef2000004f0000027f00000c3
:10b5a40035f3000018f900001a0100007f080000bc
:10b5b400990d0000860f0000ed0d000087090000c2
:10b5c4001703000066fc000070f700005bf5000044
:10b5d400a1f50000a6f7000094fa0000cefc0000dc
:10b5e4006afe0000baff00005301000007030000d8
:10b5f40083040000f30600009f0900002f0b0000e5
:10b60400860a00000a0700007e010000a9fa000073
:10b614001cf40000c5ef0000acee000024f10000b3
:10b62400a0f6000091fe0000d5060000020d000007
:10b6340051100000f60f0000450c0000d705000073
:10b6440089fe0000c7f800008ef50000faf400003f
:10b6540074f6000067f900003dfc000003fe0000e2
:10b664004bff0000aa0000008f0200002a04000023
:10b67400e90500004a080000060a00002d0a00003f
:10b68400d40700001e030000ebfc00005cf6000081
:10b6940084f100007bef00007ef0000061f4000004
:10b6a40009fb000029030000020a0000560e0000f6
:10b6b4005d0f0000170d000035080000a601000012
:10b6c40055fb000011f700008cf5000004f60000a3
:10b6d4000ef80000a5fa00009dfc00004cfe0000de
:10b6e400d2ff0000a10100007c03000077050000e8
:10b6f40058080000f30a0000cb0b0000140a0000f5
:10b70400c305000096ff00008bf8000070f20000f3
:10b7140015ef00002def0000bdf20000f7f8000067
:10b72400fa00000092080000de0d00006410000022
:10b73400770f0000900b000058050000aafe0000df
:10b744007bf9000066f6000077f500006df6000056
:10b75400e9f8000062fb000036fd000013ff000062
:10b764003c0100008d030000be0500001b08000022
:10b77400b10a00003e0c00006c0b0000dc07000066
:10b78400e8010000b7fa0000faf30000a7ef000098
:10b79400a5ee0000d7f000000ff6000089fd0000c0
:10b7a400650500007a0b0000f20e0000880f00000f
:10b7b4003f0d000052080000da01000013fc0000f5
:10b7c4000ff80000ccf500007af50000bdf600008b
:10b7d400c2f80000fbfa000077fd000046000000fc
:10b7e400d60200003d050000fa070000d80a000058
:10b7f400d40c0000650c000062090000190400006c
:10b8040045fd000083f600004bf1000029ef000025
:10b8140043f0000031f400008cfa0000c501000080
:10b82400610800003f0d00008c0f0000070f0000ae
:10b834009a0b0000110600003900000040fb0000d4
:10b844007cf700006bf500005cf50000d5f6000005
:10b85400eff8000087fb0000aafe0000b201000020
:10b8640098040000960700008a0a0000010d0000f9
:10b87400820d0000410b000074060000ebff000085
:10b8840026f9000057f30000c0ef000054ef000059
:10b89400d7f10000e3f6000081fd0000250400005c
:10b8a400c30900007d0d0000030f0000e70d000038
:10b8b400190a0000ee0400008dff0000aefa00003b
:10b8c400e1f60000acf4000085f40000f8f5000097
:10b8d40034f8000025fb00008cfe0000f10100009c
:10b8e40065050000f8080000400c0000340e00005c
:10b8f400b30d0000720a0000f404000005fe00000d
:10b9040020f70000b8f10000e5ee000012ef00009f
:10b914001df200009df7000069fe0000070500000d
:10b924002b0a0000850d0000cd0e0000640d000000
:10b93400910900008e04000066ff0000bdfa0000bb
:10b9440018f70000faf4000081f400003df500004f
:10b954000af70000d5f9000054fd00002b01000097
:10b9640047050000c5090000ab0d00006b0f000087
:10b97400630e0000710a00006a04000077fd0000f5
:10b984008df6000034f1000092ee0000ddee0000c0
:10b99400fcf1000068f7000004fe00007f040000d2
:10b9a400d1090000ae0d0000420f0000c20d0000de
:10b9b400250a000087050000740000009cfb0000bd
:10b9c400acf7000034f5000053f400008cf40000e0
:10b9d400eff500008af8000015fc00004b000000a1
:10b9e400a6040000be090000810e00009c100000a7
:10b9f4009b0f0000b60b00007c0500001bfe00003e
:10ba040015f7000094f10000e5ee000041ef00009e
:10ba14001df200003af700007bfd0000a8030000bf
:10ba2400be080000950c0000930e0000d70d000026
:10ba34003b0b0000960700003f030000adfe000032
:10ba440048fa0000fcf600000cf5000038f4000091
:10ba5400d0f40000d8f600000efa00004dfe0000fd
:10ba64001d030000e6080000710e00002a1100000a
:10ba7400b4100000780d0000f0070000e70000009b
:10ba8400dff90000f6f3000037f0000060ef00007b
:10ba940008f1000013f50000aafa0000b20000004b
:10baa4001b060000910a0000d60d0000590e00008c
:10bab400650c0000350900002c050000c6000000dc
:10bac4003cfc00005af80000a6f5000025f4000034
:10bad400ecf3000039f50000d0f700008efb000005
:10bae40025000000780500006a0b00005e0f0000ce
:10baf40078100000f70e0000980a00006d040000a2
:10bb040062fd0000bff60000c2f1000075ef000006
:10bb1400e0ef0000abf2000090f7000062fd0000cf
:10bb24001103000007080000f40b0000f00d0000f2
:10bb34004c0d0000140b0000d8070000b0030000f7
:10bb440039ff0000d7fa000062f7000025f5000075
:10bb540007f4000071f400005bf6000088f90000af
:10bb6400d0fd0000bd020000be080000600e000011
:10bb7400de100000621000004c0d0000d50700002c
:10bb8400fd0000000efa00002bf4000081f000001c
:10bb9400adef000053f1000058f50000defa00009c
:10bba400cc000000170600008c0a0000c20d000043
:10bbb400150e0000140c0000ed080000fb0400004a
:10bbc400ac00000034fc000066f80000b0f5000092
:10bbd4000cf40000baf300000bf50000aaf7000013
:10bbe40083fb000044000000160600005f0c000008
:10bbf400c70f000056100000800e0000ce090000a0
:10bc0400a8030000cafc000069f60000d8f1000097
:10bc1400e3ef000066f0000025f30000e1f7000008
:10bc240043fd000072020000490700003f0b0000c2
:10bc3400310d0000b40c0000040b00004d0800009e
:10bc44006e0400002d000000d0fb000017f8000077
:10bc540055f50000a3f300009cf3000031f500004b
:10bc640016f800005cfc00006e010000ce07000026
:10bc7400c40d0000ee0f0000ba0f0000610d0000bb
:10bc8400710800008002000009fc000051f6000069
:10bc940098f20000f1f0000088f1000039f400008f
:10bca40056f800004efd0000320200002407000098
:10bcb400670b00002c0d0000d70c0000140b0000d3
:10bcc4002a08000054040000c1ff00002efb0000fd
:10bcd40049f7000075f40000fbf2000028f30000af
:10bce400e0f4000021f80000abfc000011020000a9
:10bcf40096080000820d0000080f0000910e00005d
:10bd0400a50b0000d5060000480100004ffb000011
:10bd14004df600001cf30000b1f100004cf20000ed
:10bd2400baf4000086f8000018fd0000b30100001a
:10bd3400bf060000240b0000d40c0000cf0c000050
:10bd4400a60b0000a008000069040000c1ff000069
:10bd540003fb0000f8f600005cf4000014f300009c
:10bd640076f3000068f5000090f80000e8fc00009d
:10bd7400f901000039080000220d0000b90e00008e
:10bd8400810e0000e00b0000700700004902000073
:10bd940088fc0000a9f7000054f40000bbf2000086
:10bda400fdf20000c9f4000001f800002bfc0000c3
:10bdb4006b00000071050000770a0000dc0c000035
:10bdc400aa0d0000df0c0000bb090000980500006c
:10bdd400b0000000c9fb0000a6f70000cef400008c
:10bde40084f30000c8f30000a3f500007af8000013
:10bdf4006bfc0000c50000005a060000e30b0000c5
:10be0400f90d0000940e0000dc0c0000b8080000de
:10be140036040000d9fe0000d0f9000022f600002c
:10be2400d7f3000058f3000078f40000ecf60000ab
:10be340068fa000038fe0000c5020000480800004f
:10be4400930c0000dc0d0000620d0000520b00009a
:10be54006b070000bf0200009cfd00000df900000c
:10be6400b7f50000d5f30000b1f30000def40000e4
:10be74003cf7000092fa00006ffe0000fd02000093
:10be8400c70800009d0c0000b20d0000cd0d00009d
:10be9400540b00001d07000025020000b1fc000047
:10bea400f2f70000b3f4000011f300004bf30000bc
:10beb4000ef50000dcf700008bfb00006eff0000b5
:10bec400c9030000ec080000a40c00009d0d000054
:10bed400200d0000890a00003e06000093010000c6
:10bee40061fc0000daf70000e6f400006cf30000e7
:10bef4009cf3000044f5000014f800005ffb000010
:10bf040009ff00005c030000500800007e0c0000e4
:10bf1400fa0d0000b50d00005f0b0000f0060000f4
:10bf2400eb0100007cfc0000bef7000073f400008d
:10bf3400f1f2000064f3000064f5000088f80000ea
:10bf440010fc0000b9ff0000cc030000f207000061
:10bf5400880b00008d0d0000650d0000510b0000e2
:10bf6400aa070000dc02000099fd0000d2f80000de
:10bf74003df5000063f300007cf3000014f50000bd
:10bf8400b6f7000020fb0000a3fe000059020000e9
:10bf9400a3060000dc0a00008b0d0000fc0d00006d
:10bfa400860c0000180900005c040000dafe0000a2
:10bfb40076f9000069f50000f5f200008df200004a
:10bfc40028f40000eff6000093fa00005efe000083
:10bfd40007020000f7050000c5090000940c0000ea
:10bfe400770d00005c0c00008e090000570500006e
:10bff4004100000011fb0000c8f60000f1f300004e
:10c00400fdf20000f0f300002bf600005ff90000e1
:10c0140006fd00008c0000004904000071080000c7
:10c02400190c0000e80d0000830d00001c0b00003b
:10c0340010070000dd01000024fc000035f70000bb
:10c04400c8f300002bf20000d7f2000032f5000024
:10c054008ef8000092fc00004e000000e90300008e
:10c06400ad070000030b0000ea0c0000e40c000024
:10c07400180b0000a707000016030000defd0000f7
:10c08400f9f8000041f500001ff3000003f300007d
:10c094009df400006bf7000005fb0000b3fe0000f8
:10c0a40015020000b1050000bf090000e30c000008
:10c0b400fa0d0000c70c0000b10900002b050000b8
:10c0c40090ff000005fa000075f500008bf20000f7
:10c0d400c6f1000024f3000013f60000ecf90000a0
:10c0e40003fe000099010000f1040000590800005b
:10c0f4000f0b0000740c0000320c0000150a000045
:10c10400a60600003702000037fd00009df800007d
:10c1140010f5000026f3000011f30000bef4000047
:10c12400b2f700004efb00000dff00007b02000090
:10c1340004060000ef090000ec0c0000a70d00004d
:10c14400620c00006909000002050000acff000059
:10c154002afa0000b7f50000f2f2000032f2000003
:10c1640080f300006cf6000040fa000049fe000075
:10c17400c0010000e404000006080000be0a00003c
:10c18400560c0000f30b0000160a00001407000010
:10c194001603000054fe0000b2f900002af6000065
:10c1a400f5f30000a9f30000eff4000068f70000c5
:10c1b400e2fa000073fe0000c90100001e05000041
:10c1c400f8080000470c00003f0d0000660c00005a
:10c1d400d4090000df05000039010000fafb00006b
:10c1e40089f70000adf4000076f30000f8f30000d6
:10c1f40004f6000017f90000bcfc00004000000039
:10c20400420300006e0600009f090000e60b0000d8
:10c21400790c00003b0b000085080000c2040000fc
:10c2240046000000b0fb0000d2f7000039f5000022
:10c234002df400009cf4000072f600006bf900007d
:10c24400d9fc00000c00000034030000cb06000001
:10c25400540a0000660c0000be0c0000490b0000ec
:10c264001d0800001904000044ff00007dfa0000ce
:10c27400d6f6000086f40000d2f30000d2f40000e9
:10c2840023f7000063fa0000ccfd0000f600000074
:10c294001204000060070000a60a0000100c000051
:10c2a400e40b00006b0a000041070000710300006a
:10c2b40000ff000096fa00002ef7000019f50000b8
:10c2c4004ff4000018f500003ff7000032fa0000b8
:10c2d40092fd0000cb0000001f040000ce07000008
:10c2e400400b0000a80c0000360c00006e0a000091
:10c2f4001c0700003a030000bafe000074fa0000b4
:10c3040052f7000047f50000b5f40000a6f5000060
:10c31400fbf70000edfa000019fe000034010000f4
:10c32400490400001c080000190b0000550c000013
:10c334001d0c00000c0a0000da060000ee020000ea
:10c344006afe000043fa00001ef7000025f5000015
:10c35400a6f40000a8f50000f1f70000defa0000e2
:10c36400f3fd0000000100004e0400002908000055
:10c37400ee0a0000fd0b0000650b000046090000fa
:10c3840069060000910200003bfe000052fa000022
:10c3940039f7000035f500009cf4000090f500002a
:10c3a400c1f7000082fa000091fd0000aa0000001d
:10c3b400320400002a080000c70a0000f10b000044
:10c3c4002b0b0000f10800003206000056020000aa
:10c3d4002ffe000045fa00001ef700002ff50000b4
:10c3e4008ef4000074f5000081f7000027fa0000c5
:10c3f4002cfd000046000000f5030000ff070000cc
:10c40400980a0000970b0000f20a0000c20800001e
:10c41400e20500002d0200000dfe00003dfa0000c0
:10c4240023f700002cf500008ef400004bf500000b
:10c4340044f70000e4f90000cdfc0000e6ff000032
:10c44400cf030000d6070000490a0000740b000067
:10c45400a00a0000dd08000075060000b00200001c
:10c464009cfe000093fa000044f700001cf5000055
:10c474005af4000019f5000010f70000cef900008e
:10c48400eefc000014000000c2030000ac07000032
:10c494006c0a0000ab0b00001c0b000078090000c4
:10c4a400d0060000fd020000cffe00009efa00004e
:10c4b4003ff7000021f500004ff4000019f50000db
:10c4c4000ff70000d0f9000006fd00002d00000069
:10c4d400e1030000dd070000e30a00000f0c000088
:10c4e400820b0000b3090000b2060000f202000053
:10c4f400a1fe00008bfa000063f700004ff5000076
:10c50400a5f4000083f50000b4f700007dfa0000f4
:10c5140096fd0000b00000000b040000fe070000c0
:10c52400bc0a0000fa0b0000d60b0000c60900008c
:10c53400b1060000d40200005afe000045fa0000d3
:10c5440018f700001df50000a7f40000abf500008b
:10c55400f7f70000e0fa0000f4fd00000801000015
:10c56400790400005d080000030b0000ef0b0000dd
:10c57400380b0000100900001c0600002302000014
:10c58400cafd0000f7f90000f9f6000010f50000fc
:10c59400a6f40000c0f5000003f80000cffa000084
:10c5a400e5fd0000fe0000009d0400008508000079
:10c5b400fd0a0000f90b0000f50a0000b3080000b2
:10c5c400da050000e2010000bffd0000e6f900000a
:10c5d400def600000df5000093f40000a2f5000063
:10c5e400c0f7000072fa00007dfd00009d0000000d
:10c5f4006504000058080000c70a00009f0b0000f3
:10c60400c30a00007c0800008c050000bf01000084
:10c614009efd0000def90000e1f600000af50000ce
:10c6240090f4000076f5000084f700002dfa000075
:10c634001dfd00003e000000460400002a08000022
:10c64400760a0000700b0000530a00008408000002
:10c65400060600003002000028fe00003ffa000039
:10c6640017f7000015f5000072f4000043f5000010
:10c674003ef70000e1f90000f3fc000017000000a1
:10c6840008040000fe070000710a00008c0b000083
:10c69400b10a0000ff0800006f06000093020000ca
:10c6a40083fe00006efa000026f7000011f500007a
:10c6b4004ef400001ef50000fff600009df9000096
:10c6c400aefc0000c8ff0000d9030000ef07000023
:10c6d400820a00007d0b0000c70a00000209000066
:10c6e40055060000b7020000b1fe0000c2fa0000c7
:10c6f4008ef7000061f5000078f4000024f50000d6
:10c70400faf600006df9000052fc00006bff000017
:10c7140034030000350700009a0900001d0b0000d7
:10c724005e0b0000870900000e0700009c03000058
:10c734004fff000040fb0000bdf7000066f500005d
:10c7440065f40000dcf40000baf600002af90000e9
:10c75400fefb00001cff0000e402000010070000c4
:10c76400bf090000f60a0000250b0000d9090000eb
:10c7740076070000450400003d00000033fc000083
:10c78400b9f8000027f60000f9f4000032f50000c3
:10c79400d3f600003ef90000fdfb0000d8fe0000c7
:10c7a400490200005406000045090000fa0a00008e
:10c7b4008e0b0000700a000077080000be05000020
:10c7c400d7010000c9fd00001cfa000029f7000091
:10c7d4007bf5000029f500005af6000072f800000d
:10c7e40008fb0000f4fd0000260100002f050000f6
:10c7f40073080000730a00007a0b0000840a00002a
:10c80400e808000093060000f5020000f8fe0000ae
:10c814001afb0000eef70000e4f5000016f5000036
:10c82400d1f5000093f70000e6f90000bafc00001f
:10c8340096ff000044030000e30600001c0900000a
:10c84400c30a0000ae0a0000040900003e0700000d
:10c854005704000080000000c3fc000059f90000e8
:10c86400d4f600006cf5000067f50000aff6000098
:10c87400cef800006cfb000026fe00007f010000e3
:10c884002005000032080000ee090000810a0000c3
:10c89400ef0900004308000027060000d80200004a
:10c8a400effe00004bfb00002bf800001df600001b
:10c8b40044f50000f6f50000b9f7000026fa000080
:10c8c400c9fc0000bcff000055030000690600001d
:10c8d40076080000b10900002d0a00004909000093
:10c8e400d107000059050000ac01000005fe00005e
:10c8f4004efa000073f70000bcf5000053f5000089
:10c9040097f60000a1f800002afb0000e8fd0000f3
:10c91400f400000066040000e50600008208000040
:10c924009e09000091090000cf08000036070000ae
:10c93400860400001701000029fd0000bef9000074
:10c9440010f7000091f50000a4f50000d9f60000ee
:10c95400ddf8000076fb000007fe0000190100006e
:10c964004604000066060000410800003409000087
:10c9740064090000c40800001807000096040000c1
:10c98400fc0000003afd0000d4f900001ef700008e
:10c994009cf500009ff50000dff60000f4f80000ad
:10c9a40081fb000012fe00002e0100003b04000089
:10c9b40038060000e10700003209000050090000b9
:10c9c400840800001b0700009a04000030010000e6
:10c9d40062fd0000e9f9000027f7000094f500006b
:10c9e40097f50000d9f60000d7f8000074fb0000aa
:10c9f40012fe00003201000033040000d2050000e2
:10ca0400a8070000d408000004090000a1080000e1
:10ca140014070000bd0400004d01000078fd000073
:10ca240016fa000044f70000a3f50000b3f5000077
:10ca3400e6f60000ebf8000084fb0000fffd0000b8
:10ca44002c010000180400008f05000023070000db
:10ca5400a60800000a0900004808000005070000b5
:10ca6400c204000062010000cdfd00004bfa00008a
:10ca74006ef70000b7f500007ff50000aaf600008d
:10ca84008ff800001bfb0000c2fd0000f500000051
:10ca9400ad030000a60400006c0600002608000098
:10caa400b00800009408000089070000fb0500009e
:10cab4000d03000068ff0000f2fb000099f800007d
:10cac40060f6000098f5000038f60000cbf700008f
:10cad40026fa0000bffc0000deff00003203000065
:10cae40004040000ef040000ed060000fb07000052
:10caf400a8080000730800007d07000087050000f7
:10cb040072020000c4fe000010fb000022f80000c6
:10cb140025f60000caf50000b2f6000061f8000036
:10cb2400f0fa0000affd000083010000b303000031
:10cb3400f70300003605000098060000bc0700005b
:10cb4400660800007208000092070000ad050000ae
:10cb540076020000abfe000014fb000016f8000093
:10cb640047f6000004f60000caf6000080f8000052
:10cb740022fb0000f0fd0000da010000ad0300001c
:10cb84007c030000b8040000bd050000fa060000a4
:10cb940017080000480800001d080000680600008f
:10cba40079030000fcff00001bfc00000af90000f0
:10cbb400c8f60000f3f5000055f60000abf70000de
:10cbc40029fa000002fd000013010000990300008f
:10cbd400cd030000b3030000c504000040060000bc
:10cbe400190700007e080000790800009207000081
:10cbf400bd0500003e0200007bfe0000d9fa0000e3
:10cc0400e8f700002bf60000c1f500006cf6000008
:10cc140067f800000efb000099fe0000b702000058
:10cc240007040000c3030000380400008b04000064
:10cc34008f050000fa060000c90700002a0800005a
:10cc440068070000540500004302000071fe000064
:10cc5400d6fa0000f4f700002ff60000bff500003c
:10cc640070f6000066f800003dfb000003ff0000c2
:10cc74003a03000050040000160400002e040000d3
:10cc840071030000570400008205000098060000ac
:10cc94006b070000e2060000d505000060030000f9
:10cca400dcff00005dfc000046f900000ef7000008
:10ccb400fff5000008f6000065f70000cef900005b
:10ccc4002cfd0000e5010000220400000304000024
:10ccd4009a030000b0020000610200008f0200000d
:10cce4002f040000a8050000920600003c07000085
:10ccf400ed05000056030000050000006afc00007a
:10cd040070f900001ff7000004f6000018f6000098
:10cd140053f70000acf9000040fd0000be01000024
:10cd2400580300003d03000019030000e90100005e
:10cd34001701000018010000bf0200008e0400006b
:10cd44002106000061070000d7060000210500004d
:10cd54005d020000f2fe0000bbfb0000def80000f4
:10cd6400eef6000040f6000086f600002ff8000002
:10cd7400bbfa000038ff0000c8020000e202000015
:10cd84002703000078020000860000004f00000026
:10cd9400060100004b02000013050000ac06000071
:10cda4001f0700004c07000095050000e302000087
:10cdb400c3ff00005afc000074f9000080f7000073
:10cdc40077f6000045f600008cf7000015fa000025
:10cdd40075fe00001002000091020000170300001d
:10cde400f102000051010000710000004c0000003d
:10cdf400a8000000af02000025050000b1060000f5
:10ce0400ac0700006a070000d90500006e030000ab
:10ce14006200000014fd000013fa0000dcf70000bb
:10ce240090f6000055f600005df70000edf90000f3
:10ce340011fe0000890100002003000082030000ad
:10ce4400c5020000e201000068000000abff000022
:10ce54005c000000470100000604000046060000d4
:10ce6400e8060000af0700008f0600005904000028
:10ce7400da01000083fe00008cfb000017f90000bb
:10ce840078f70000a7f6000030f7000024f900004e
:10ce9400d5fc00003b01000063020000bf0200005b
:10cea400120300006c01000064000000ecff0000ad
:10ceb400bcff00002001000019030000050500006c
:10cec4009d0600001d070000ae0600001a050000c4
:10ced400a3020000a7ff00009afc000012fa000061
:10cee40040f800004ff700007df700000ef9000045
:10cef4006dfc000005000000f3010000f5020000d5
:10cf0400a7020000d6010000c2000000b6ff000026
:10cf140006000000920000009f0200003b05000094
:10cf24002206000042070000fd0600003305000051
:10cf3400540300004f00000046fd00008cfa00007e
:10cf440063f800002af7000007f7000078f80000f3
:10cf540065fb000010000000360200005c020000c7
:10cf64001b0300009801000050000000bbff0000fc
:10cf7400d3fe00009dff0000bb0000006b02000018
:10cf8400d6040000070600001c0700003e0700004e
:10cf94000c0600002b0400009401000010ff0000a8
:10cfa4008efc000072fa0000e2f8000010f80000a5
:10cfb4007bf80000f7f90000ddfc0000ceff000064
:10cfc400fe0000009e0100008b010000e400000050
:10cfd4005d00000099ff000079ff0000cdff000014
:10cfe400b60000003e0200006b030000af04000026
:10cff400a905000000060000f5050000d6040000a5
:10d0040002030000230100000cff0000d1fc00001b
:10d01400e5fa000092f900001ef90000aaf90000e8
:10d024005dfb0000cdfd000091ff00007d000000cd
:10d034001d010000e9000000860000000f00000050
:10d04400a8ff0000c7ff0000d5ff00007600000025
:10d054007e010000c701000092020000d803000016
:10d064002f040000bf040000ec0400004004000092
:10d0740067030000c6010000a2ff0000bcfd000021
:10d08400defb00004afa00008ef9000096f9000069
:10d09400abfa00002ffc0000cbfd0000e5fe000011
:10d0a4007aff00005500000088000000a200000084
:10d0b400770000004c0000003800000099ff0000d9
:10d0c400e5ff00002a00000058000000fd000000f9
:10d0d4005e0100000b020000e40200004f030000a8
:10d0e4006b0300002b0300007802000034010000f1
:10d0f400a8ff000040fe000007fd0000effb000059
:10d104004dfb000053fb0000eefb0000c0fc0000e0
:10d1140090fd0000b9fe000056ff0000bcff0000b7
:10d12400d3ff0000c8ff0000ecff0000b2ff0000c6
:10d134003c000000f0ff0000d7ff00009f0000004b
:10d1440076000000b30000002f010000c1010000c0
:10d154000d02000010020000bb02000040030000aa
:10d164000d0300009d0200000602000018010000eb
:10d17400f7ff000004ff00000cfe0000bcfc0000f0
:10d1840058fc00007dfc00005afc0000eefc00008e
:10d19400d5fd000094fe000061ff0000daff0000ee
:10d1a400ebff000033000000820000008a00000052
:10d1b4008c000000ad000000c5000000c5000000a8
:10d1c40097000000920000007e0000007300000041
:10d1d400b9000000be000000e8000000600100008b
:10d1e4008d010000950100001402000057020000a8
:10d1f400cc0100006a0100001e010000470000008d
:10d2040097ff0000bffe00000afe0000fffd0000c3
:10d214008dfd0000bffd0000c0fe000015ff0000f2
:10d2240059ff00001d00000051000000b000000084
:10d23400270100002c0000009d0000000e010000ea
:10d244009900000018010000c10000003a0000002d
:10d25400470000005f00000081000000cc000000d7
:10d26400c8000000ba000000d0000000d600000092
:10d27400230100002c010000e90000009c010000d3
:10d28400880100000901000009010000c10000003c
:10d2940081000000f9ff000061ff0000ecfe0000c7
:10d2a40010ff0000f3fe00000fff000010ff00005d
:10d2b400befe00001eff000074ff000080ff00009f
:10d2c400efff0000fcff000028000000a1000000a8
:10d2d400280000005200000038000000b4ff0000e5
:10d2e400e5ff00000700000002000000300000001d
:10d2f4008400000028000000daff00005f00000046
:10d304004e000000030000000c000000f1ff0000cc
:10d314004800000071000000d2ff0000d7ff0000a9
:10d32400aeff000030ff0000b1ff0000cfff00009f
:10d3340098ff0000b3ff0000f9ff00006d0000003b
:10d344005d000000270000000e0000008eff0000ba
:10d3540066ff0000cfff0000ffff00003100000067
:10d36400750000006e0000003a000000f1ff0000ac
:10d3740014000000750000005e000000540000006e
:10d38400d1000000cc000000a1000000ad000000ae
:10d394006200000005000000efff0000a2ff000093
:10d3a4001dff00006fff00004aff000035ff000072
:10d3b4006cff000056ff000094ff0000b4ff000063
:10d3c40098ff0000c9ff0000cdff0000100000001e
:10d3d400760000002c000000510000001e00000038
:10d3e400cdff0000eeff0000f1ff00000000000090
:10d3f400100000005c00000009000000bdff0000f8
:10d404004a0000003b0000000b0000003800000050
:10d4140042000000bd000000030100003c000000c9
:10d4240019000000c8ff000022ff000092ff000066
:10d43400a2ff00002fff000034ff0000f5ff0000f2
:10d444004e0000000e000000ecff000085ff00000d
:10d45400e8fe0000f5fe00008bff0000c8ff00009e
:10d46400ffff00003b0000002e000000d0ff000082
:10d474003aff000076ff0000d6ff00009fff000087
:10d48400c6ff0000fbff00000f0000002f0000009b
:10d4940044000000e6ff000067ff0000f6ff000004
:10d4a400090000006aff000012000000d6ff00001f
:10d4b40075ff000030000000840000007e000000c2
:10d4c40037000000c7ff000058ff000058ff0000ad
:10d4d400a7ff000005000000440000003300000026
:10d4e400d6ff00003800000001000000aeff00007d
:10d4f4003e000000c7ff00001c00000042000000c6
:10d50400d2ff0000e1ff00009eff0000a6ff000024
:10d51400a6ff00000e00000068000000e0ff00000d
:10d52400b7ff0000d7ff0000cfff0000f5ff0000a9
:10d534001d000000600000008b0000005600000089
:10d544006200000043000000ecff00001d0000002a
:10d55400070000000b000000400000002b0000004a
:10d564006700000039000000140000002d000000d6
:10d57400e6ff0000e3ff0000ffff0000e4ff0000ff
:10d58400050000003a000000230000001f00000016
:10d594002600000013000000390000006e000000a7
:10d5a400720000005c000000ebff0000e8ff0000d8
:10d5b400e0ff0000cbff00002a0000000c00000088
:10d5c4001000000026000000fcff0000daff00004d
:10d5d4000600000039000000730000005d00000038
:10d5e400c9ff0000d0ff0000aaff0000a5ff000053
:10d5f400f6ff00000d00000019000000e9ff000024
:10d60400c2ff000007000000220000000400000028
:10d6140015000000feff0000f9ff0000d7ff000026
:10d62400c5ff0000daff0000efff0000f3ff000079
:10d63400e1ff0000f1ff0000e1ff0000daff00005d
:10d64400b0ff000088ff0000b7ff0000caff000021
:10d65400070000002d0000001a0000002000000058
:10d66400d6ff0000c9ff0000e4ff0000deff000059
:10d67400fdff00002d0000001a000000d8ff00008c
:10d68400d2ff0000c2ff0000bcff0000d0ff00007a
:10d69400f4ff00000c00000015000000e7ff00008c
:10d6a400c8ff0000e2ff0000e6ff000028000000c1
:10d6b4002a000000fbff0000f8ff00000900000042
:10d6c4001f0000000700000006000000e3ff000048
:10d6d400cbff0000e0ff0000e0ff0000f7ff0000c8
:10d6e400eeff0000caff0000d0ff0000beff0000f4
:10d6f400cdff0000f4ff0000d5ff0000b7ff0000dd
:10d70400a4ff0000baff0000ccff0000b6ff000039
:10d71400bcff0000abff0000aaff00008bff00006d
:10d724007aff000093ff0000a0ff0000a9ff0000a3
:10d7340090ff00008dff00008dff0000a5ff00009a
:10d74400b0ff0000a6ff0000b2ff0000b0ff000021
:10d75400a3ff000082ff000075ff00007cff0000b3
:10d7640095ff0000bfff0000daff0000daff0000b1
:10d77400b3ff0000bdff0000b6ff0000b7ff0000cc
:10d78400f0ff0000f1ff0000f1ff0000e5ff0000e2
:10d79400d2ff0000ddff0000edff0000fbff0000f2
:10d7a400b8ff000078fe0000c2fd00005afd000032
:10d7b40063fd0000c8fe00004cff00007cff000079
:10d7c40065ff000080ff0000cb000000df000000c8
:10d7d400670000005afe000030fc00006efe0000ee
:10d7e4007e0000004e0200009302000021010000b0
:10d7f40097020000c2020000c203000054040000ab
:10d804004102000060010000b5ff000010000000ac
:10d81400f5000000bf000000e0000000030000006d
:10d82400940000006a000000fdfe000030fe0000cd
:10d83400aafc0000f0fc000054fe0000c1fe000041
:10d844004aff0000bcfd000054fd00006cfc000019
:10d85400cafa000054fe0000c90000006102000082
:10d864000e02000047000000b7020000dd030000c4
:10d874008905000042060000cf030000c00200003a
:10d88400ae0000000c000000a0ff000056fe0000e7
:10d89400f1fe000037fe00002afe0000bdfe00007d
:10d8a4009bfd000060fd0000c6fc00008ffc000032
:10d8b400c1fc000061fc0000e1fc0000f0fc000081
:10d8c40005fb0000cbfb00007000000023030000f8
:10d8d40013040000b4010000ed0000005402000035
:10d8e40090020000460500000f05000079030000c7
:10d8f40039020000700000007600000095ff00006f
:10d90400cdfe00002ffe00000bfd000035fd0000e1
:10d91400a0fd00007ffc000083fb00006cfa000007
:10d9240008fa00006df9000064f70000ecf900004b
:10d9340070fe0000b70100007a0300006a020000d4
:10d944005b0300009304000059050000e106000099
:10d954001505000008030000840100004a000000cf
:10d96400b6ff000081fe000080fd0000b9fc00004d
:10d9740068fc000011fd00000afd000036fb0000f9
:10d9840082f9000012f900000efa000001f800000c
:10d9940067f90000a9ff0000600300002b050000e8
:10d9a400a40300006a030000d00300001d0300006c
:10d9b4002a0500006d04000023020000fd000000a1
:10d9c400f9ff00002b00000065fe000070fc000061
:10d9d400b3fb00001ffa000080fa0000fefb000009
:10d9e400a2fc000074fc000043fa0000c3f600002f
:10d9f4001bf80000040000001c05000040050000a6
:10da04003802000047010000370300003204000020
:10da1400c70600004906000044020000afff0000f2
:10da2400e9ff00007d00000031fd00007ff90000e7
:10da34004ff8000064f80000c9fa00000afd000075
:10da44003efc0000b5f6000050f3000042fa00006e
:10da5400f90100003a060000a40500002b030000b1
:10da64006b040000aa050000cf0800007508000040
:10da7400f302000005ff000080fc0000ebfb000047
:10da84006cfc0000cefb000030f900004ff70000f2
:10da94006ef900005afd0000e3fa00001ef60000d3
:10daa40052f9000079ff00007703000059050000d7
:10dab400280600008a0600006d05000082060000aa
:10dac400400700003103000054ff000095fc0000f3
:10dad4007ffa0000d2f8000052f8000010f90000ac
:10dae40097fa00006cfb00008ef800005dfa00005d
:10daf4005a0100006c05000048060000e70400001d
:10db0400240600002d070000010500000f0400009a
:10db1400ef000000e7fd000033fc0000def9000028
:10db240033f8000008f600003bf600002cf6000075
:10db3400a1f80000a70200005e0a0000750c0000b6
:10db4400e70a0000730700009a0300007200000057
:10db54009a01000075ff0000ccf9000046f70000b0
:10db64009bf50000bdf3000025f30000bff80000a2
:10db740024010000770500002d090000b50d000008
:10db8400040f0000740b00008a050000da00000096
:10db9400d4fb0000c9f900000ef9000033f50000c1
:10dba40067f200003fef00008bf30000ddfd000092
:10dbb400b804000025090000da080000ef0900009d
:10dbc400f10b00007d0c0000800b00009d030000a1
:10dbd4009bfd000097fa0000ddf6000044f600000b
:10dbe400f6f60000a6f60000f5f200001af40000b4
:10dbf400c6fe0000e1050000ec070000ef0800008d
:10dc0400de090000380a0000520a00003e0b000042
:10dc14005705000028fc0000b6f700005df5000081
:10dc2400def30000a8f400003df3000054f400000b
:10dc34007ffd0000800600001a0b0000290c000084
:10dc44008b0d0000820c000041080000c905000093
:10dc54004201000085fb00006bf6000048f3000061
:10dc640019f3000098ef00001ff3000010fe0000fd
:10dc740031040000ea070000160900003c0c000013
:10dc8400320f0000c50e0000c60b0000a802000001
:10dc9400defc000004f90000f2f20000c2f1000012
:10dca400f5ee000098ee00009cf900005903000016
:10dcb400b208000069090000b20900008b0d0000e1
:10dcc400200e0000050e00000f080000e7ff000012
:10dcd4007afa0000c8f300005df100009bf2000036
:10dce400aef0000053f3000072fe00007106000065
:10dcf400270a00009a0a0000fa0b00008e0d0000ab
:10dd0400bc0d00006f0c0000f2040000bcfd00001c
:10dd14008ff70000bef1000090f100008fef0000cb
:10dd2400f5ee000002fa0000a30300009f080000c3
:10dd3400070b00008d0b0000970e00009d0f0000e4
:10dd4400b00f00003108000093ff0000b5fa000096
:10dd5400d2f10000c3ee0000dbeb0000d2ec0000c7
:10dd640031fa00008d030000c3070000e30900003e
:10dd7400be0b000013100000e3100000461000006a
:10dd840073080000abfe00000ffa00000df3000062
:10dd9400d9f00000a5ec0000edea000082f80000d4
:10dda4003c030000810700001a0a0000880a0000f2
:10ddb400cc0c0000020f0000a0110000e70b0000d3
:10ddc40074010000f6fa0000b7f1000098ef0000bb
:10ddd40054f00000e2ec000016f5000068000000ba
:10dde400940400002f0900000d0c0000990d0000a0
:10ddf4004f0e0000e20f0000bd0c00001b030000ea
:10de04005ffe000023f5000014ef00001fee000089
:10de1400b7ea000047f60000f10200001606000011
:10de2400120700009d060000110b00004b0f0000bc
:10de3400a1110000eb0c0000bb010000c8fd0000b4
:10de4400a3f5000021f10000f1ef00009cea0000be
:10de5400f0f500008d020000c906000094070000e0
:10de6400220600000b0a00005e0d00007511000080
:10de7400240d0000e001000085fd00009cf400007a
:10de8400f1f0000082ee000056ea00002ff70000d7
:10de9400ff020000b806000088070000b906000071
:10dea400350a0000eb0d0000aa110000330b00003e
:10deb40064000000ccfc0000a5f3000016f1000093
:10dec400c3ee000008ea000081f700002704000008
:10ded40009080000290800005b06000098080000fb
:10dee4008a0d0000f5110000b80a00006f0200005e
:10def400f6fd0000fdf50000f4ed0000d4e500009f
:10df040045ec000094fc00004f050000520800009e
:10df1400d2040000f50300002d0e00005b15000084
:10df2400171200007909000006fd000019f2000034
:10df340075ef0000bdea00008fea0000d0f6000093
:10df44004fff00005b060000330c00007309000063
:10df54005c090000bf0f0000330f0000d30700006e
:10df6400d50200002af70000cced0000ccf100003f
:10df74004df100002bf2000022ff00003e080000db
:10df8400b0090000e5090000690500003002000046
:10df940076090000d90b000092050000fe03000082
:10dfa40098fa000071f200005ef600008cf20000a6
:10dfb400f1f100002ffc000032030000b205000064
:10dfc4003107000062050000f50300001d0d00008c
:10dfd40047110000440a0000b80900000ffd0000ca
:10dfe400c9ec0000fbe8000000e40000c3f20000fc
:10dff400e304000092050000010800008c05000005
:10e004003d0400001c0f0000e7110000630b00003a
:10e01400f70400001dfb0000a2f400006af00000f9
:10e02400b6e700001eee0000030000003c080000fc
:10e03400e10c00003c0a0000f70000001a06000092
:10e04400f00c0000030b0000710a00008c010000ba
:10e0540094f5000054f1000027ea0000f5eb0000fd
:10e0640065fa000012030000dd08000061090000e9
:10e074004a0500009e04000043090000840c0000cf
:10e0840081080000a405000000fe00007cf30000ed
:10e0940095f2000022ef0000d6ee000069fd0000ba
:10e0a4007c090000070b0000b509000040040000d3
:10e0b4006aff000041070000780b000076070000ab
:10e0c4002207000017fd00006bf3000040f400007d
:10e0d4008aef0000bbf0000034fc00001d050000c6
:10e0e40047070000d2060000f90400002d020000da
:10e0f400d20a000087100000360a00001f0a000040
:10e104001cff0000c0ee0000b9ea000018e50000a2
:10e1140047f0000032030000240600002408000039
:10e124003f060000730300005a0d000004120000b3
:10e13400080c0000f3050000e3fb000095f4000068
:10e144006df100008be80000feec00006bff0000a6
:10e1540086080000810d00008a0c00000601000002
:10e16400f90200003a0a000062080000550a0000a3
:10e174003204000087f70000acf2000063ea0000fc
:10e184009eeb00008efb0000d00400008d0a00000e
:10e194007a0800009d020000960100006d04000052
:10e1a400bf090000d50800007b070000a60300009b
:10e1b40068f9000054f4000061ed00002deb00004c
:10e1c4000afb0000ae0a0000110d0000c6090000a1
:10e1d400ca0200007bfb000004040000470a0000a0
:10e1e4008a090000b30c0000d9000000a5f5000066
:10e1f40056f1000081e70000c5ed000092fd00002b
:10e20400920a00001d0d000059060000fe020000e5
:10e21400ddfc00004a0500000c0c0000a60700000d
:10e224005f0b00004d00000029f50000a6f300007c
:10e2340086ed000026f00000dcf90000990a0000d9
:10e24400d60e0000c6070000bb040000e6f600007e
:10e25400a0ff0000040a0000ec040000cb12000040
:10e26400a10800001bf90000b5f4000023e700003a
:10e2740061f100002ef40000fafb0000d40d000050
:10e28400d6020000840800009604000024fa00006e
:10e29400830b000066030000ed0800006e1300000d
:10e2a400ecfd0000e3fc0000a5ee000016e7000012
:10e2b4002df900006bf10000890000002f0f000011
:10e2c400790400007d0c0000de00000025f8000049
:10e2d4002a060000f3ff00004e0900008d1600001e
:10e2e4005f0a00008103000066ee000089df000081
:10e2f400f1e9000026ea0000cefc0000c111000094
:10e30400300b0000910e000026050000b3f700005a
:10e314002c040000eefd000034030000d1150000c1
:10e32400e70a0000b90500002af40000fee100003d
:10e334000cee00003fee0000bcf900005f1300008b
:10e344006d110000d80b000004050000a5f30000c7
:10e3540012f90000830000007dfd0000031200009c
:10e36400a3160000870d0000a2030000f5e40000de
:10e37400cce0000019ee000047f800006c04000037
:10e38400480a000043100000de0800009804000062
:10e39400f5fd0000a5f30000d5ff00003c030000dc
:10e3a400bd0b000010170000300d0000d900000064
:10e3b4007eeb000014e40000b3f00000a7f30000bb
:10e3c400a3fd000014100000380e0000290b00000b
:10e3d4003106000048f20000baf80000c1fd000058
:10e3e4002d010000b0150000e9120000f10e00003c
:10e3f40062fb0000ebdf00000fe400001cf50000ee
:10e404005006000079070000040800002b0c0000ef
:10e41400ec070000b706000020f9000009eb00003b
:10e42400def40000af020000e80f0000c71800008f
:10e4340085160000ae0a0000ecf20000a6e300001e
:10e4440069e3000085f3000071010000d7020000b9
:10e45400590f00001c0e0000ff04000039010000e9
:10e46400f5ee0000bff300008b040000610a000019
:10e47400d716000068100000ba03000026f300005d
:10e484007fe50000dff0000011ff0000c00d000078
:10e494005603000020fc00005e0a0000c7000000d4
:10e4a400b100000089f8000004ea00005f030000e6
:10e4b400520e0000211400009c1700009b0900006c
:10e4c4009c050000a7ee000098dd00005ce700005a
:10e4d400b1f700000408000069080000fc0b00000c
:10e4e400f20e0000560400005eff000078f0000009
:10e4f4000eef0000570200000d0b0000ad150000e8
:10e5040036130000e6090000d4f800006fe80000ac
:10e514004bed00002cf700005406000056000000ec
:10e5240006010000010e0000030300005e04000069
:10e5340068f7000024ec000024030000eb0900004d
:10e54400b4140000de140000440700003f00000083
:10e554007ce90000bde400005ff1000086030000d8
:10e56400071100009f040000040400005507000088
:10e5740002fe000027ff0000efef00000ef1000094
:10e584001809000078100000e61800005d10000073
:10e59400f50600006ffb0000fbe4000091e50000bd
:10e5a4003af1000088020000860b0000ca04000053
:10e5b400b50b00004d090000a0ff000072fb000035
:10e5c4001bed00007ff90000860900008e1000009a
:10e5d400bb150000fa0b00004d01000048ee0000de
:10e5e40002eb0000d3f30000a6010000af07000017
:10e5f40077fd00005b080000440600001e010000d7
:10e604001e010000f1eb0000b0f900005d0a0000fb
:10e61400ed0f0000261900005b0a0000110600003f
:10e624003cf60000d0e0000057e600009bf5000037
:10e63400600e000083140000ad0300009a06000081
:10e64400ea02000034fc00001bfc00004eea00005b
:10e654001bf80000000e00008e1500004417000097
:10e66400580a000063010000ccf10000e3e9000057
:10e674007df0000041fa0000bc0d000079050000a7
:10e68400f7f90000bc0b0000e5ff0000a00000004b
:10e6940044fd00008bec0000d9050000380e00009a
:10e6a40032120000c6100000cb040000caff0000b4
:10e6b400a4ed0000a7e600003aef000014020000f9
:10e6c400ab1900007b0b0000acf90000090200004c
:10e6d4000af900002c00000027fb0000b5ee000042
:10e6e40005080000da130000601a00002614000078
:10e6f4007a01000089f30000b4e60000b3ec0000e6
:10e70400c1f70000a8060000fd0c000077fd000022
:10e71400ec040000ff0700007bfb0000aafc0000e3
:10e724006fef0000b4fb0000ae1000005b130000ac
:10e734002f1600000b080000e0fd00000aed0000a9
:10e74400ebe10000aff100002c050000301d0000db
:10e754002313000089f00000c5fa0000c9fc000082
:10e76400aafd0000e902000027ed0000fe01000000
:10e77400631700007c1800005f12000059fc0000c1
:10e7840092f80000fbf300002eee00002df20000d2
:10e7940069fa0000ea0900006c0600007302000038
:10e7a400630900007ffb000099fb0000d9f700001b
:10e7b40060f50000de09000023100000a71300002c
:10e7c4005c0e00007b020000caee0000badf00000d
:10e7d400b2ee0000d8060000371a0000631a0000e9
:10e7e4006cf5000097eb00006a0200006dfa00006f
:10e7f4000101000001f8000039f30000e3180000f3
:10e80400ac190000870c000000fd0000bcf50000fe
:10e81400e2010000c6f7000067ef000081f000008d
:10e82400c4fe0000320c000094ff0000aa070000a0
:10e83400dc0200004cf8000078ff0000bef200008b
:10e844005fff0000060e0000d20f000096130000c8
:10e85400e30600000ef8000003e300009be500005f
:10e8640067020000fe130000f61b0000cefc00004f
:10e8740035e60000950300007cfd00003bfd000030
:10e8840008fd000074eb0000eb1300008e1f000075
:10e894004d0d0000f5fe000036f10000b802000046
:10e8a400f1fc0000f6ed0000b0ee00002cf90000d1
:10e8b400e0140000c40a000081fb0000ef00000027
:10e8c400b4f4000027ff00003bfd000015f5000034
:10e8d400140d0000e5130000f012000056060000bd
:10e8e40041f5000082ed000079ea000050fb0000d1
:10e8f400530a0000a5150000120f0000fee90000f5
:10e904009cf40000e8000000d2f30000b10600000f
:10e914006bf8000054020000c21f0000180d000034
:10e924007f03000002f6000056f6000008fe000017
:10e9340030f200006df4000006fc0000ee0d000053
:10e94400ea0c0000e3f500006eff000041fb00004c
:10e95400b9f800008e03000082f500005b0500009a
:10e9640079160000ba0f000092080000aff800000a
:10e9740026f100007cee0000b2f50000f704000070
:10e98400740f000085100000a6f100005ef1000085
:10e994000505000027f400000401000009fd000043
:10e9a40064fb0000221f0000ff110000e1020000d0
:10e9b400d7f90000e5f2000099fe000056f30000cc
:10e9c400c6f000003dfd0000f70e00001815000021
:10e9d400f7f8000005f600007bf80000fff30000e4
:10e9e4001c040000fbfc0000250400009419000036
:10e9f4008d110000740400005df40000d1ee0000ed
:10ea040044f3000075fa0000cc0500009b0c0000e4
:10ea1400f60c00004ff10000fff300004405000075
:10ea240064f10000afff0000a0fc000066ff0000de
:10ea340046200000860d00004601000065f9000034
:10ea4400eef60000bc010000dded000081eb0000eb
:10ea540037ff000046170000ea1a0000c0f5000066
:10ea6400c1ee000068f50000e1f40000ee040000cf
:10ea7400c6fc0000640600005f1f00006412000072
:10ea84007bfb00003beb00007df20000e1fe000098
:10ea9400c60000006b000000620500006bff000070
:10eaa40042f500005b0a0000faf90000deef000006
:10eab400c3fd0000daf6000043140000191600003c
:10eac4001e060000d20600002afb00003bfd0000e9
:10ead400a4eb0000acdd0000c1f900001720000029
:10eae400bb2b000063ff00005ae4000000f40000a8
:10eaf400c2f50000b6ff000036fd0000dbfc00009c
:10eb0400621d00006f1f0000cfff0000ece3000057
:10eb140006ed0000690900001b0d0000a5fb0000c4
:10eb2400d7f60000e0f80000a5f70000fe11000091
:10eb3400f3030000bfed0000defb0000d5f700008a
:10eb4400db090000d30e00003d040000050e0000a8
:10eb5400a7070000c8fd000081ec000006db0000f0
:10eb640032ef00001e1a0000ae2d00008d0d0000d3
:10eb7400bae7000045f100003bf7000084f500000f
:10eb8400bffc0000a1fa00009817000061260000f5
:10eb94006e06000048e70000c2e50000b50400006e
:10eba4001e110000c7fd000018f5000015fe00004e
:10ebb400e6f8000011060000e20800002bf0000057
:10ebc40035fd0000bdfd0000d3ff0000a90b0000cf
:10ebd40098030000b70c0000620b0000fefe00006a
:10ebe40071f30000d1e2000004eb00008f09000083
:10ebf40078250000281a000020f00000fdee000037
:10ec0400bcf8000040f100000efb0000defb000039
:10ec1400120e0000f52500009e0e000098ee000084
:10ec2400b7e60000f3fc0000ba0e00003400000058
:10ec340097f400005dfe00001af90000d600000001
:10ec4400010f00006af60000c0f7000040fb00005e
:10ec54009afa0000840c0000a7070000d40a000000
:10ec6400d80c000088020000d2f600006de4000019
:10ec740012e70000b2fe0000af1f0000d720000022
:10ec840068f9000079f20000c8f600009aec000070
:10ec940050f5000008fb00008d0d0000f725000072
:10eca40027140000fdf20000b9e8000020f800007d
:10ecb40068070000c1ff000094f500008d02000009
:10ecc4009bff0000a80000005f0d000085f4000019
:10ecd400a9f20000f0f900002dfb000091100000e3
:10ece400ed0c0000370a000083090000e8fd000075
:10ecf400bcf6000075e800006ded00003600000071
:10ed040045190000a91800005efa00006ffd00001c
:10ed140066f50000e5ea0000fff3000097f7000045
:10ed2400251500001e2300002610000068f50000d1
:10ed3400dbea0000dffd0000d000000059f800000d
:10ed440073f60000d00500004a0b0000e500000047
:10ed5400580500001af4000013f00000d0fb000076
:10ed64000bfc0000df0d0000061400001a0d00006b
:10ed74005e030000dff60000a0f4000032f10000a2
:10ed840026f50000360500000814000057020000b4
:10ed9400c4fe0000c408000042f50000f2f00000c8
:10eda400e8eb0000c5f8000050190000771c0000d3
:10edb400d60d000095f80000e0f40000f2fe00001b
:10edc40075f200009eed000016fb00007b130000ae
:10edd4002316000082fe0000a0fc00003df00000ad
:10ede40060f000003ffc000067fc00008c10000095
:10edf400551c00004b1000003af80000c9ed00005b
:10ee04004af40000bafc00001ffd0000db0400000f
:10ee14004d0c0000aaf9000070060000c9060000ad
:10ee2400d2f10000abf300000cf00000c2010000be
:10ee3400c91500004c1600004b0a0000e0fd00005c
:10ee4400a2f9000077f50000eaed00007eee000074
:10ee54004d060000181c0000180f000084fa000082
:10ee6400d8f8000067f100009df4000046f90000a6
:10ee7400effe0000b8150000221d0000900b0000fa
:10ee840003ee000046ee000038fd00000902000019
:10ee94007bfe000076ff0000040b0000dbf800009e
:10eea400ae010000ef05000092f4000087fb0000b3
:10eeb400c8f1000006ff00007f1100005f1400008d
:10eec400110d00002dfb000046fb00004ff8000070
:10eed4009ff00000c4ef0000380000000618000096
:10eee400340e000051fe0000defc000023f200009e
:10eef40065f3000043f6000056fd0000c81300004f
:10ef0400321d0000e30f00003af10000faed0000aa
:10ef14007dfa0000a0fe000066fe0000abff0000ca
:10ef2400bc0d000059fb000041ff00003d0700003c
:10ef340039f300004afa000050f2000067fd0000b7
:10ef44005b130000c3130000880d000006fc0000e2
:10ef540066f90000c8f800006aef000004f0000041
:10ef640082010000051a00005710000064fa000036
:10ef740067fa000031f200002ef5000006f90000e7
:10ef840085fc000046140000a21c0000ff0d0000d8
:10ef9400baef0000a7ec000080fd0000b9010000fa
:10efa400c6fe00008cfe0000d80a0000b2fa000081
:10efb4008aff0000b105000007f5000096fc000080
:10efc40081f30000a6fe00001c10000001130000e5
:10efd400380d0000e4fb000095fc000015f700006c
:10efe40022f0000037f000001c0100006c19000042
:10eff400120c000023fe00001ffd0000ecf20000d4
:10f00400b7f40000acf3000038fd00004f15000019
:10f01400a31d00002a1000005ded00007ded00003e
:10f02400b5fe0000ecff0000a0ff000094fb000010
:10f03400840e000051fd0000acf800006e070000d3
:10f0440072f400002101000048f5000092f800006d
:10f05400671000003c100000b311000095f9000097
:10f06400abf80000e4fd0000e0f1000017f300003d
:10f07400b5f90000a815000039120000d1f900000c
:10f08400c3fd00001af40000eff60000b3f800001e
:10f0940014f60000d81000006d1a0000721400006d
:10f0a400a5f5000093e600001b000000020000002c
:10f0b400b9ff000054fb0000b1090000a70a0000da
:10f0c40013ef00002a010000cdf9000032ff000018
:10f0d4008f030000f9ef0000ca0800007e0e000054
:10f0e40088100000890400007def00005d0300002b
:10f0f40070fc000092f10000d5f70000d804000075
:10f1040053160000f6fd0000cdf80000a3fe000039
:10f114001bf6000082ff0000adf3000007ff0000b3
:10f12400c71600000d15000044090000bbeb0000e9
:10f1340013f600005c0200004dfa000093ff00008b
:10f14400b7020000690d00000af7000031f8000062
:10f154001d05000096f800009f0400009ef30000c7
:10f164002ffa00004c120000c50d0000f30e000041
:10f1740019f50000e1f80000a3060000ffee00000e
:10f1840082f50000dd0200001a100000d208000021
:10f19400def3000057ff00004cfb0000c4fd00003c
:10f1a400e0f9000090f20000b50e000086160000a1
:10f1b400f611000077f800009aeb0000b20200009c
:10f1c4002efc000003fc00008a010000200a00005d
:10f1d4007f040000f1f000001802000078fc000039
:10f1e4008600000009000000d4ee0000c7080000fb
:10f1f400f60f0000cb1000001204000028f00000fd
:10f20400b8030000f3fa000017f0000033fd00001b
:10f21400ed060000941000003cfb0000c1f9000062
:10f22400c9ff000087f800009f00000059f10000aa
:10f234002fff0000b8150000ad130000a90900005d
:10f24400e6ec000078f600000601000090fa0000e9
:10f2540038ff000091020000130c000016f80000b3
:10f26400c9fa0000f102000021f60000f8020000d3
:10f2740013f50000fdfb0000f51100008c0d0000eb
:10f28400b60c000040f800004bf80000ee0000004f
:10f29400a0f100002cf700004f010000240f000033
:10f2a4008906000034f70000520200009af50000bd
:10f2b400d5f9000039fa000065f700007a12000061
:10f2c400731400005b0c00008ff80000f7ef0000df
:10f2d400bafd0000dbfa000075fd00009902000091
:10f2e400360d000048fe000083f20000a106000075
:10f2f40038f80000e0fc000052fc0000d2f30000eb
:10f30400950f0000101100005c0b0000d9fe0000f6
:10f3140068f40000c501000058f700002df3000058
:10f32400a3fe0000480a0000680b00005cf800001f
:10f33400f3ff0000bdfb00000cf6000094fd00008c
:10f34400cff40000d1070000de1500001a10000001
:10f354005f000000baee000064fa00004afc0000fe
:10f3640005fc0000d8020000140900005906000042
:10f3740086f0000097ff000065010000f4f800002b
:10f38400ae010000a3f20000fc00000049130000dd
:10f39400ee0e00009c050000f3f30000eefd0000fb
:10f3a400bdfd000057f000007ffd0000cc07000009
:10f3b400380d000080fb0000e5f50000f0030000bc
:10f3c400b1fa0000c3fe00001df70000d1f60000f2
:10f3d400651100005a160000100a000080f30000b6
:10f3e400aff4000025ff0000a5f90000b4ff000001
:10f3f400cd040000620b000039f900009bf300000b
:10f404004408000048fb0000bafe0000e1f90000d7
:10f414002ff300002b0e0000d3140000390c000061
:10f4240070fa0000aef7000026ff0000e6f30000cb
:10f4340086f7000008010000850d0000e8050000c3
:10f444000cf600008404000032fa0000a0f600006c
:10f4540003fc00005df60000da0c00004518000013
:10f46400820c000039fa000036f40000c2f80000f3
:10f4740068f800000aff0000a7040000230e000043
:10f48400f0fa0000c1f1000001090000a8fc00002e
:10f49400f2fa0000b6f900001df40000f70d0000b8
:10f4a40085160000760c0000ccf900000cf8000072
:10f4b40034fa000054ea00008502000070140000d1
:10f4c4005d0c0000eeff000096ea000044f300002b
:10f4d40078000000830500002d0700006af6000094
:10f4e4009efb0000721400008e1200009afa0000c5
:10f4f40062ee000085f6000051090000431100008f
:10f50400f7fd0000b6f70000beec00006df400004b
:10f51400461b0000ff050000e0f70000abfb000005
:10f524000cf1000087070000aa0c0000b5040000dd
:10f53400ac080000920700002bfe0000bae70000b0
:10f54400a3ef0000410500004f130000f9ff000085
:10f554001eee0000110a0000c9090000b9040000f1
:10f564008cee0000d5e10000240a0000b91f000061
:10f57400921c00002dfe0000fce900007bf200005c
:10f584000af900004d03000015ff00002c0c0000d8
:10f5940059fd000043fb00007a100000eff1000069
:10f5a40011f8000007f7000057f900008d1600005d
:10f5b400c4110000910e00007600000044f0000029
:10f5c400dff00000e0f50000d6fd0000ce0c0000e6
:10f5d40075ff0000c3f300000d160000c80400000e
:10f5e40075f2000022ed000072eb00008b120000a7
:10f5f4008c1e000099150000f6080000f6f10000ca
:10f60400abe20000fef300008b000000a80c000039
:10f61400850a000056ef00005c1200006e0d000029
:10f6240093ef000001eb000071e70000f60f00000b
:10f63400731d00001a140000a3060000e4fb000080
:10f644009ef4000014eb000096f800000700000090
:10f65400290e0000b0fe000040fd000095160000d9
:10f6640030fa0000c6ed00008aea000014fa000037
:10f67400ed170000b4180000a40f0000c4ff000040
:10f6840079f70000ddea00003ef000004e020000c1
:10f694005a0e0000e40c000023ee0000a90600004e
:10f6a4004f1100006bf30000caef000012ee0000df
:10f6b4009506000000190000b013000028060000a1
:10f6c40070fa00003efd00008af100000ff3000014
:10f6d400c2fc0000260700000108000044f90000f5
:10f6e4007210000050040000beec000035f500006c
:10f6f400e3f300000109000027180000471300008d
:10f7040081060000a5f700001cf200002ded0000aa
:10f71400bdfb0000eb050000e00f0000ea02000062
:10f72400d3f400003f0f00006afb000058f1000012
:10f734001ffb0000c4f30000dc0b000021160000d6
:10f744005c1000009604000074f700008df00000c7
:10f75400dfe70000db050000e9130000c00500003e
:10f76400d5f300001ef500009f0d00005dfd0000b4
:10f77400e1fb000098fc000086f00000100b000084
:10f78400c416000094100000530000001ae30000a7
:10f7940008f10000af120000a70b0000e4fe000017
:10f7a400fbed0000bbe600001c1d000089180000f2
:10f7b40053ef000027f400008ff000008e030000d8
:10f7c4003f100000a3090000090d000075040000ab
:10f7d4001bf50000a3ed00005bfb000058000000d7
:10f7e400ba020000c8f4000012fd00005e1a000016
:10f7f40009080000affc0000cdea0000eeea0000ba
:10f804009004000090120000a1200000fe0d0000f2
:10f8140023f0000016e00000d7ef000040060000cf
:10f824000f0e0000f10200006df000002215000030
:10f83400fe0c00009bf20000f4eb00007cec0000e6
:10f84400ea0e0000a11400005b1400002809000067
:10f854003afa000038ed000084ea000019fd0000c7
:10f86400670a0000c904000022ed000038100000ff
:10f874001714000047f7000018eb000009e8000027
:10f88400780e000019130000de1100005e0f000066
:10f89400b5ff00008bed000072e30000cbf6000022
:10f8a400680a0000550e0000a4f10000e7090000fa
:10f8b400fc160000e6f40000c8e9000027e300009d
:10f8c4003f0e0000281b0000510d00006b090000d2
:10f8d40097000000e9f90000f7e40000f4ef0000ed
:10f8e400b20400008314000011fd0000ebf50000d9
:10f8f4007416000034ff0000a9ee0000cae3000003
:10f90400dffd00002f1f0000a01000006b070000a7
:10f9140054fd00002600000021f3000071ea0000fd
:10f92400aefa0000890d00006e0d0000e5f0000045
:10f93400fa040000870d000021f70000baeb000074
:10f94400eded000032110000371800000a0d000030
:10f95400f9ff0000d7f900000e0100006eee000070
:10f96400adef0000edfe000088100000d30c000095
:10f97400f0ef000096070000b201000048ef00001d
:10f9840060f7000035f70000091400006716000056
:10f99400fe07000001fb00000cf400003bff000028
:10f9a4004cf20000c0fb0000e40200007b0f0000ea
:10f9b4008e01000042e700008f110000f6fe0000f7
:10f9c40081f500005dfd0000c0f000000c14000093
:10f9d400101100007c070000f6fd0000c4f70000d1
:10f9e40021010000bbef00005df70000d7fd00001f
:10f9f400971000000c06000052ee0000c50e000037
:10fa040077fa000024f70000f9fa000070f0000013
:10fa1400ae130000ec140000fa0b0000a3fb00007e
:10fa240092f00000b5f90000ecf6000000010000bf
:10fa340014ff0000e50c0000960000008ef10000a9
:10fa4400190f0000c4f7000026fa0000f4fa0000c1
:10fa540000ef00001d1400003b1700009f0e000083
:10fa6400e8fc0000edec0000abf50000caf6000075
:10fa7400fefe0000de0200005c1000005cfe0000e0
:10fa840036f400006f0a0000e3f300004ffc0000ae
:10fa940023fa0000c3f5000085180000b01500002b
:10faa400c20a000013f500003eea00004cf6000014
:10fab400aafe000031070000e0030000290d000049
:10fac4009df50000b5f40000cc08000005f6000028
:10fad400f7040000eef600008cf500007f1600002d
:10fae40097130000830b000031f400007eee000049
:10faf40082f50000acfb00003f0b00000405000091
:10fb04003b050000d0f0000067f80000ce0c0000b8
:10fb14001afd0000be0300006fee0000c2f40000f6
:10fb24003e1a000057180000f407000004ee00001d
:10fb340041ee0000d7f70000ce040000390a0000af
:10fb44008bff0000c206000029ee0000fffc00004d
:10fb5400b40d000026fb00004b040000abe90000dc
:10fb64003bf90000931d00001a1400007507000003
:10fb7400b1ef0000a0f30000aef70000dbfd0000d1
:10fb8400750400004303000092080000e7ed000044
:10fb940050050000680900009af8000023fe0000e8
:10fba400ace60000df090000b8200000711000007e
:10fbb400ad0000001be90000a1f20000abf9000059
:10fbc400bb050000bf050000fc080000cd040000d8
:10fbd400b4e800005b0800000f04000008fc00000b
:10fbe40036fd00009feb00002712000052170000b2
:10fbf400900c00007b00000058ec0000a2f4000010
:10fc0400e9f600000f070000d00500001006000010
:10fc14005ff60000dbf200006a17000014fc00002d
:10fc240036f50000e3f20000ccfa000025200000c5
:10fc3400a40f00007008000082f80000dde7000057
:10fc44006bf2000091ff0000110f0000d6090000c4
:10fc540061ff00008fea000071050000f21000004f
:10fc64002ef3000067f8000040f30000ce0c000003
:10fc7400e2180000f80500007608000024f60000f1
:10fc8400f5e90000a1f30000870700005f0d000004
:10fc94005405000075ed0000a3f50000741b00007e
:10fca40090ff00007cf00000b9f100004dff00005f
:10fcb400691c0000bd0d000073050000e2ff000098
:10fcc400f1ef0000baeb0000effb0000b80b0000fe
:10fcd400920d00001802000007e600006e08000004
:10fce400c11100002bf4000047f7000009f30000e5
:10fcf400550c0000c215000022070000d8050000c2
:10fd04008ffc00003bf0000014ee0000cf01000067
:10fd1400500a0000520c0000cef7000037e8000043
:10fd24009c140000fc0900006df2000094f6000031
:10fd3400dcf500005d1200007e1500005206000094
:10fd440096010000f7f40000cfee0000caf50000b1
:10fd5400f10400005f0900003d0d0000adf5000056
:10fd6400a9ea000063130000830200009af7000070
:10fd740065fa000072f200008b1400006d1400009c
:10fd840023070000f000000091ee000015f10000d0
:10fd940018fa0000d70600001c08000059080000eb
:10fda400d9f00000e4f10000ef16000031fd00007e
:10fdb400aef80000c1f5000086f70000151c000035
:10fdc40044110000e40700007ff9000050e800003f
:10fdd400dcf20000690100003c0c00005708000040
:10fde400a10100006deb000095010000331100003b
:10fdf4007df50000f3fa000039f4000098060000d5
:10fe0400b01800003b09000074080000c9f50000a8
:10fe140033e900001bf50000f7060000ec0b0000be
:10fe2400df05000098f100002bf50000a11400008c
:10fe34006d01000002f3000051f40000b3fe000065
:10fe440070170000d80e0000f30600000400000044
:10fe54009fef000086eb00001cfd0000750b000006
:10fe6400610d0000f00000005ce60000840a000060
:10fe74003c100000ddf3000036f7000060f30000e2
:10fe8400b90d000021150000db060000af050000dd
:10fe9400fbfb0000c2ef000097ee0000b40200007c
:10fea400580a0000420c000016f600006ae900003f
:10feb40002160000240800008ef2000056f600002e
:10fec400c5f600008d1300006d14000083050000ca
:10fed4006e01000044f500005eee000017f600001d
:10fee400360500002a0a00007f0d0000a3f100007f
:10fef40095ec00001c160000e4000000ddf6000094
:10ff04006af90000faf40000f5150000cc120000b4
:10ff140027050000ff000000d5ee0000fcef000004
:10ff2400e3fb0000c1060000a6090000e30800008e
:10ff340039ed000026f20000d81600008cfd000008
:10ff44004cfb000066f70000d4f400009b1900008d
:10ff54007512000048070000a0fa00004be80000fa
:10ff6400cef30000d4020000eb080000ee0600000f
:10ff7400ff040000f1eb000056fb00003713000003
:10ff8400b5f8000092ff00008df40000eaf90000cb
:10ff9400861a00004d0f0000d808000005f6000086
:10ffa40068e70000ecf70000410300000f090000bf
:10ffb400e4080000bd02000014eb0000bdfb0000db
:10ffc400f80f000093fc00007602000029f1000005
:10ffd400bffa00008a1c0000ce10000022070000b7
:10ffe40038ef0000aee80000c1fd0000820400000c
:10fff400b00800008f050000afff000025ed0000f1
:020000040001f9
:1000040007010000de0c0000b9fa0000de02000067
:1000140042ef000072000000b01c0000540f00000a
:100024007c050000feea0000a5eb0000d6fe0000ff
:10003400580600009c0900006b04000093fd0000ba
:1000440014ea0000b5040000f20c0000dafc000021
:10005400c1000000edea0000a8060000e81d000051
:10006400d10d0000d601000097e70000f2ef000078
:10007400d70000001e070000ba0700004603000076
:10008400f7fb0000b0eb0000ea0a0000940800004f
:10009400bdfb0000bafd0000dfeb0000840f000090
:1000a400781b00004e0a0000b8fd000010e90000b3
:1000b40033f600000aff00006c050000040700008e
:1000c400f5050000a0f600004eeb000059120000f8
:1000d400950600006ffb00001af60000e9ed000031
:1000e400681a0000921900004107000093f800000c
:1000f400a4e800004bf9000008fe00009806000088
:10010400e60600007e090000bff6000035e70000a7
:100114001f12000091040000f4fd00001cf8000010
:10012400b8ee0000fe1b000045140000cd040000e2
:100134006af9000011ec0000f3fa0000cdfc0000a5
:1001440090060000320600006608000012ee00006f
:100154001ded0000071a0000f5000000b5fb0000cb
:10016400c1f00000d5f5000033230000ae100000fc
:10017400fe02000041f5000010ec0000a4fb0000aa
:100184003aff00004708000078060000a1060000be
:100194002aeb0000e4f400001618000047fc0000fd
:1001a4007afc000087f00000b0fc0000e0210000b1
:1001b400e30b0000fe03000031f40000a5ec000096
:1001c400ebfb0000cd0000007e080000f0050000fd
:1001d400a301000025e80000d4010000211500005f
:1001e400dcf60000fafb0000e4ee00006307000008
:1001f4001e20000059080000f7020000c9ef0000ab
:1002040048ee000084fc0000e6040000380800000a
:10021400c9050000d6fb0000e0e80000540d000012
:100224003e0c0000f2f4000078fb000056ef0000e2
:10023400a0100000ec1b0000650700005e01000038
:1002440036eb000098f0000023ff00009306000046
:100254004c0700006b050000f3f40000fded000006
:100264008e1300003604000022f8000057f8000046
:1002740037f00000b2170000971800004007000094
:10028400adfc0000ceea000042f60000e2fe0000f1
:10029400ee0500006c0500006d0600004af4000045
:1002a4002ef00000a2130000d1ff000032fb00007a
:1002b400acf5000072f00000681c0000f5170000a7
:1002c400ff0600005cf80000ecea0000b3f900004f
:1002d400f3fe0000fa050000340300004d0700009f
:1002e400cbf20000b9f20000fc15000053fc000042
:1002f40043fa0000a6f1000069f500007021000037
:10030400881400004904000065f600000eef0000a8
:100314009df90000a2fd0000700400000f0400001d
:100324003509000082ed0000eafb0000141500000e
:10033400a7f500008bf80000e1ed000027020000a3
:1003440055230000640d0000ec00000030f60000ae
:1003540035f500005ff70000cefb00001404000038
:100364007307000066070000cae8000048050000a3
:10037400481200002cf100006cf60000f3ec0000c1
:10038400e40c00005d2300000c080000c1fc000028
:1003940036f400004afc000025f8000018fa0000ba
:1003a400e7020000730700006908000095e60000fa
:1003b400b1080000b010000048ef00003bf7000057
:1003c4003deb00006c1100003f240000c10500005b
:1003d4001efc0000bcf2000056fb000005f8000003
:1003e4007efc000029030000030900003f0900000f
:1003f400f1e60000480800007c0b0000f7f0000064
:10040400a4fb0000a3ec00000c1200006920000013
:10041400a3030000acfb0000d0f30000ae0000001a
:100424005df900003cfa00000400000081080000af
:100434009c07000090e70000c60d00002e0a000093
:1004440094f000007af80000eeea0000351700008e
:1004540082210000ca0400002bfa0000bcf1000055
:10046400f5fe000059f90000a2fb00005a0000004c
:100474009e0c00008a07000040e80000800b00008a
:10048400a6050000f8f30000eef9000007ed0000f7
:100494003c170000f01d00005904000082f8000021
:1004a4004bf30000be02000016f800008cfb0000b5
:1004b40067fe0000e20c000041080000e5e50000d2
:1004c400cd0d0000a20400005df4000012fa00004b
:1004d400afeb0000d4190000bf1d0000df030000d3
:1004e4003ff70000aff20000e70200004bf8000005
:1004f4005afb0000e0fd00006e0e00005c050000e9
:10050400b7e90000870f000034ff000066f4000024
:1005140013f80000f3ef00003d1d0000f119000086
:100524007502000099f300004ef400003908000041
:10053400c1f600009af9000091fd00008b10000044
:100544007a0a0000aae10000200a00004d0600001b
:100554007ef700006efa000038ea0000251a000059
:10056400811d0000730100009bf100002cf30000ca
:10057400cb10000059fa0000caf2000071f9000023
:100584000a0e00002310000004e100001807000018
:10059400d10b0000b3f50000e2f8000071e70000a1
:1005a400c317000001230000c902000093f10000fa
:1005b400d6f00000460d00009ffc000001f2000090
:1005c40049fb0000900f0000ac14000092e0000012
:1005d400f8fa00009c10000078f900005cfb0000b1
:1005e4007ee90000e40d0000ed2200008f0300000e
:1005f400d5f20000bff1000017100000d102000086
:100604008dec000042f700008d080000c9180000be
:1006140046e8000099f20000cc160000f7f800004c
:1006240032f8000006eb00005b050000d82800004b
:10063400a1080000a5f20000f1ef000093080000fb
:10064400c506000090ee0000d6f80000f408000093
:10065400661b0000c3ee0000e3e100004216000048
:10066400420300001cfa00000ef0000054f70000e2
:1006740001250000c70e000016f40000adf20000d2
:100684005f060000b90e0000d5ee0000b7ef0000d1
:10069400de010000bd1900008aff000090de0000aa
:1006a400b30e000025090000a7f60000eff40000d7
:1006b400eaf00000be1f00004819000074f50000b5
:1006c4005cf2000062fe00007f0c0000b8f5000040
:1006d40093f0000041040000b916000096060000e3
:1006e40085da0000c20200004a1300005cf8000032
:1006f400c2f80000dfec0000381400004e1f0000b8
:10070400f1f80000a3f3000049fd0000110f000000
:1007140014fb0000f5ea000025fc0000a511000010
:1007240035120000d8df000049f80000d41700009b
:1007340090f800006cf80000fdeb00002d0b0000a9
:100744001f26000061ff000019f20000b6f7000048
:10075400920c000079030000baea000088f9000056
:10076400fd0c00006a170000ede9000034e9000008
:100774007518000040ff0000f4f700008def000042
:10078400e8fd0000c2260000d00800001ff20000af
:10079400edf500006a0700001e0a000008ed0000e5
:1007a400d6f40000b70800004718000031f7000035
:1007b40015df0000cc120000f8070000a5f60000c9
:1007c40044f400000af40000bb2100006e12000093
:1007d4005ef30000b1f5000062030000460e000065
:1007e40025f10000bfee00004903000015170000ca
:1007f400b0030000f7db0000a70a0000be0f0000f2
:10080400dcf40000f0f50000caee0000d51b000087
:10081400831c0000d2f5000077f300008cfd00007b
:10082400910e00002ff80000ffec00005f020000b2
:10083400671400007b0c00002ddc0000d6fb0000d8
:10084400d317000029f800001ff80000eeec0000a8
:10085400110f0000ba2200009dfa000055f30000b9
:100864003bfb00002710000053010000b7e7000025
:100874001efa0000a70c0000d1150000c6e8000015
:100884009fee0000c019000077fa00003af600005d
:10089400bfef00002f0400001d2700000a03000022
:1008a40072f20000bff600000a0900003d090000d2
:1008b400f5e90000dbf80000150c0000e515000068
:1008c4008ff30000acdf00001416000017070000cf
:1008d400f1f300006ff4000042f80000022200006f
:1008e400250d0000d1f2000001f9000065050000ab
:1008f400890d000084ed00008af00000af060000be
:10090400dd130000ca0000009ede0000aa0e0000f5
:10091400f40d00007fef0000fef50000eaf4000093
:10092400311d00005216000025f4000013f70000ea
:10093400bcfd0000a10e000072f6000027ed0000cf
:10094400ca060000ff100000830b0000f5dd000064
:1009540034f90000651a0000e9f500005bf70000b7
:1009640045f20000e50b0000601f000043fa0000a0
:100974008ff6000053fc0000110d00004c03000032
:10098400dce70000d9fb0000820a00005a130000d3
:1009940070ee0000c8e80000a21a0000c0fd0000cc
:1009a4006cf200002ff6000011ff000098220000f6
:1009b400a5060000d2f3000017fa00004a03000065
:1009c400130900008cee00004cf80000dd0a000062
:1009d400571200001bfc0000fedb0000040e0000a8
:1009e400060f0000a3f10000b3fa000058f5000060
:1009f40004170000e1130000bbf4000012fb000028
:100a0400370000008d0d000009f80000c7ec00005d
:100a14000c030000860c0000670b000094e3000048
:100a2400d9fb000019190000a5f100009df7000092
:100a340067f60000b70a00001120000052fb000016
:100a44009cf6000069fb00006f060000e50300004f
:100a540068ed000099ff00003a0d0000820f0000cd
:100a64002fef00000ae50000c21600007503000025
:100a7400c6f40000a6fa00009ffa00004c1c000017
:100a840027090000dcf400005afc0000d902000031
:100a9400b40d000039f20000bff100004906000067
:100aa400490e0000b3000000e5e000002a0b00003e
:100ab400781100006af000006bf9000001f50000f5
:100ac400111500002f190000ddf60000ccf800001d
:100ad4007dfc0000cb090000abfc0000b5ee00007b
:100ae4002a040000020f0000700c0000bce50000a6
:100af40024f10000af17000002fa0000b7f900006b
:100b040028f900002b020000f51c0000ceff0000b5
:100b14001df6000009fd0000d0070000c509000013
:100b240014ed000015f600000e080000e90f0000a7
:100b3400d7f9000062e4000017100000f807000075
:100b44008cf20000d9fb000002f90000fc18000040
:100b54002611000071f4000060f9000058ff000045
:100b64003e0a00008af8000082f1000083060000bb
:100b7400e30f00002906000014e100006af90000f8
:100b8400d2150000a8f8000000fc00006df700007a
:100b9400ef0600005a1a0000e8fb0000bdf8000050
:100ba4003e000000aa0500007a010000b9ef000031
:100bb40065fc0000f50b0000220b000084ea000035
:100bc4007fef00009c180000c2fe000086f50000c4
:100bd40088f8000014fe0000e41c0000e306000096
:100be4001ef60000abfd0000150200002506000003
:100bf400c6f300001cf60000ff0600007810000099
:100c0400e8fc000022e30000db090000520a0000b7
:100c140015f400001afe0000e8f70000c9130000f4
:100c2400d41300004bf600002afa000080fe0000f6
:100c3400280900002cfc00002cf000009c0200009d
:100c4400240f0000660900002ee3000031f50000c7
:100c5400ad16000015fb000070fb0000fff600005d
:100c6400f5030000ee1b000017ff0000f8f700007a
:100c740013ff00001c04000033030000b3f1000064
:100c84008afa0000a00a0000500c00008dec00005d
:100c940068ed00007a170000870000003bf50000b3
:100ca400e6f800006cfc0000301c00008509000020
:100cb40077f6000033fd0000880000004b060000ba
:100cc4000ff6000037f500008d050000321000001b
:100cd400d5ff000003e300001c060000520c0000d6
:100ce40095f40000acfe000092f7000073100000c1
:100cf400f2150000b1f700002efa000005fe000016
:100d040032080000b7fe0000a2ef0000e6ff00007a
:100d14003c0e0000d90b000081e500005ff10000eb
:100d2400f016000072fd0000f1fa0000e6f6000083
:100d34000c010000eb1c0000740200006ef70000c0
:100d4400e9fd0000580200009004000062f4000075
:100d5400d3f80000d60800006c0d00009bee0000e4
:100d6400edeb0000e7150000c30100005ff5000093
:100d740033f9000020fb00005d1b0000de0b0000c7
:100d8400b3f7000061fc000047fe00001a070000f2
:100d940015f9000006f40000cb020000e00e00008c
:100da400ad0300008ee4000046020000260e0000a1
:100db40077f5000077fe000031f700004a0d0000cf
:100dc400bb18000003fa000094f9000033fd000092
:100dd400930500005c010000d4f00000c6fd000093
:100de400530f0000e30b000009e6000064f100006b
:100df400e11500001dfe000048fa00002cf7000079
:100e0400e6010000861c00009e020000eff70000cf
:100e140065fe0000430200005b040000faf30000da
:100e2400e4f80000e5080000f40d000049ed0000be
:100e34007bec000097180000eeff0000d6f40000e1
:100e440080f800000efb00009d1d0000080b000050
:100e5400c1f7000061fa000098fd0000390c0000a1
:100e640075f8000018f2000081020000ee0d000089
:100e7400ba04000044e400006d0300006e0e00009c
:100e840037f30000a4fd000016f60000db0e00009e
:100e94008a1a00004ff90000b7f60000b4f8000009
:100ea400210d00009b080000fae9000086f900000b
:100eb400140d0000a21000002fed00002de800002a
:100ec4006114000056030000e6f8000006f7000075
:100ed4000dfc0000cd1d000028090000cbf400002b
:100ee4006af60000370300005e13000064f400009b
:100ef40044ee000078040000fd0f0000a5fe000091
:100f04000ae2000069090000550f000075f50000b1
:100f14004cf9000076f300004914000008190000a1
:100f2400c0f9000090f5000068f7000067100000a9
:100f3400ee06000098ea0000e1fa0000ca0800008a
:100f4400c11000004df20000e8e700007c11000031
:100f5400ab010000d3f90000dcf9000004fb000041
:100f6400681c00009e09000019f4000025f600002a
:100f7400850300007f13000039f30000b8ec000083
:100f8400e5050000791100005204000086df00002e
:100f940007fe000096130000dcfa000068fa000067
:100fa40007f40000c70d000077190000dbfb000008
:100fb400dbf60000dbfb00007e090000e0ff000020
:100fc4008eef00002cff00000f0d00008a080000c7
:100fd400d2e300003ff7000045180000c7fa000004
:100fe400dbf80000daf30000e0040000321e000029
:100ff4006e01000044f8000014fb00005e030000d2
:101004008a0500003ff1000075f900003609000070
:101014007c0e0000f6f10000a8ea00005513000061
:10102400f00000001bf6000082f90000b5fb000090
:101034004e1d0000cf0a00003ef60000e3fa000057
:10104400bbfe0000b10a000079f70000a2f1000025
:10105400da0300006811000014ff000043e20000fe
:10106400ab0800009d0c0000f3f500009cfa0000a2
:1010740051f40000d9150000ff17000001f800002a
:101084009af8000001fb000083090000d5ff00006e
:10109400dfee000001ff0000530f00006c0a0000a7
:1010a400f1e20000daf60000831500004efa0000b9
:1010b400fffa00006df30000460700000c2000005a
:1010c40022ff00004df60000fff90000f8040000c4
:1010d4004107000035f0000002f90000da0a0000c0
:1010e4003c0f0000c4ee000081e900003b14000046
:1010f400f801000071f70000a9f8000000fc0000ee
:10110400d51d0000d009000008f500001efb0000fa
:101114007a0000008b0a0000bff50000c2f2000054
:101124004b0600003d10000019fb0000efe2000038
:101134006b0c0000780b000049f400000afb00006f
:101144008ff60000ad16000079140000e2f60000ee
:10115400b3fa00008ffc0000f7090000c0fd000096
:10116400fbee000094010000d90d0000b40600005d
:10117400aae4000091fc00004e14000006f60000f2
:1011840000fa000063f60000fd0a00006b1c00007a
:10119400a0fc000046f90000ddfa0000470500004d
:1011a400bb05000014ef000062fc0000620a0000ae
:1011b4001c0d0000c4ef000031ea00000615000019
:1011c40005000000f9f50000c4fa0000c2fd0000ab
:1011d400f01c0000370700007df60000f5fc00005d
:1011e4008bff0000fc080000d2f4000099f5000019
:1011f400330700005e0e0000b2fb0000d4e10000e3
:10120400be0b0000740c0000aef3000065fc00008f
:101214005af70000971500008b1200001df600001d
:101224003bfd00009ffd00006b0800009afc0000dd
:10123400c4ef000087020000310c0000f00700003a
:1012440071e400004bf900006f17000098f50000ee
:10125400b6f90000e2f7000003080000ce1c00000d
:10126400affb00006bfa0000d5fd0000e6020000b1
:101274009a0500004eef000093fa0000560a0000a1
:10128400320e000048f000007ee8000084160000e2
:101294005a00000002f40000b9fb00009cfc0000ae
:1012a4005e1d0000ea0600007ff600007d000000dd
:1012b400dffd0000960700007ef500005ff40000eb
:1012c400c60700002b0e000045fa000012e30000e0
:1012d400040f00007a0b000002f000000bfc000079
:1012e400abf800007a1700006f1100000bf6000045
:1012f400d0000000a8fc00005f050000cefb000049
:10130400e5f1000081030000b50b0000d4060000e5
:1013140010e4000066ff00004b150000dcef000045
:101324008dfb00003bf90000c50b0000ae1b000064
:10133400aef80000affd00007dfe00006301000078
:10134400b4020000c6f000004cfe0000310a0000a8
:10135400b80c00008aec0000bfee00005a18000030
:10136400e9f8000079f500002ffd0000a900000055
:10137400e21d00009e01000077f8000075020000e5
:10138400befd00001c0400009ef3000095f900005f
:101394001e090000da0c000054f6000014e60000f8
:1013a400a7140000ca03000074ee000043ff00000d
:1013b400fdfb0000291a0000230b00001bf50000b0
:1013c4000604000018fd0000fb02000017f80000ee
:1013d4004ff50000bc0600005f0c0000ec000000ac
:1013e400dee1000046090000731000008deb0000f0
:1013f40041fe000040fa0000f51100000016000054
:101404002cf40000ef01000099fe000035010000fb
:101414003cfe0000c8f00000490400000d0b000071
:10142400aa07000004e70000f2f60000511a0000c9
:10143400def10000b1f6000032fd0000f10600000c
:10144400051d0000a4f9000005fc00001e030000b7
:10145400d2fd00004302000066f100007cfe0000a3
:10146400530a00006b0b0000a8f200000fe7000015
:10147400421700002d000000f3ef0000f50000000b
:1014840063fd00001c1b0000a6050000ebf4000037
:10149400190600005ffd0000dd03000085f6000072
:1014a40061f60000b6080000b80a00006dfe0000f6
:1014b40052e20000560a0000c310000065eb000071
:1014c4001ffe0000e7fb0000e21100009213000081
:1014d4004bf30000270300008dff0000c70000004d
:1014e40070fd000095f100003c050000660a000054
:1014f400a606000075e6000027f70000191b00008f
:1015040006f1000033f700000dff00004a0500005b
:10151400611b0000a9f80000c2fc00009a0300004f
:10152400e8fc0000c5040000b9f10000c7fc00009d
:10153400410900009709000069f6000095e50000e4
:10154400301400002f0400004bee000007020000de
:10155400f7fb0000c6170000de08000074f400006a
:10156400e104000078fb0000ff050000f1fa000030
:1015740029f300004e060000a1080000b805000091
:10158400f9e300007cfb00004d17000043f100006c
:101594001dfd000023fc0000ef07000058180000a8
:1015a4006af60000e1fe000059000000c5000000da
:1015b40054050000a7ef0000acfd0000cd090000b9
:1015c400bd09000035f200002be70000da15000029
:1015d400e5020000d2f200002500000078fb0000c4
:1015e4009b180000060600002cf600009002000084
:1015f400e9fc0000d609000087f80000eaf00000ca
:101604009d070000830a000030030000bbe30000d4
:10161400cefb00003317000052f5000021fc00004f
:1016240031fa00008a08000036180000ecf70000c8
:10163400d5fb0000dcff0000ba040000ee0500004a
:1016440003ed000036fc0000430c00003e0a0000dd
:10165400ddf3000050e2000041120000030c000022
:1016640061f3000080fd00001afa00007817000002
:101674007a0a00007df20000c30000000e010000a1
:101684005e0a0000d7f80000a2ed0000190800006f
:101694004a0b0000b505000058e50000ccef00003f
:1016a400411d000070fd000019f7000056fb00000a
:1016b400d8020000141c00002afa0000c3f4000041
:1016c400100400003706000022080000bcec0000f3
:1016d4001ef70000e50d000028090000d3fa000001
:1016e4001ade000080070000aa1a0000b3f200000e
:1016f40023fa000098f90000e41000007a130000b7
:1017040078ef000098fd0000cf0500003c090000c0
:10171400f0fd0000efe9000058040000b40d0000e3
:10172400700300007bec000055e80000271b00005c
:10173400b5090000a2ef000070fb00007dff00006f
:10174400d319000079030000a8f00000d7030000bb
:1017540049060000e407000060f20000eaf000001f
:10176400160c0000490b0000060000001ce20000fb
:101774009ff70000511f00001cfb000066f50000ed
:1017840051fb00006b080000481800008df50000b4
:1017940003f70000a8070000c7080000b00100001c
:1017a400d1ea0000dffc0000180e0000570700001b
:1017b40007f700002ee00000760e0000411600003e
:1017c400a1f00000acfb000034fc00003e1300005c
:1017d400c40d0000daee00006b000000b207000048
:1017e4003c080000edf9000071ec0000c0060000a8
:1017f400f60b00007703000063ec0000c1e9000071
:101804008e1b000036080000cff00000eefc000044
:1018140013010000a4170000fe0000008ff1000077
:101824001b060000e3070000db0400008ef100004b
:10183400b1f30000550c000074090000b9fe00006b
:1018440010e5000069f80000a11d00005dfc000027
:10185400f7f4000096fd0000700700001415000066
:10186400b8f7000081f70000ca080000a0070000d4
:1018740084ff00009ced0000dcfc0000c90d0000aa
:10188400a00600008af60000b5e20000e4090000aa
:101894008d1800000df4000034f9000003fe000070
:1018a400320e00006d0e0000c6f20000aefe000015
:1018b4000e09000029050000abf8000074ef0000d9
:1018c4006b050000290c00001003000091ed0000de
:1018d4001ae90000561700005d0c000082f10000b8
:1018e400ebfc000036000000e2120000b00400002f
:1018f4005ff200006904000056080000460300007f
:10190400f5f3000039f30000b90900000e0a0000e5
:101914008afe0000f1e60000cef30000ae1d0000d8
:101924002202000013f200007afd000049040000c6
:1019340080140000fbfc000000f5000075070000a7
:1019440041070000c3ff000043f10000cff800008e
:101954000b0c000008080000e6fa00007ce500001b
:1019640000fd0000281c0000fbfa00001df600002a
:10197400b2ff0000d5060000d7110000c4f7000034
:1019840040f80000d209000063060000b9fd000021
:1019940025f0000036fc00008b0d0000040600005a
:1019a400a0f400002ee400006e0800001a1b0000e2
:1019b40093f5000000f80000fffe0000330a000069
:1019c400d20f000062f4000019fc0000730a00004a
:1019d4006e040000cdfa0000bbf00000910000008e
:1019e4006f0c0000850400003cf00000b7e6000026
:1019f400e2120000eb1200000af2000069fc000091
:101a040094fd0000d90e00001b0c00008df10000b5
:101a14000f0000008d080000d004000029fa000027
:101a24000ef00000690300007a0b0000880100003a
:101a3400c6ec0000a1eb0000e41800007e0c0000de
:101a4400acf1000019fd000099fd00000513000031
:101a5400bf07000018f10000ab020000e20700001d
:101a640039030000aef600001cf300006907000013
:101a74001e0a00004fff0000adea00002bf000003a
:101a8400c61a0000f90600001bf400003efe000028
:101a94009cfe0000111400002d02000082f20000e0
:101aa40016060000a2070000f9010000caf30000b6
:101ab40021f500003c0a0000ba08000071fb000098
:101ac4000ae7000026fa00005a1d00004cfe000040
:101ad4006af50000effd00003e030000e61400007c
:101ae4006cfb00007ff50000030800008c0600007a
:101af40022000000b6f100006cf90000230c000085
:101b0400fb060000bff60000a4e40000f30400009c
:101b1400121c000008f8000080f70000f3fc00002d
:101b24006b080000f21200003df600007ff900008f
:101b34002e09000099050000c1fc000081f000009e
:101b44006afe0000550c00002505000057f2000055
:101b5400cae50000660f0000c015000029f300006c
:101b640040fb0000d5fc0000640d0000cc0e00001a
:101b740043f20000fbfd0000a00800004005000047
:101b84005afb0000c7ef0000d7010000ca0b000099
:101b9400680200007dee000099e900008b16000049
